:020000040000FA
:1000000000F8020269340000F50F0000A1110000A1
:1000100000000000000000000000000000000000E0
:1000200000000000C0DF000008E00000F50F000045
:100030000000000000000000F50F0000C5350000C2
:10004000E90D0000F50F0000F50F00008D340000F1
:1000500059120000B5310000850F00002510000086
:10006000810C0000BD0B0000F50F0000F90F00002F
:100070002D1200003D390000093400003534000025
:10008000F50F0000F50F0000F50F0000ED35000042
:100090000D360000F50F0000F50F0000F50F000011
:1000A000913600009B360000EB0D00001D33000070
:1000B000F50F00001D3200000000000000000000ED
:1000C0000348854600F04AFD004800479973000048
:1000D00000F8020230B50B46014600202022012420
:1000E00009E00D46D5409D4205D31D469540491B6C
:1000F0002546954040191546521E002DF1DC30BDB5
:1001000070B500242546002801DA01244042002968
:1001100001DA01254942FFF7DDFFAC4200D0404241
:10012000002C00D0494270BDF8B5002425460029B6
:1001300004DA0E46012400214042B141002B04DACA
:100140001E46002352420125B34100F003FC8C46B9
:1001500017461E46AC4203D0002540428D41AC46B6
:10016000002C02D0002657429E4161463A46334653
:1001700001B0F0BD03460B439B0703D009E008C95B
:10018000121F08C0042AFAD203E00B780370401C47
:10019000491C521EF9D27047D2B201E00270401CD5
:1001A000491EFBD270470022F6E710B513460A46F7
:1001B00004461946FFF7F0FF204610BDF8B5024689
:1001C0004A40D40F42004B0052085B089A4202D2C8
:1001D0000246084611464A0023D0C30D4A00DDB24C
:1001E000120EAD1A202D35DA49020126490AF6050C
:1001F0008A19002C00D0524220214F1B1146B940D1
:100200002A411018C20D9A4221D0002C17D0012D7E
:1002100008DCDA05801AD20F8019D207DBB200F0B1
:1002200005FCF8BDDA05801A012340001B06C01842
:1002300080185A428018CA0F1043490007E0490845
:10024000C2071143DA05801A80194008801800F0AF
:10025000E5FBF8BD61000122511A001BF7E70122FE
:10026000D2075140AAE70122D2075040A6E7024632
:1002700070B54A40D30FDB0740002DD04A002AD08A
:10028000010E140E000212020919400A520A8418C3
:10029000E50104465443000A120A2E045043A419EF
:1002A0004219200CC543AA18120C0125AD03521C9B
:1002B000521912047F39240400D0521C104301D477
:1002C0004000491EC2B20C06C0092018401C40085C
:1002D000802A02D003E0002070BD400840000029C1
:1002E00000DA0020184370BD70B502464A40D50FB1
:1002F00040004A00ED0740085208002814D0002AA8
:1003000012D0C40DD30D41020120C0055202490A8A
:10031000520AE41A091812187D34914201D3641C60
:1003200000E04900002C01DA002070BD002391425A
:1003300001D3891A0343400849000028F7D1002956
:100340000AD0914202D10121C90705E0914201D2B0
:10035000012101E00121C943E005C018401900F066
:100360005DFB70BDF0B507460846584087B0C00F2A
:10037000049048000E46590040084908BC1A8841BC
:1003800005D2384631461E4617460B4602465800EF
:10039000400810434CD0300D039040055900400DEB
:1003A000490D0590401A0290402872DA1803012185
:1003B000000B09050843019004980092002805D01D
:1003C00001995242002088410092019002984021F8
:1003D0000A1A0199009800F0EDFA05460C466B46A2
:1003E00007CB00F008FBC0197141039A0E0D0023E2
:1003F000D71756401A467A40164344D0049A002A2A
:100400002DD0029A012A039A15DC1205C01A9141D7
:1004100001263605001C7141D20F059ED2070093BC
:10042000019202962A46234600F046FB07B0F0BD33
:1004300038463146FAE71605224A0F46B218C01A66
:10044000B74101210905001C4F4100187F411146A9
:1004500018187941E20F10436D19644113E0E20767
:100460006D0815436408C2071443039A0126120558
:10047000C01A91413605001C7141CE074008304337
:100480004908C01851412A46234600F008FBCDE731
:10049000FFE7049801224000C117121A00238B4184
:1004A00004983146C417381AA141EEE730B401244C
:1004B000E407634030BC55E730B40124E4076140F1
:1004C00030BC4FE70000E0FFF0B51FB488B00B99D7
:1004D0000998002448400999C00F4900490809912A
:1004E000C0070B990090490049080B910999089899
:1004F000A64608431CD00B990A98084318D00998BF
:1005000001244000420D4800410D099824050003D4
:10051000000B204309900B980003000B20430B9025
:1005200050181C494018002201901446104605E05E
:10053000002001460DB0F0BD032801DA034600E0BB
:1005400003239C46C11A0AAE0AE05F0008ADED5BCA
:100550004F00F75B7D430027AA187C41491C5B1EB6
:100560006145F2DD410004AB5A522104120C0A43EA
:10057000240C401C0828DFDB01980290009970468B
:1005800001910090059B049A0799069800F094FA4F
:10059000D0E700000DFCFFFFF0B50C465C4085B0D5
:1005A000E40FE40703944C000026640859009446C5
:1005B000490802460296224321D062460A431ED0D1
:1005C0006200570D4A000E032303550D0124024615
:1005D0002C492405781B1B0B360B4018234326435C
:1005E000614600901C46501AB44103D30098401C49
:1005F000009002E0921800985B41002803DA002086
:10060000014605B0F0BD00200121090507468646D8
:1006100011E064461D46141BB54106D36546521BC6
:10062000B341744607430C43A646CD07400849082A
:10063000284392185B4105460D43EAD11046184302
:1006400013D06046194650407140084306D06046BA
:10065000101AB34106D20122002306E00022012332
:10066000DB0702E00122D2435310009874460105D3
:10067000381C6141029C039D0019694100F00FFA8A
:10068000BFE70000FD0300000122D207002800DBC5
:10069000101A002900DB511A814201D8012070474D
:1006A000002070470122D207002800DB101A002921
:1006B00000DB511A814201D20120704700207047AF
:1006C0000122D207002800DB101A002900DB511A92
:1006D000814201D301207047002070470122D207D8
:1006E000002800DB101A002900DB511A814201D9D1
:1006F00001207047002070470122D207002800DB4C
:10070000101A002900DB511A814201D101207047E3
:100710000020704710B5002904DB0C460121C907F1
:100720004042A141002B04DB1C460123DB0752425F
:10073000A341801A994101D3012010BD002010BDB2
:1007400010B5002904DB0C460121C9074042A14134
:10075000002B04DB1C460123DB075242A341101A85
:100760008B4101D3012010BD002010BDC217C10F65
:10077000504010B54018CA079623002100F056F9E2
:1007800010BD10B500229623114600F04FF910BDA0
:100790000EB5C217C10F5040CA0740180021054BC3
:1007A0000293019200910A460B4600F085F903B0CE
:1007B00000BD0000330400000EB505490291002180
:1007C00000910A460B46019100F076F903B000BD96
:1007D000330400003EB5CA17CB0F002450405140EF
:1007E000C0186141DA07054B02930192009422463A
:1007F000234600F061F903B030BD0000330400006F
:10080000C20F410040020123400ADB05D207090E56
:10081000C0187F2901DA00207047962903DC96234F
:10082000591AC84001E096398840002AF4D0404265
:100830007047410040020122400AD205090E80188B
:100840007F2901DA00207047962903DC9622511A8D
:10085000C8407047963988407047000070B5CD0F8A
:100860004A0009030123090B1B0519430B4BED0734
:100870000024520D9A4201DA002070BD074B343338
:100880009A4203DC9A1A00F0A5F802E004495118D4
:1008900088402C43F1D0404270BD0000FF030000AF
:1008A000CDFBFFFF70B5CD0F4A0009030123090BF3
:1008B0001B0519430D4BED070024520D9A4202DA35
:1008C0000020014670BD094B34339A4203DC9A1A6A
:1008D00000F080F803E0064BD21800F06BF82C43D0
:1008E000F0D0002240428A41114670BDFF03000053
:1008F000CDFBFFFFC20FD207400040080BD0C10D57
:100900000723DB01C91840020905400A1143C20848
:10091000400711437047002001467047CB0FDB07AB
:10092000490010B5490802460A4307D00A0D0724BA
:100930000903E401090B121B002A01DC002010BD91
:10094000C900440F0C43C100E018D205801800F024
:1009500065F810BDF0B51FB40646002082B005460C
:100960004024019100901BE0019922460F46304639
:1009700000F030F8049A059B801A994110D3104674
:100980001946224600F016F8361A8F410197224682
:1009900001200021009F00F00DF838184D41009013
:1009A0002046641E0028DFDC019B00982946324661
:1009B00007B0F0BD10B5202A04DB0146203A914073
:1009C000002010BD914020239C1A0346E3401943A8
:1009D000904010BD10B5202A04DB0846203AD040D4
:1009E000002110BD0B46D340D0402024A21A9140D4
:1009F0000843194610BD10B5202A06DBCB17084660
:100A0000203A1041C1170B4306E00B461341D0407A
:100A10002024A21A91400843194610BD002904DA87
:100A2000401C490001D140084000704770B40024C8
:100A3000050C05D11024000402D1002921D0112475
:100A4000050E01D100020834050F01D10001241D5B
:100A5000850F01D18000A41C002801DB4000641C2C
:100A6000002908D020252E1B0D46F540A14000D0BE
:100A700001212943084301061B1B000ADB1D02D587
:100A8000002070BC7047DB05181880180029F8DAC0
:100A9000401C4900F5D170BC40084000704710B5BB
:100AA000002B08DA0024401C614192185B411A4374
:100AB00001D14008400010BDF0B51FB482B005461A
:100AC0000C0003D008460BF05BFA02E00BF058FA7A
:100AD00020300246009021462846FFF76BFF049B1A
:100AE000059A04460F4618431143084314D018468C
:100AF00010431BD0009840210A1A18460599FFF7A9
:100B000069FF05460E46009A05990498FFF752FFC3
:100B1000084305D0012004E02046394607B0F0BD67
:100B20000020C11705430E432C43374300990E980C
:100B30006305401A7905E40A00220C43FD0A0A30D5
:100B400002D500200146E9E70105101969410C9C16
:100B50000D9D00196941FFF7A2FFDFE7064C012553
:100B6000064E05E0E36807CC2B430C3C9847103455
:100B7000B442F7D3FFF7A8FA84DA0000A4DA000041
:100B800030B58C180278401C13071B0F01D1037875
:100B9000401C120906D10278401C03E005780D7054
:100BA000401C491C5B1EF9D101E00B70491C521E10
:100BB000FBD1A142E6D3002030BD000010B5214892
:100BC000016A8A0715D44A0715D4C90732D01E49CD
:100BD0008A89002A15D0531E8B8182688C6904C4CF
:100BE0008C610A691B040DD0002A22D10121016009
:100BF00010BD022100E00421C16113488021416140
:100C000010BD0A69012A09D1026801239A430260D2
:100C1000C361FF20683099300C4A106001204861A0
:100C2000CA69002A05D0886909898B00C01A9047D3
:100C300010BD10BDFF226832054806A109A308F0C7
:100C4000F3FFC04608D001402095010280E200E099
:100C500028CA00004144435F49525148616E646CA8
:100C600065720000556E6578706563746564204137
:100C7000444320696E746572727570740D0A0000C9
:100C800070B582B000230193444801688A6A4C68B9
:100C900013252540132D02D1CB689B07DB0F436141
:100CA000930772D453070AD4D30711D1130724D55D
:100CB000048F838E1C1B102C0EDD102310E00420EB
:100CC00088620220032142A209F0DCFF02B070BD5D
:100CD0000120886202B070BD048F1B1B1C0610D05F
:100CE000DBB20024058FC66A75192D5D0D74641C76
:100CF000A342F7D1048FE3180387D20607D400215B
:100D00002FE04B6A0824A3434B62D206F7D5CB6889
:100D1000C28E448F141B5B04DB0EA34201D3438FAE
:100D2000D31ADAB2002A16D0097D438F046BE1543E
:100D30000199012A10D001231C46890145582D7DB7
:100D400041184E8F9B19096BCD54641CE3B2019975
:100D50009A42F2D800E000218B01C3185C8FA218E0
:100D60005A878A0181184B8FCC8EA3420BD3012363
:100D70000B61805800224262CA6B002A03D03A31CC
:100D8000098801A8904702B070BD0220886204481B
:100D900004A1084A08A308F047FFC046409001029A
:100DA00041CA00004145535F49525148616E646C2D
:100DB00065720000CE02000041455320696E7075D7
:100DC00074206F766572666C6F770D0A0000000004
:100DD000414553206F757470757420756E6465722B
:100DE000666C6F770D0A000070477047F0B587B0EA
:100DF00050480068FFF7CCFC04460D464E48406A58
:100E0000FFF778FD02460B4620462946FFF7C4FB54
:100E100002460B46002449492046FFF747FB039052
:100E2000029101200590400201904549454F06E09E
:100E3000534A10517F1C891C241D642C78D03878AB
:100E400005284148F4D10497069140480159404E85
:100E5000316240480359B3613F480059B0623F4A8C
:100E60001259326300275D1A3564736AF16999413A
:100E7000059B00DB3B46002B01D0019BC918344E7B
:100E80007164F36A716B101A9941059A00DB3A4656
:100E9000002A01D0019A8918FFF79CFC02460B46F4
:100EA00003980299FFF710FBFFF7FCFC284A9063B8
:100EB000D163401BC10F4018401010601546FFF76A
:100EC00067FC274A274BFFF7FFFAA864E964264A24
:100ED000264BFFF7F9FA3A46254BFFF7F5FA3A4663
:100EE000244BFFF73FFA05460E461948056141615C
:100EF00028463A46204BFFF70DFC00280699049F30
:100F000098D10022284631461C4BFFF719FC069960
:100F100000288FD1088800B2FFF73AFC02460B4642
:100F200028463146FFF71EFAFFF798FC06997FE73F
:100F300007B0F0BD089701023CC000000000F03F80
:100F4000C898010234970102FFFF0100FC980102DA
:100F5000589601026099010218B401027CB40102A2
:100F6000699006699006903F52257997532ED33F9A
:100F70000000594000003E4000408FC0006AF84029
:100F800040A70102B0B582B0194C2068056801A9DC
:100F90000020087007E090470198401C01A90870E4
:100FA000C0B2082822D2012211048140294209D06E
:100FB0002268516080002018826A002AECD001A8C3
:100FC0000121E8E7130283402B4201D0022104E013
:100FD00082402A42E0D003211346226853608000F9
:100FE00020188268002AD7D001A8D4E702B0B0BD8B
:100FF00090920102FEE7000010B509480168CA6935
:1010000020231343CB610269032A08D101229305EF
:101010000C689C430C605102C26E0A43C26610BD4C
:1010200000930102F0B581B05C4C2068856BE80745
:1010300007D0E168002904D00020884720680121FA
:101040008163A80707D52169002904D001208847BA
:10105000206802218163680707D56169002904D0EF
:1010600002208847206804218163280707D5A169E9
:10107000002904D003208847206808218163E806FE
:1010800007D5E169002904D0042088472068102191
:101090008163A80607D5216A002904D00520884766
:1010A000206820218163680607D5616A002904D081
:1010B00006208847206840218163280607D5A16A59
:1010C000002904D0072088472068802181630126F9
:1010D000E80507D5E16A002904D0370208208847CF
:1010E00020688763A80507D5216B002904D0770203
:1010F0000920884720688763680507D5616B002948
:1011000004D0B7020A20884720688763280507D5DE
:10111000A16B002904D0F7020B2088472068876361
:10112000E80407D5E16B002904D037030C20884779
:1011300020688763A80407D5216C002904D07703B1
:101140000D20884720688763680407D5616C0029F3
:1011500004D0B7030E20884720688763280407D58A
:10116000A16C002904D0F7030F208847206887630B
:10117000E80307D5E16C002904D037041020884724
:1011800020688763A80307D5216D002904D0750462
:10119000112088472068856301B0F0BD809301026B
:1011A00004217046084204D0EFF30983EFF308826C
:1011B00003E0EFF30883EFF309829BB004A8F0C0CB
:1011C00044464D4656465F4608A8F0C01846F0C84B
:1011D0006846F0C018690C90202018440D9058699A
:1011E0000E9098690F90D8691090EFF310801190CD
:1011F000EFF31480129009490868139008490868B1
:1012000014900849086815900749086816901793C4
:10121000189270461990684608F020FF04ED00E02F
:101220000CED00E010ED00E014ED00E080B50748A3
:1012300001210170064802680A43026005480268FD
:10124000002A02D000200146904780BDFAA6010284
:101250001C100050FCA60102F0B599B0F548017BC6
:10126000C67A427B0E92F44C221F1368F34A12682E
:10127000069242780C9202790592C76A04931F4045
:1012800001200F907A0200D5BCE03A0200D5BFE001
:10129000FA0102D50F9802062260502508968A1995
:1012A0001826BB0102D50F984306236041230795FA
:1012B00069430A96354655431426FC0210D50F980B
:1012C000040538463746DC4E3460DA4CA469B46411
:1012D000D84CE4697464DA4C241D34603E460746F9
:1012E00090000B90D8040D90681809900E9B7343E2
:1012F0000F988203B902D04D22D50F98410529607D
:10130000CC480E961646024681692965C169696511
:1013100009990D9801430898000108180B99401885
:10132000C018C849098892794A4380180A301C4677
:1013300003F0E8FB234632460E9EC04988672A60C8
:101340000F98C404380300D52C60F80302D50F9819
:10135000000428600F984104B80300D529603804C0
:1013600000D4E4E1039402910E9308920D980B9936
:101370000C180A980C9941430C910F98C0030B90DC
:10138000286006F07BF9002801D003F09DFB0C9843
:10139000005B410B43D1099800190E99401805993B
:1013A000090140180E90E74D287B079B4343E97ADB
:1013B0000A010D9C2243D21841188B00D2180A9BB7
:1013C0004B43D1186A7B564389190E9E2A7910180F
:1013D000DF4A12884243881816903068C000800D9A
:1013E00010A9C882002511957079C0077ED110A878
:1013F0000F998182069C00940020E8A2049B09F0CA
:1014000041FC78E00F98820522603A0200D43FE761
:101410000F98C2052260FA0100D53BE73DE707219E
:1014200049030840032149038842089A00D07EE11D
:10143000069705F003FE0020169009901590C14C08
:10144000E07A217B08180A99414380000D9A1043E5
:101450004118627B0E9672438A186178A379079EC1
:101460007343D718FA683F26324063789A420C9744
:101470006ED105960A9A4A4380580F210A07024006
:101480000398401EC04B1B68DB090340981810905E
:101490000F98C0020B90B868800767D42C46283C90
:1014A00008F094FB05462068000609D5C320840196
:1014B000786A400704D408F089FB401BA042F7D9A2
:1014C00005980002B96849080140B348036882687A
:1014D000B868C40C20202040DB0700D095E0002332
:1014E00010221D461C460E9E0B9FB1E010A885825F
:1014F000B0681190069C701D924B1979E20707D1D4
:10150000491C1971D97A1A798A4202D31D7100E0F7
:10151000D970017842781202511882781204891821
:1015200003229143017035715878401C5870D87A65
:10153000197B08185978884200D85D70D879401E08
:10154000D871596B002901D010A888477E4DEDE075
:1015500010A80B998182F8683040637800900020D1
:101560007CA20F9909F08EFB0E9E94E0388A874A80
:10157000024010A8C2822022BA5C9307DB0F3C68AD
:10158000C3720F9B1A4082726205D20C0D9B1A43E4
:101590001692FA68130E0372BB69FC697C4D2D68C4
:1015A0002D0C05745204920F427211931394654CE2
:1015B000A07B002809980E9E0B9F5FD0754800689D
:1015C000007A0328099859D00C98007D0840092812
:1015D000099853D1C320840108F0F8FA05460C9805
:1015E000406A41070BD4594909680906890F06D199
:1015F00008F0ECFA401BA042F1D90C98406A410374
:101600000898884310A9888237E0D2070E9E0B9F66
:1016100003D108230022154619E00C9B9A68029C0E
:10162000224211D19A68520C02249443002213469C
:1016300015460DE004A7010228A000503CA100506F
:10164000FC1F000000A701020425002213461446D7
:101650000843104318432843204310A98882384286
:101660000BD10C9B198A494A0A4010A9CA821968F1
:101670004905C90C0D9A11431691324C2921615C20
:10168000002908D03037B84205D010A908461130DB
:10169000123107F0CFFBE77A2A48047BE519294885
:1016A00000790E9027484078401C2946FEF712FD2D
:1016B00088000D9A10431890079961433801104330
:1016C00040182049497B4E4380191C21694340182A
:1016D0000E9909191B4B1E4A12884A43801817900D
:1016E000099A0C998A60987B002800D04A62987900
:1016F000401C9871187B99798142069F00D39A719A
:101700005978491C5970D97A0818597888420E4D71
:1017100000D85A70187A401E18722820185C0028C9
:1017200004D0996B002901D010A88847089A174265
:1017300002D00F98000328601C480449486019B083
:10174000F0BDC04604A7010228A000503CA10050F3
:1017500000A7010248572045542069647820256479
:1017600020616E64204554206964782025642069D6
:101770006E2052582064657363206D69736D6174C7
:1017800063680D0A0000000038200040FF030000DD
:1017900094300040E8930102604000404D414320F6
:1017A0004556542025782025780D0A00FFFFFF03B9
:1017B000F0B5A5B01E460C9208910024239422A9EE
:1017C0000C8016A90C8024A909250D80598C0D9137
:1017D000FEF780FC2A99012900D0DFE03189012938
:1017E00000D0DBE0318C012900D0D7E00D99002931
:1017F00000D1D3E0224607962C990B912B990691A4
:1018000080B205900F9415A8058090000E900C9959
:101810000C582E460025204629461746FEF734FF71
:101820000028119636D12C200A9778430899081879
:1018300017A90A4668C868C2E8C8E8C2E8C8E8C28A
:10184000079F119880B280000E5822AD019523A801
:10185000009020463946059A069B02F0D5FD0F9868
:10186000401C0F90288800282DD03B8A239913AC68
:10187000039416A8029014A8019015AE009617A81C
:1018800024AA02F09BFF2588308811900120149E25
:101890000A9A05E013A8058014952E4628463A4674
:1018A0000E9F51000B9B119C5C52591808830D84AC
:1018B000D81986600F981885521C0D9882426DD0F9
:1018C00024A805889FE7099616A800250580149589
:1018D00024A80688239812902F46109503E06D1CCB
:1018E000A8B2B04213D8A8B2800017A90C5820465D
:1018F0001299FEF7D7FE0028F1D1002FEFD115A8DD
:10190000058016A80127078014941094E7E715A80E
:101910000288B01A012805D115A80680099F1497DE
:10192000119628E010200799095E0129119221DB08
:10193000551CA8B20C18109F0E9B099403E06D1C57
:10194000A8B2844218DDAAB2B242F8D8800017AA21
:1019500010581090394634461E46FEF795FE334621
:101960002646099C0028EAD115A80580109F1497E7
:101970001195E4E7109F0E9B1C463E46384612998F
:10198000FEF7B2FCFEF73CFF0546052800D305250F
:1019900013A8058001200A9A274682E725B0F0BDEA
:1019A000F0B58BB00243159A149C139E2BD00546BC
:1019B00001A856C0129CD869196A09900A911E465E
:1019C0009F6B0123009309A807AA0146059304F021
:1019D0006FFD716C3846FEF787FC0746E06A616B65
:1019E000FEF782FC002D069613D00446119801994B
:1019F000012924D10921081A0421069A515E88423E
:101A000029D16425B1E000203080207010700BB027
:101A1000F0BDB08800226425002829D005926949CC
:101A20003846FEF75BFE0028049C039E6FD1664992
:101A30003846FEF753FE00281DD05A2567E03C25A6
:101A4000082800D191E05F492046FEF747FE0028B4
:101A500019D0502589E00A291DDB1D293BDC594995
:101A60003846FEF73BFE0022002854D05A253AE0C3
:101A70003346049C39E055493846FEF72FFE0028CE
:101A800021D0502543E050492046FEF727FE00288C
:101A90002ED0462569E03C25012866D049492046DC
:101AA000FEF71CFE0028D4D147492046FEF716FE5B
:101AB0000028EED145492046FEF710FE002854D1FB
:101AC000434920466EE042493846FEF707FE0028AB
:101AD0001CD128251BE03B493846FEF7FFFD0022BC
:101AE000002832D05025049C069B0299039E41E0B9
:101AF00036492046FEF7F2FD002836D1344920460B
:101B0000FEF7ECFD00282FD114252EE03725029991
:101B1000059A069B2EE005922B493846FEF7DEFD1E
:101B2000002896D129493846FEF7D8FD0028B0D1C3
:101B300027493846FEF7D2FD0028049C069B0299EF
:101B4000039E059A3BD11E2514E005921E49384696
:101B5000FEF7C4FD00289CD11C493846FEF7BEFDA7
:101B600000281DD03C2500E02325049C069B0299FB
:101B7000039E059A25803270002008703078002876
:101B80000CD118681349FEF79BFD002806D1208868
:101B9000102803D30F3820800BB0F0BD0BB0F0BD80
:101BA0000B493846FEF79AFD0028049C069B0299D3
:101BB000039E059A01D11425DCE72325DAE72D25BC
:101BC000D8E7C046CDCCCC3DCDCC4C3DCDCCCC3CEB
:101BD0000AD7233C0000204070B588B00C4606466A
:101BE0004088002820D0FEF7CCFD059005A804A968
:101BF00001252A4604F0C6FE3088B188081AFEF78F
:101C0000B5FD0390049903A807AA2B4604F07AFEB9
:101C10005249079D2846FEF761FD002808D0BF20E5
:101C20000006206008B070BD0020206008B070BDC4
:101C30004B492846FEF736FD002804D03F20000619
:101C4000206008B070BD47492846FEF747FD0028D0
:101C500001D0002010E000212846FEF73FFD0028BB
:101C600001D0022008E040492846FEF737FD002851
:101C700001D0042000E0062001957F21C9050291D2
:101C800080003A49091801A806AA022304F0EEFDD3
:101C90000698206008B070BDF0B587B00C460546C8
:101CA0004768002638463146FEF726FD002802D058
:101CB000266007B0F0BD049704A803A901263246A8
:101CC00004F060FEA8682968FEF7C9FA029003993B
:101CD00002A806AA334604F015FE2049069D2846B0
:101CE000FEF7FCFC002804D0BF200606266007B0E3
:101CF000F0BD1B492846FEF7D5FC002804D03F2044
:101D00000606266007B0F0BD16492846FEF7E6FC39
:101D1000002801D0002010E000212846FEF7DEFC5C
:101D2000002801D0022008E00F492846FEF7D6FC23
:101D3000002801D0042000E0062000957F21C9057D
:101D40000191800009490918684605AA022304F098
:101D50008DFD059E266007B0F0BDC046CDCC0C3F82
:101D6000295C0FBFCDCC4C3ECDCC4CBEF0930102D4
:101D7000F0B587B00C4606467F270088002801D0C2
:101D8000FD0503E0B08800282ED0334DFEF7F9FCA6
:101D900003907088FEF7F5FC049003A802A90126C1
:101DA000324604F0EFFD029904A806AA334604F077
:101DB000A9FD2A49069E3046FEF790FC002802D075
:101DC0003F20010641E026493046FEF76BFC002823
:101DD00002D0BF20010638E022493046FEF77EFCE3
:101DE000002805D0002024E00020206007B0F0BDCE
:101DF0001D493046FEF772FC002801D0022018E091
:101E00001A493046FEF76AFC002801D0042010E091
:101E100017493046FEF762FC002801D0062008E092
:101E200014493046FEF75AFC002801D0082000E093
:101E30000A200096F905019180000F4909186846AB
:101E400005AA022304F012FD05992846FEF70FFAB1
:101E5000206007B0F0BDC046000080BF00003843DE
:101E60003333733F0000C84200007042000020423C
:101E70000000A0410000C04010940102F0B59DB0E8
:101E800015460B917F210391C9051C9102911B916D
:101E900019A900248C80199418941794598C0691D0
:101EA000198C0F91DE8B998B0791997805911F887A
:101EB0002B21CA432799914201DB7F0015E0402284
:101EC000D243914211DC4922D243914202DB79088C
:101ED000CF190AE05322D2439142EEDA5D22D24377
:101EE000914201DBBF0000E0FF000A971396269E97
:101EF000597E00290BD0002132460F46D1709170D7
:101F000051701170121D7F1C5C7EA742F6D30C939A
:101F100011952599149122990D91159041088C42A3
:101F200011D2FD4A2346A00084583454270A451C88
:101F30007755250C871CF555240EC01C34545B1CAA
:101F40009CB2A142EFD823981090012009900090F4
:101F500030463146149A159F3B4604F0B7FA0D9867
:101F600000060890400E139D00D186E068000490A2
:101F7000002F3FD0002210461146144606E01C46B2
:101F80001146159F401C82B2BA420ED283B2AB42B8
:101F9000F8D09200149B9A5E0FB2BA42034600DC5E
:101FA0002346BA42EBDC0A46E9E7002F25D000229F
:101FB00010461146129206E012931146159F401CDE
:101FC00082B2BA4214D283B2AB42F8D0A5B2AB42CD
:101FD0000CD09200149B9A5E0FB2BA42034600DC0A
:101FE000129BBA42139DE7DC0A46E5E7139DE6E73C
:101FF000129903E00024214600E00021129110987C
:102000000183C4828582049FF057FEF7AFFB7921DC
:10201000C9050E91FEF72BF91099C861099807437D
:10202000F057FEF7A3FB0E99FEF721F9109F3862D7
:102030002004C40B3057FEF799FB0E99FEF717F9F1
:102040007862601C3056FEF791FB0E9C2146FEF72D
:102050000EF9B86212980004C70BF057FEF786FB22
:102060002146FEF704F9109CE062781C3056FEF71A
:102070007DFB0E99FEF7FBF82063119805800C9804
:10208000407E410000278D4228463A46149E1ED3CA
:102090000A9880B28AB29300F45E84420BDA491C3B
:1020A0008AB2AA42F6D9002728463A4681B2691A6E
:1020B000012910D01BE0F018119B19800788080433
:1020C0000FD0500040008019001F0288084681B2DE
:1020D000691A01290BD1A800301811990D800788C1
:1020E00026E00020024681B2691A0129F3D00A993C
:1020F00089B2079B4B43BB421AD306998A4217D831
:102100000599002914D0401C82B2891803E0401CB4
:1021100082B291420CD983B2AB42F8D89200B35E3E
:10212000BCB2A342F3DDB218119B18801788EEE70A
:1021300012970B980580119800882B1A002B16DD3A
:1021400002210F9A1143032942D10E93411C421ED2
:1021500010B281420EDA0E98032824DB0C98808C92
:10216000012820D019A818A9FFF736FD1FE000208C
:1021700018902BE00026F443374608E0B8B2400040
:1021800019AD2B527F1C521C10B28142E3DB13B2FB
:10219000A3423346F2DD159B98423346EEDA8000C7
:1021A000149B1B5AEAE719A818A9FFF7E1FD149E32
:1021B000139D0F9A012A13D0032A11D0022A04D1A9
:1021C00011980088281A02280ADA0020179034E0B3
:1021D000022A01D1022BB8DA00201890012AEBD193
:1021E000681C691E0FB2B84208DA0C98808C01286E
:1021F0001DD119A817A9FFF7BBFD1CE00022D3438E
:10220000144608E0A5B26D0019AF7E53641C491C4A
:102210000FB2B842E9DB0DB29D421646F2DD159DC4
:10222000AF421646EEDABD00149E765BEAE719A8C7
:1022300017A9FFF7D1FC149E139D249F189C179992
:102240002046FEF70CF80F99012900D82046386087
:102250000D98002800D1CBE011990888109FB8860E
:102260000888281AB880129880B2FEF78AFA792175
:10227000CC052146FDF7FBFF2146FDF7F8FFB863CB
:10228000119F3888002849D081008919091F0988C1
:10229000129C0C191599884203D2800080198088FD
:1022A000041915984300534916AA304604F0ECFA75
:1022B000169810994864FEF7BCFAA4B2A04201D166
:1022C0004D480FE0001BFEF75CFA1C901CA81BA9F0
:1022D000012204F057FB2046FEF753FA01461B98F3
:1022E000FDF7C5FF109908603988491B4A1C92B256
:1022F000032A02D20021159F17E009B20229159F77
:1023000012DB3F210906FEF7E9F9002802990CD1FA
:102310000998810709E0C046402100400020129C36
:1023200015998842B9D3BCE73449109801610898DF
:10233000800E5DD0002F1CD000221146144610469E
:102340004B1B1DB2ED135B196B40139D1BB292002A
:10235000B25E53431818A418491C8AB2BA42EFD38C
:10236000FEF70FFA06462046FEF70BFA002C03D1C3
:1023700000E000260398C0051C901CA81BA901259D
:102380002A4604F0FFFA1B9C20463146FDF76FFFFA
:10239000014610988160002F119422D00024274616
:1023A000264613951291B8B2FEF7EBF91299FDF794
:1023B00056FF0546A0001499085EFEF7D7F90146BE
:1023C0001398C00785432846FDF751FF0146304664
:1023D000FDF7F4FE06467F1CBCB215988442E2D39A
:1023E00000E0002611983146FDF741FF1099C860C2
:1023F0001DB0F0BD98A00102000020410000404047
:10240000F0B58FB00692F74A09AF70CA70C770CAAC
:1024100070C70328079320D88800F3A10858F6490D
:10242000FDF7CCFE0446F549FDF7C8FE0D90F449D2
:102430002046FDF7C3FE0C90F2492046FDF7BEFE94
:102440000B90F1492046FDF7B9FE0A90EF4920466E
:10245000FDF7B4FE0990EE4969E0042822D0062871
:1024600020D88800EBA10858EE49FDF7A7FE0446E6
:10247000ED49FDF7A3FE0D90EC492046FDF79EFEC9
:102480000C90EB492046FDF799FE0B90E949204658
:10249000FDF794FE0A90E8492046FDF78FFE09906B
:1024A000FD4944E00838022821D88800FBA10858DB
:1024B000D149FDF783FE0446FC49FDF77FFE0D90F0
:1024C000FB492046FDF77AFE0C90FF20810520464F
:1024D000FDF774FE0B90F7492046FDF76FFE0A905A
:1024E000CA492046FDF76AFE0990FE491FE08800B0
:1024F000F1A10858F449FDF761FE0446F349FDF7E0
:102500005DFE0D90F2492046FDF758FE0C90F14912
:102510002046FDF753FE0B90EF492046FDF74EFE97
:102520000A90EE492046FDF749FE0990EC490094D7
:102530002046FDF743FEEC4909680E90EB4804681D
:10254000EB4801684808EB4F05463D400022002D4E
:1025500008922DD0CA01120E07D0280CE90D12D115
:102560004000E649085AE6490AE0C903090E0CD0C2
:10257000280AE90B10D14000E049085A8F21890050
:102580004018E4300DE0DC490AE081B27F2905D82B
:102590004800DA49085A04E0D94901E08F2189004E
:1025A000401800B2FEF7E2F8D649FDF760FE024699
:1025B0000292039507252606D34B1A68002A08982D
:1025C00040D0791C8A420BD21102090E13D0110C93
:1025D0001F46D00D1FD14800C849085AC84907E016
:1025E0001F46110E002A13D44800C449085AC24994
:1025F0004018E4301FE011041F46090E0ED0110AE6
:10260000D00B12D14800BD49085A8F218900EFE74D
:10261000BE4808180FE0B84808180CE091B27F29AE
:1026200006D84800B549085A05E0B548081802E040
:102630008F218900501800B2FEF798F8B149FDF7D4
:1026400016FE3B460590159F2C40F50E5B69B04980
:102650001940089810D0DA02D20E34D0C80B3E21AF
:102660000140A648405AA6494018E43000B2FEF79F
:102670007DF8A449FDF7FBFD0490149E6800A5A118
:10268000085EFEF773F80146A00009AA1058FDF78E
:1026900095FD0146B8B20128089F019102D1022C94
:1026A0000AD9A74F052C24D1189808900C2D20D8B2
:1026B0000B2D16D3A44918E00027022C089718D038
:1026C0008120C70515E01A04120E00D1CAE0080ADD
:1026D000C90B00D0CDE040008849085A8F218900FD
:1026E000C2E7092D00D2C7E096490898FDF766FDBC
:1026F000089001200021B542034600D30B46052C6B
:1027000000D308461799169A1A9C199D1843069BE0
:10271000012B12D1079B402B22D1002840D03846F4
:10272000FDF74CFD01460198FDF748FD0146009874
:10273000FDF795FD059A04998AE0079B402B1FD170
:10274000002838D03846FDF739FD01460198FDF7DD
:1027500035FD01460098FDF782FD059A049977E062
:10276000002833D03846FDF729FD01460198FDF7D2
:1027700025FD01460098FDF772FD059A049967E072
:1027800000285BD03846FDF719FD01460198FDF79A
:1027900015FD01460098FDF762FD059A049957E082
:1027A00002981146FDF75BFD0399002900D16748A7
:1027B000059A04994CE002981146FDF750FD0399E3
:1027C000002900D16148059A049941E00298114618
:1027D000FDF745FD0399002900D15C48059A04994D
:1027E00036E0C046CCBF0000000068C1000088C1D0
:1027F00066665EC1000084C1000084410000B441EF
:1028000000004841000020400000F0C0000084C1EA
:102810000000F841333323C1000050C19A9929C107
:102820009A9949C19A9949413333CB4166667641B9
:10283000CDCCAC40333393C09A9949C1029811462C
:10284000FDF70DFD0399002900D14048059A049930
:1028500028601046FDF703FD0899FDF700FD206094
:102860000FB0F0BD99B27F2911D848002349085A0A
:10287000FCE623494018F9E6C12001060898FDF757
:102880009DFC0890062D00D933E7002030E78F210A
:1028900089005818EAE6C0463333F341000058C1B6
:1028A0009A9961C19A9969C1000084C10000AC4144
:1028B00000003841000008C1CDCC80C1CDCC88C11A
:1028C00033338FC1333397C133339741CDCC8C41F0
:1028D0003333F3409A9919C0666646C1333397C1C2
:1028E000CDCCB4410000D4410C0000405030004039
:1028F00068400040FFFFFF007C08000044C3000068
:102900005C050000919AF63C642000409C0B00009E
:10291000FFFF1F00FAFFFCFFFEFF000002000400A3
:10292000060008000A000C000E001000120014003F
:10293000160018001A001C001E00200022002400AF
:10294000000080BF0000A0C0000040C00000DCC24A
:10295000F0B5FFB0ECB017460E460D900021E9919E
:10296000E891DC9199919891979196911491139196
:1029700012919AA8F49DF39CF29A002E00D1E6E100
:102980000B938030F09B1180099529602546DBACC4
:10299000218095AC21800C952980DA917F24E40573
:1029A000B994B894B794B694B594B494B394B294DB
:1029B000B194B094AF94AE94AD94AC94AB94AA940B
:1029C000A994A894A794A694A594A494A394A2943B
:1029D000A194A0949F949E949D949C949B949A946B
:1029E000046644668466C466046744678467C46793
:1029F000046444648464C464046544658465C46593
:102A0000046244628462C462046344638463C46392
:102A1000046044608460C460046144618461C46192
:102A2000B0090B250B2800D3AE011095012B0B9D8F
:102A300000D070E12B89012B00D06CE1298C00299A
:102A40000E9200D18BE16B8C002B00D1FAE1AA8CA5
:102A50003021695C002900D188E10892109F5F4312
:102A60001196304639460F93FDF734FB0590FDF77C
:102A70007DFE01462046FDF737FC8321C905FDF7A1
:102A8000F6FB064696A8021D119887420A9200D8C6
:102A900079E155A811909AA9069196AF15463A4644
:102AA000059C234603F0E2FE15A80F9006992A46DE
:102AB000234603F0DBFE02230D93384631463A46A7
:102AC00003F020FF012308930093E8AA10923846F0
:102AD000394603F0EDFCE898DD901198069D2946F3
:102AE0003A46234603F0C2FE0F9829460A9A234627
:102AF00003F0BCFE384631463A460D9B03F002FF18
:102B0000089B009338463946109A03F0D1FCE898A8
:102B1000DE9011982C4629463A46059D2B4603F037
:102B2000A5FE0F9821460A9A2C462B4603F09EFEDE
:102B3000384631463A460D9B03F0E4FE089B00936D
:102B400038463946109A03F0B3FCE898DF901198A4
:102B5000069D29463A46234603F088FE0F982946EB
:102B60000A9A2346254603F081FE384631463A4606
:102B70000D9B03F0C7FE089B009338463946109A18
:102B800003F096FCE898E0901198069C21463A469E
:102B90002B4603F06BFE0F9821460A9A2C462B46D3
:102BA00003F064FE384631463A460D9B03F0AAFE18
:102BB000089B009338463946109A03F079FCE89850
:102BC000E1901198069D29463A46234603F04EFEB1
:102BD0000F9829460A9A2346254603F047FE3846B1
:102BE00031463A460D9B03F08DFE089B0093384614
:102BF0003946109A03F05CFCE898E2901198069C24
:102C000021463A462B4603F031FE0F9821460A9A98
:102C10002B4603F02BFE384631463A460D9B03F017
:102C200071FE089B009338463946109A03F040FC29
:102C3000E898E390119821463A462B4603F016FE99
:102C40000F9821460A9A2B462C4603F00FFE384671
:102C500031463A460D9B03F055FE089B00933846DB
:102C60003946109A03F024FCE898E4901198069DE8
:102C700029463A46234603F0F9FD0F9829460A9A59
:102C80002546234603F0F2FD384631463A460D9B71
:102C900003F038FE089B009338463946109A03F03B
:102CA00007FCE898E5901198069C21463A462B4689
:102CB00003F0DCFD0F9821460A9A2B4603F0D6FD5F
:102CC000384631463A460D9B03F01CFE089B0093A4
:102CD00038463946109A03F0EBFBE898E6901198D5
:102CE00021463A462B4603F0C1FD0F9821460A9A29
:102CF0002B4603F0BBFD384631463A460D9B03F0A8
:102D000001FE089B009338463946109A03F0D0FB29
:102D1000E898E7907AE010880C9A10809991989141
:102D2000DA9E08460F46099DF59CFDF798FA286043
:102D3000DC9827606060A6600C34DDA80EC80EC465
:102D40002EC82EC42EC82EC47FB06CB0F0BDFF209C
:102D500010800021296020807FB06CB0F0BD00227F
:102D600001233021695C002900D076E6DDAA1ACF64
:102D70001AC23ACF3AC23ACF3AC20B213046FDF7D7
:102D8000A9F9054642E000200690059D0796089F98
:102D90001190069801460D9C0F9A4A43D219109B38
:102DA0005A43119BD218D200A35889002E4655AD24
:102DB0006B503546121DA25815AB5A50401C01B23B
:102DC0008E42E9DC55A89AAE96AC314622462B4697
:102DD00003F04CFD15A831460A9A2B4603F046FD38
:102DE000022320460799224603F08CFD012300931D
:102DF000E8AA2046214603F05BFB119B9800DDA961
:102E0000E89A0A505B1C0B2B1846C1D1F19EDDA835
:102E10009AA9DCAA0B2303F029FD09210E980F9132
:102E200001800B98C168DC9C2046FDF720FA014622
:102E3000A8B2E69F0F281BD808280DD30846FDF737
:102E4000BDF914E0FF2010800021099A11600C994F
:102E500008807FB06CB0F0BD042803D381220846FF
:102E6000D10502E0412208461106FDF700FA0146AD
:102E70002B20C04386420D9704DB0846FDF79EF9E0
:102E8000014603E04020C043864244DD0E9A0C9C7C
:102E90000B98408A002811D00B98038A95A80390BC
:102EA000DBA80290DAA801900094DDA80D4601F09D
:102EB00085FC29462488DA9E099D68E011910F98C7
:102EC000208000273D46109705E00E9804887F1C5F
:102ED000B8B2A04211D8B8B28000DDA90C58204683
:102EE0001199FDF7DFFB0028EFD1002DEDD10C98F3
:102EF000078001250F971094E7E7DBA805800F9A5C
:102F000090B2201A012811D10C9804800D9FDA97F5
:102F10003E46099D3AE04920C043864200DA8BE0F4
:102F2000FF2208469105FDF7A2F9A9E710200B99A9
:102F30000E5E012E00DA90E0551CABB21846A1B22D
:102F4000AAB28A4217D805E00E990C88A1B2AAB29B
:102F50008A4210D88000DDA90C58204610991F46DF
:102F6000FDF792FB3B46002805D10C9805800B9895
:102F7000068A0F95109430B2C1186D1CA8B2814218
:102F8000E2DC109EDA960F9C099D0D9F1199304648
:102F9000FDF7AAF9FDF734FC052800D3052095A913
:102FA0000880A0B20E990988814218D9401C611E80
:102FB0000CB2A04218DA12A898A9FEF76DFE0E987E
:102FC0000188481C491E0CB2A04221DA12A899A916
:102FD000FEF762FE99999898099D0D9FA4E600213D
:102FE0009891999108469FE60022134608E09CB20A
:102FF000A40012AF3D515B1C491C0CB2A042DADBAD
:103000008DB20A2D1546F2D8A400DDAD2D59EEE79C
:103010000022134608E09CB2A40012AF3D515B1C95
:10302000491C0CB2A042D1DB8DB20A2D1546F2D854
:10303000A400DDAD2D59EEE75320C043864200DBEE
:103040001BE70E460B9881692046FDF71DFB002803
:103050000C9C08D10B98808B07E01446099D0D9FAE
:103060001199109E93E70B98C08BFDF78AFB0146E0
:103070003046FDF7FCF8119021E70000F0B58BB069
:103080001C4609930E46034600200A9040480088DB
:10309000224F05970AA9049103940292109C01946F
:1030A000012500950B21414389B230331C4A30463B
:1030B000FFF74EFC3868079078680890B86806906B
:1030C00033480088334F009501940297324E3036D2
:1030D0003249334A3346FEF76BFB0698F86207988D
:1030E000386308987863099800882E4905912E491D
:1030F00004912E4903910297019000962C4B28468B
:1031000029462A46FEF74CFC432001060A98FDF7A3
:10311000AEF8FDF775FB0BB0F0BDC04660A0010234
:10312000D4B30102F0B589B00F9F0E9C002815D0D2
:103130001098079016480088164E012500950191B9
:1031400002960893144B30331449154AFEF730FBAE
:10315000089BF76207983063746303E00D48476388
:10316000C462002518880F4905910F4904910F4941
:1031700003910849029101900748303000900121E5
:103180000B4B28460A46FEF70BFC09B0F0BDC046C3
:10319000F6A6010298A80102C4990102189801023A
:1031A000A4A70102909D0102F4A60102A0A60102BB
:1031B000A8A6010280B5124801681F220A400260D9
:1031C00003200840022812D10E480268D30D02D015
:1031D000FF231B06D2180C4B1A600C4A12680C4BCA
:1031E0001A6080680B4A1080000C0B4A10801A4845
:1031F0008268002A02D082680020904780BDC046C5
:103200007420004064400040B8A7010278300040BC
:10321000BCA70102289A01028EA8010280B50D48C0
:10322000016889070FD5052101600B48C178002985
:1032300008D00021C170C168002903D0C26841686C
:103240000020904780BD054805A10B4A0BA306F05E
:10325000EBFCC0462C040040D893010295CE000040
:103260005048595F54494D45525F49525148616E2B
:10327000646C6572000000008D0A0000556E657870
:1032800070656374656420696E74657272757074BC
:103290000000000070B50446401E012814D8032029
:1032A000084011D13F2040030818050B2819802839
:1032B0000AD8164E317801204840294602F0A8FA73
:1032C000641E6D1C002CF5D170BDC04680B5002079
:1032D000014601F0C1FF002800D080BD0B4801214C
:1032E000017080BD70B516460C460546FF22FCF7FE
:1032F00053FF0548311805480278012050402A46FE
:10330000234602F02DF970BD00E0070498A20102E7
:10331000012000037047012040037047F0B583B0DF
:1033200030480068C16B0901890F01D003B0F0BDBE
:10333000C16BC06B2C4D05404800400F082602961B
:1033400086400227384600F081FF01907043C10B90
:103350004A1B26485043FCF7D3FE044606F048FBC0
:10336000032123A238461F4F0091234607F08AFC11
:10337000F88A002817D0019840012946FCF7AAFED8
:1033800046431822324001200F2A014600D800216E
:1033900073095B181B4CA3420DD8194DED1A6D052E
:1033A0000F2A0CD80CE038680021C160112000F011
:1033B0003DFF03B0F0BD5D1C6D050F2A00D95642DC
:1033C0002A0C029D2E4009018919A34202D80098B7
:1033D000000400E04004081880183968086303B04E
:1033E000F0BDC04668940102FFFF1F0040420F007D
:1033F00052434F33324B2070706D2025640D0A000C
:10340000FF070000FE7F0000B0B582B015490868D4
:103410008269D2070CD00122C2610D69002D07D04C
:1034200000686C46214605F0FBFE00212046A847B7
:1034300002B0B0BDB0B582B00A490868026C92070C
:103440000ED5026C012313430364CD68002D07D011
:1034500000686C46214605F0E3FE00212046A8479F
:1034600002B0B0BD6894010207480168032291438D
:103470000160016801220A43026008F0C5FA00F009
:10348000ADF806F0D7FAC0462800004080B50D49D7
:103490000868002810D5224802680423032A01D0B6
:1034A0001A4300E01A460A601E490A68002A02D040
:1034B00041680020904780BD03A00CA19E2211A36B
:1034C00006F0B2FB2C100140696E636C7564652FC9
:1034D000647269766572732F6D6B5F736C6565706E
:1034E0005F74696D65722E6300000000534C4545A2
:1034F000505F54494D45525F49525148616E646C6A
:1035000065720000556E657870656374656420733C
:103510006C65657020696E746572727570740000F8
:103520000890010294A80102B0B582B00446007868
:10353000002811D0094D01A908702868416A0029A6
:10354000FCD101A901220020034608F0E7F8611C24
:10355000607800280C46EED102B0B0BD8094010224
:10356000F0B50C784D782D022C198D78C9780902A8
:10357000491909040C1981000D4D6C509478D578C7
:10358000167852780B4F7B50120292192B021B199E
:103590001B049A18084B5A50059A13785278074C16
:1035A000079D65501102C9184000054A1152F0BD2F
:1035B000FC9801027CB401026099010218B4010276
:1035C000C898010280B504480168491C016000697F
:1035D000002800D0804780BD00B4010201480249A4
:1035E00001607047389001020026B80380B582B0B0
:1035F0000E4908680022C2600192CA68002A02D0FF
:10360000016801A8904702B080BDC04680B582B075
:10361000064908690022C26001220192CA69002A93
:1036200002D0016801A8904702B080BDD892010283
:10363000B0B502F04BFE154CE060A178002900D037
:10364000B0BD21790029FBD10121217100281AD0B8
:103650006425281AA168814215D0A0682018007D31
:1036600021698847A068401CA060A068642801DB2D
:103670000020A060E168A068022D04D36422511AE2
:103680006D1E8842E9D100202071B0BDE095010295
:1036900080B5002007F016FD80BD80B5012007F041
:1036A00011FD80BDB0B582B0602833D0622843D010
:1036B000642854D101A82F490180EFF3108072B61D
:1036C00000242046214601F0C7FD2B4D002805D1DE
:1036D000012002030020294601F018FD103501AA3F
:1036E00002232046294602F013FA62B623A0FFF710
:1036F0001BFF64201B490C5205F03AFF1A4800F0EA
:1037000075FEBFF34F8F194819490160BFF34F8F02
:1037100000BFFDE76020134900220A5205F028FF90
:10372000114800F063FEBFF34F8F1048104901604D
:10373000BFF34F8F00BFFDE762200A4900220A5203
:103740000A8005F015FF084800F050FEBFF34F8FC8
:10375000064807490160BFF34F8F00BFFDE702B085
:10376000B0BDC0469AA20102A08601000CED00E0A7
:103770000400FA05AAAA000000D00204BDF8C8EBB4
:10378000C9FDBCB6C4A3CABD0D0A0000F0B581B026
:10379000644FB96808291BD88A0001A39A58974634
:1037A000C5370000D1370000D1370000E1370000F5
:1037B0000B3800001738000021380000EF370000F8
:1037C0002B380000552848D10120B86001B0F0BD69
:1037D000AA2838D1012936D10220B86001B0F0BD45
:1037E0000421B9600021B970787001B0F0BD397959
:1037F0007A181073481C3871C0B27978491F814219
:103800002FD10820B86001B0F0BD0521B96046494C
:10381000087001B0F0BD0621B960B87001B0F0BD0C
:103820000721B960387001B0F0BD797806291AD344
:103830004B1F002422463D192D7B521992B2641C65
:103840009C42F8DB10E0032807D1022905D10120B2
:10385000F8700320B86001B0F0BD0020B870B86007
:10386000787001B0F0BD0022101841182E48007881
:103870000918BD7849193C780919FA78002A00D04E
:10388000C91CC9B2FF2945D1012819D0022841D14C
:103890002748401939460C312246FCF76BFC387B2F
:1038A000012802D12846FFF7FDFE05F061FEBFF3B7
:1038B0004F8F204820490160BFF34F8F00BFFDE7C5
:1038C0001A4EB47103203071B070AA207070552068
:1038D000307068087071651DF57040001449091852
:1038E000F01D2246FCF746FC301DE11CEAB2D21C5A
:1038F000037892B2D218401C491EF9D1A019D143C5
:10390000C171090A0172093400203146224603467A
:1039100007F004FF0020B870B8603871787001B00B
:10392000F0BDC046709501023C900102B2970102C1
:103930009AA201020CED00E00400FA0580B582B005
:10394000002001900448C268002A02D001A800218A
:10395000904702B080BDC04610950102F0B583B01B
:1039600000242046FFF7B2FCFFF7D5FC274EB060DD
:10397000FFF7CEFC7060264F0BE001A8C18880885D
:10398000084319D101A8408824180834B06884423B
:1039900035D201AD082128462246FFF7A3FC28882E
:1039A0000028EAD0B8422AD001AD0421284600F010
:1039B00007FDA9888842E5D03460B06884420CD203
:1039C00001AD022128462246FFF78CFC2888B84228
:1039D00003D0A41CB0688442F2D370682118491E39
:1039E0004042084030600DD0002425460120294681
:1039F000FFF750FC03CE4D19083E8542F6D33460E4
:103A000003B0F0BD0024346003B0F0BDA8960102FD
:103A1000FFFF0000F0B585B01F4604920646C817A8
:103A20000C1844400A2C039114D301250A21204686
:103A3000FCF750FB6D1C632C0446F7D804998D42AB
:103A400000D329460A9C002F09D00398002808D4E7
:103A5000002207E0012504998D42F2D2F2E700220C
:103A600005E00122042323409B081343FA1A022392
:103A7000234004980028029412D1002B10D0F4683F
:103A8000002C62D40398002825D40298400734D52E
:103A90007068B5686F1C87422FD830682B2423E0EC
:103AA000E407ECD1002A0AD1E9E73768202038552D
:103AB000B560F068441CF460521E002CDFD49142C3
:103AC000DDD27768B468651CBD42EED9F468521E39
:103AD000002CF4D5D3E7404203907068B5686F1CA2
:103AE00087420AD830682D244455B760F068441CDA
:103AF000F4600025ED43A84227DB002B1CD00120F9
:103B0000029B1840049B184316D1002A03D113E0EE
:103B1000521E002C0ED491420CD27068B3685D1C0A
:103B20008542F5D830683024C454B560F068441C30
:103B3000F460EDE7002C08D40092029801900A226C
:103B400030460399049B00F003F805B0F0BD000077
:103B5000F0B587B01F4615460290012406919142A8
:103B6000009407D3012406982946FCF7B3FA641C95
:103B7000A842F9D20D980C9ABC42039700D3039443
:103B800000990140002A009109D00029029C25D10A
:103B90002021800705D40846002F11D004E0029CA4
:103BA0001CE03020002F0BD0084609E02368585451
:103BB000A260E168491CE1603246721E00290DD402
:103BC000039991420AD216466368A1684A1C9A4238
:103BD000ECD9E1683246721E0029F1D5E068002870
:103BE00059D40590012401E07F1E6C43022FFBD2C3
:103BF000069821461646FCF76DFA3246A842F4D2E2
:103C0000029880680490069F0195069738462146E1
:103C1000FCF760FA049D691C029F7A68914206D9FC
:103C2000069F059A019D0592002A0ED516E01B4AB3
:103C3000125C3B685A55B960FA68521CFA600491EC
:103C4000069F019D0592002A08D460433F1A204632
:103C50002946FCF73FFAAC420446D6D20098002829
:103C6000029C059B049D16D0002E14D0701C01E010
:103C7000002B10D4401E039981420CD2691C62684B
:103C80009142F5D8226820235355A160E268531C65
:103C9000E3600D46ECE707B0F0BDC0467CC2000013
:103CA00070B5002801D0012070BD0C4616252846AD
:103CB00000F0C4FA284605F0A5FA002C05D01B48F0
:103CC000183014222146FCF755FA28211748415C88
:103CD000002915D04168002916D403220B469343CE
:103CE000144A9C588D07ED0EFF26AE40B4439C50FD
:103CF0001F220A40012191400F4A11600F4A1160B2
:103D000001210161002070BD8A07D20EFF2393407C
:103D10000F220A40083A03218A43054954589C431C
:103D2000545001210161002070BDC0464090010245
:103D30001CED00E000E400E080E200E000E100E0D3
:103D40005A21014A50527047C4990102F0B581B01E
:103D500013490A78002A13D0052A01D104220A70D7
:103D60009300CD18561C00231C462F686F60F9176E
:103D7000DB194C412D1F761E012EF6DC084902E0AE
:103D80000022134614464860521C0A70C1171818C6
:103D90006141D2B20023FCF7C7F901B0F0BDC046C3
:103DA000409501025C21A0480022425282847A217F
:103DB00041840284C2830283C2820282114941602B
:103DC0008260C2603D21490441834182090C8183A4
:103DD000818270475C2194480022425282847A2179
:103DE00041840284C2830283C28202820549416007
:103DF0008260C2603D21490441834182090C818374
:103E0000818270474C3C3C3C70B5C2484C210160FB
:103E100001252C02601C00F091F9322000F0E6FA36
:103E200000F04AF9284600F051F9284600F060F801
:103E300000F03CF90C4800F081F90026304631468C
:103E400000F08CFA2846314600F088FA204600F04F
:103E500075F9022000F072F94834204605F05CFE46
:103E600005F0BAFE70BDC0460102000010B5052085
:103E70000424214602F0CEFA0620214602F0CAFAB6
:103E80000A20214602F0C6FA0920214602F0C2FAB1
:103E900000240121204602F0BDFA022120462246DC
:103EA00002F0E0FA10BD80B5072002F087FA80BD6D
:103EB00080B50020084907F037FA08480268002A50
:103EC00003D01120022102F009FA072002F086FA3D
:103ED00005F082FE80BDC046189001028C9A010256
:103EE0000248016801229143016070475800004078
:103EF00002490A6802408242FBD1704704600040D8
:103F0000B0B5494D28688107484C0ED528797F21E6
:103F1000084022688A431018206023680B40022062
:103F20000321434A06F0AEFE286880040ED55E20C9
:103F3000285C7F21084062688A43101860606368CB
:103F40000B40022003213B4A06F09CFE172000F0A4
:103F500075F93948016802220A4301218A43026047
:103F600036483749016037480021C17181791F25E2
:103F700029408171817A427C837C1B029A18C37C20
:103F80001B04D218037D1B06D2182F4B9A4218D15E
:103F9000427B837B1B029A18C37B1B04D218037CD1
:103FA0001B06D218294B9A420BD1C27A037B491EB9
:103FB000122906D819028918254A914201D12021D7
:103FC00001720178CA0602D11022114301701C3C13
:103FD00020682021884320601E481F4901604168F5
:103FE0000029FCD503F090FA0446022003211BA20D
:103FF000234606F047FE0A20C441032C05D80220C0
:1040000003211DA206F03EFEFEE71848C1680F22FC
:104010009143C1600168164A0A40026019200001FC
:10402000144948600D60B0BD2C9A01024800004060
:1040300070CA00005ACA0000040200400C0600408A
:10404000AF6B100A6B0001404D383650312E3236BE
:104050000734000000600040FE1C00804368697067
:104060002049443A20253038780D0A00C8600040C5
:10407000FEFFC3FF0C0400404F6C6420636869704E
:10408000206D6F64656C206973206E6F742073758A
:1040900070706F727465642062792074686973202F
:1040A00053444B2121210D0A0000000080B5172048
:1040B00000F0BCF8002080BD10B51724204600F0A9
:1040C000BDF8204605F09EF8002010BD0121C9076B
:1040D00001430148016070470060004010B582B0A4
:1040E00003460C480168022B01DD012204E0022294
:1040F000D24393420CDCFF227F248A18A143224042
:104100008918016000920448032104A206F0BAFD58
:1041100002B010BD48000040020800005854414C55
:10412000206C6F6164206361702074756E6520255A
:1041300064203A2025640D0A0000000010B5C1B2C9
:10414000000AC2B202290CD0012913D0002930D1B3
:10415000911E7F4802291BD20121032A2AD049043B
:1041600029E07B484168002A1FD00246203A1143CB
:10417000416010BD76480168D31E022B10D3012A7E
:1041800029D0002A41D1012292079143016010BD3C
:10419000002A16D10121490702688A43026010BD36
:1041A0000123042A1FD05A041EE0012292079143E2
:1041B000416010BD0904194A7F32C36A134059187F
:1041C000C16217498A699207FCD501214907026833
:1041D0000A43026010BD0522120791430246203AAD
:1041E0000A43026010BD1A04836A0C4C1C40A218DA
:1041F00082620B4A131F00241C600A4B0A4C1C608D
:104200000D235B0214681C431460054A93695B0626
:10421000FCD5052212071143016010BD80FFFCFF91
:104220001402004004010040FF0F00000121814002
:10423000474802688A4302607047C04601218140B6
:10424000434802680A4302607047C04610B505281B
:1042500011D8C0467844007940008744020E1924E2
:1042600034393B490A680868C0003CD53A482039CF
:104270000A425DD03BE0002010BD35490A6808685D
:10428000C00035D534480B46203B1A4237D134E0C4
:104290002F490A680868C00036D52F480B46203BD6
:1042A0001A424CD135E02A494C680120C0030A6803
:1042B0000B46203B1C421AD00C68E4003BD5264C30
:1042C0001A423CD03AE0224800680120C00310BDE9
:1042D0001F490A680868C0001ED51F480B46203BCE
:1042E0001A4220D11DE01B4820390A4220D010BDBF
:1042F00018480B46203B1A4201D10120C0034968EF
:104300008900890FC84010BD12480B46203B1A4255
:1043100015D10120C00312E00E480B46203B1A4283
:1043200001D10120C00349680903890FC84010BDAD
:104330000120C00310BD074C1A4200D020464A6835
:104340009200920FD04049680901890FC84010BD02
:1043500020000040006CDC020026B80304282CD8A2
:10436000164AC0467844007940008744020A121A6F
:10437000210003200007136883438807800818186A
:104380001AE0032080061368834388070009181881
:1043900012E003208004136883438807000B181879
:1043A0000AE0FF200002136883430802181803E0A4
:1043B0001068FF23984340181060704724000040A5
:1043C000B0B5002200290CD0074B047895B22D0A15
:1043D00065406C001C5B12026240491E401C0029B3
:1043E000F3D190B2B0BDC0467CC0000000280AD016
:1043F00030B407252C02CD256419604340091238DA
:10440000001FFDD830BC7047F0B583B01F4616467C
:104410000D460146E8680291FBF729FF04460F2E7E
:1044200011D8082E04D320462146FBF7C7FE09E029
:10443000042E02D38120C10501E04120010620465F
:10444000FBF715FF04460999089E2B20C0438742BD
:1044500005DB20460F462146FBF7B0FE0DE03F206E
:10446000C04387420BDA4920C04387420CDBFF2060
:104470000F4681052046FBF7FAFE39460446688A56
:104480000880346003B0F0BD01915320C0438742DF
:1044900006DB20462146FBF791FE0446688A10E0C1
:1044A000A8690299FCF70CF9002801D1A88B00E05B
:1044B000E88BFCF766F901462046FBF7D8FE044678
:1044C000002001990880346003B0F0BDF0B581B0E0
:1044D00005460120072D66D80C46002963D04A4FB7
:1044E00038680169C90736D105263046FFF7A6FEB0
:1044F000304604F087FE03CF0369012213430361B2
:10450000002918D403200B4683438E481E58880781
:10451000C00EFF278740BE43402787403743894866
:104520001F501F2008408240874802608748026071
:10453000354800680FE08A07D20EFF2696400F2309
:104540000B40083B03218B437D495F58B74340260E
:1045500096403E435E50690140180121090242180D
:10456000E369DB069B0CA569ED00EDB2EB18536027
:1045700062685207520B23685B075B099A18A368AD
:104580005B079B0CD218E3685B075B0DD2182369AD
:104590005B01DBB2D21863699B07DB0ED218802364
:1045A00013434350002001B0F0BDC046F0B581B0C8
:1045B000002A23D005460835134C2668F668EE40DD
:1045C000F50702D0022001B0F0BD069D8600A619B5
:1045D000B560400124682018009301231D0246198C
:1045E00077680724A7437760F16032610099B16072
:1045F000415919434151002001B0F0BD03A00AA167
:1046000074220DA305F010FB90920102696E636C99
:104610007564652F647269766572732F6D6B5F6464
:104620006D612E6300000000646D615F7472616EE5
:104630007366657200000000496E76616C696420E3
:104640007472616E73666572206473742061646451
:104650007200000000015849085840687047C04681
:10466000F0B581B005460120012D4CD80C4600293B
:1046700049D0002D03D0012D04D10F2000E00E20E1
:10468000FFF7DCFDA668012E04D0002E4FD1E08993
:1046900000284CD12901294843580020D860F5074B
:1046A000AD0F27686668B607360F76192569EA07E1
:1046B000920EB618022F04D0012F03D10122164307
:1046C00000E040361D4F9E60E2681A6079188D60E8
:1046D0006269CA604968002917D403220B469343D4
:1046E000184A9C588D07ED0EFF26AE40B443802635
:1046F000AE4026439E501F220A4001219140124A9B
:104700001160124A116001B0F0BD8A07D20EFF2479
:1047100094400F230B40083B03218B4308495D580D
:10472000A543802494402C435C5001B0F0BD08A008
:104730000FA1492212A305F077FAC046D8920102D0
:104740001CED00E000E400E080E200E000E100E0B9
:10475000696E636C7564652F647269766572732F18
:104760006D6B5F6475616C5F74696D65722E63005B
:104770006475616C5F74696D65725F6F70656E0002
:10478000636F6E66696720697320696E76616C6914
:10479000640000000001084A10580160816880220E
:1047A0000A4382607047C046000103490858816887
:1047B0008022914381607047D8920102F0B58DB09C
:1047C000019315460E460A90129800240890048022
:1047D000149F3C80139809900460159804900480FD
:1047E000FF2081053046FBF742FD029030460396DC
:1047F0003146FBF7E3FC2B463D46069027460795DE
:104800000B9311E0118018888000285809990860DE
:104810000120079D28800520049908807F1CBCB2D8
:104820001888844200D9A0E028880028F6D1A0008A
:104830000A9D2E5830460699FBF734FF002817D002
:1048400030460399FBF72EFF00280B9B079DE5D10F
:10485000089A1780099D2E601888011B012934D100
:104860001080198889000A9A51582960059035E00E
:10487000089A1780099806600B9B1988081B012865
:10488000C0D00C96019825187E1CB0B28542BFD3CB
:1048900089B2B2B28A420ED880000A990C582046DA
:1048A0000C99FBF7F1FE0B9B002804D109980460DA
:1048B000089806800C94761CB0B28542A8D319885B
:1048C00089B2B2B28A42E7D9F5E70C96019962182B
:1048D0007D1CA9B216468A4205972CD2059884B24F
:1048E000A5000A9E7259002C104609D0A819001F75
:1048F000016810460C92FBF761FC0C9A062C07D855
:104900000446A81941681046FBF758FC0C90204655
:10491000079D0299FBF7D4FE00280B9B07D10C984A
:104920000299FBF7BFFE0B9B002800D076E7012021
:104930002880032070E780B2AAB282420FD8880094
:104940000A990C5820460C99FBF79EFE0B9B0028F9
:1049500005D1099804600898058005950C946D1C94
:10496000A9B28E42BAD31888E5E70DB0F0BD0000B9
:10497000F0B585B001273904494D68680491884332
:104980006860286847490143296039074648016043
:104990004648039101600024204600F0BDFD4448D4
:1049A000017849B2002902D480220A430270686962
:1049B0000290A86901903F4803683F4E7360C36846
:1049C00033603346143B1B68F3603346103B1B686F
:1049D000336133460C3B1B6873613346083B1B68ED
:1049E000B361331F1B68F3616C62FB052C460C3C02
:1049F00020689843206078046A6882436A6030BF08
:104A00006A6802436A602068184320602B4C029851
:104A10000440002901D42648017007206862002064
:104A200000F08CFD264803990160BFF34F8FBFF360
:104A30006F8F1D48016070681E4908603068C8604B
:104A4000002C08D08C622046019A10400863204652
:104A50009043C862CC611B4801688906FCD50A24D2
:104A60002046FFF7C3FCF8022968814329602046ED
:104A7000FFF7BCFC38032968814329602046FFF713
:104A8000B5FC2868B8432860284614380068C0027E
:104A9000FAD5686804990843686005B0F0BDC0465F
:104AA0002C000040011C000080E200E000E100E07A
:104AB00067000140042000501C010040FFFF03007C
:104AC00080E100E02C0200400A490A680A480240DE
:104AD0000A60FD214900094A1268515C002908D08A
:104AE00007490A6C02400A64012000060A688243F2
:104AF0000A60704700040040FFFFFF7FE893010257
:104B00002000004000207047F0B583B00D460446F9
:104B10007C26464350488719F869396AFBF7DAFA68
:104B2000A84200D892E0019502940121EFF3108091
:104B3000084002D1EFF3108272B63C4610343B6954
:104B40000025062B0CD80A469A40D3065B0F06D1E7
:104B500061231A4275D00D46002803D003E00225D8
:104B6000002800D162B6002D02D0284603B0F0BD67
:104B700000943C462034384880591021C1613E469B
:104B8000143605F023F805463868C069C00605D517
:104B900005F01CF8401B31888842F5D90621029D9A
:104BA000284600F02FFF206801994143B869091891
:104BB00038688160172179563C461734002909D599
:104BC000C16920220A43C2610121F9668905026890
:104BD0000A4302600521284600F014FF207840B205
:104BE00000250028C1D42B4800687D24E100FBF794
:104BF00071FA61014143029800F0D6FE04F0E6FF2D
:104C000004463868C069C00705D004F0DFFF001B08
:104C100031888842F5D904F0D9FF04463868C16963
:104C2000890706D504F0D2FF001B31888842F5D9E8
:104C300038680121009A116053498161284603B008
:104C4000F0BD0321216000288CD08CE7034804A12B
:104C5000084A09A304F0E8FF00930102A0CA00007B
:104C6000666C6173685F626C6F636B5F65726173C2
:104C7000650000005D020000626C6F636B20696478
:104C800078206973206F7665722072616E67650D9A
:104C90000A00000014B40102F0B583B002907C2138
:104CA0004143934A5418E56EEAB2511E02291FD2BD
:104CB00029040126090E18D001960092022100F065
:104CC000A1FE2746143704F081FF06462068C1691B
:104CD000890606D404F07AFF801B39888842F5D90A
:104CE0002068007DC007019E08D0304603B0F0BDAB
:104CF000032A36D100922804000E36D020466C30AC
:104D00002D0C0021019101602746143704F05EFF4D
:104D100006462068C069C00705D004F057FF801B15
:104D200039888842F5D904F051FF06462068C169E8
:104D3000890706D504F04AFF801B39888842F5D9D7
:104D4000206811498161E9B20120002911D00329AD
:104D50000099019E00D006202061226F002A0ED10A
:104D6000C3E70026304603B0F0BD0126304603B04D
:104D7000F0BD0099019E2061226F002AB5D002A8E3
:104D80009047304603B0F0BD000093EB70B50028AB
:104D900001D0012070BD7825CD4E705D00280ED069
:104DA00000240921204600F02DFE0F20FFF71EFBF6
:104DB0001520FFF73BFA74553461204670BD04207E
:104DC00070BDC046F0B581B00C460078484EF16821
:104DD00081422CD1032C54D1706EB16E884261D9BE
:104DE00000240621204600F00DFE3068F16D816040
:104DF0002046214600F006FE354660352CCDF06891
:104E00003168B48C414F00975B1BA34200D81C460D
:104E1000A3081431FFF7CAFBB06E0019B066306EFC
:104E200000193066F06D0019F06501B0F0BDB16891
:104E3000814255D1032C45D1F08CF16D0918F165F3
:104E4000316E09183166B16E0818B066716E814214
:104E500038D900240621204600F0D4FD3068F16DD9
:104E600081600121204600F0CDFD316EB068F38CE9
:104E70003268264C009414329B08FFF797FB01B070
:104E8000F0BD30681021C16104F0A0FE0546306815
:104E9000C069C00616D504F099FE401BB18A88424D
:104EA000F5D90FE030681021C16104F08FFE05468E
:104EB0003068C069C00605D504F088FE401BB18A81
:104EC0008842F5D90120C107326813688B4313600B
:104ED000F16E22040A4300021043F06601B0F0BDF7
:104EE0004D200201034804A1844B04F09DFEC046FE
:104EF00000930102A0CA0000666C6173685F646D74
:104F0000615F63616C6C6261636B0000C54D0000A2
:104F1000F0B581B000786E4DAA68824200D0D0E032
:104F200001263002032942D16A6DAA66AB6DAC6AD4
:104F3000A418EB652C66AB6C5B1CAB646B6E934288
:104F400035D95E30FFF752FA686CA96C02293AD362
:104F5000814238D1E88C696D081868650020062107
:104F600000F050FD2868E96D81602F6D04F02EFE81
:104F700004462868C069C00705D004F027FE001B5E
:104F8000A98A8842F5D904F021FE04462A68D0692E
:104F9000800706D504F01AFE001BA98A8842F5D9BD
:104FA0002A687420285C012841D0F10440E0F2070F
:104FB0002B681C6894431C60EA6E0904114301438A
:104FC000E96601B0F0BD0229FBD38142F9D2E88C39
:104FD000696D09186965A96D0818A8650020062182
:104FE00000F010FD2868E96D8160EF8C04F0EEFDA3
:104FF00004462868C069C00705D004F0E7FD001B1F
:10500000A98A8842F5D904F0E1FD04462A68D069EE
:10501000800706D504F0DAFD001BA98A8842F5D97D
:105020002A687420285C012822D0F10421E031058F
:10503000334B3B405918012802D01920400601E0AB
:105040000720C00608182F4940185060002F0DD0C7
:1050500004F0BCFD04462A68D069800706D404F039
:10506000B5FD001BA98A8842F5D92A682B6D1FE07F
:105070003105234B3B40C918012802D019204006B6
:1050800001E00720C00608181E4940185060002F94
:105090000DD004F09BFD04462A68D069800706D431
:1050A00004F094FD001BA98A8842F5D92A68EB8C8C
:1050B000296EA868144C00941432FFF777FA01B0F7
:1050C000F0BD044804A10C4A0C4B04F0ADFDC046F1
:1050D00000930102A0CA0000666C6173685F646D92
:1050E000615F77726974655F6E62797465735F631F
:1050F000616C6C6261636B007204000087CA00001F
:10510000FF3F000000808000114F0000F0B587B025
:1051100004460126880E14D01546002A11D00F46E9
:105120008120C004401B88420BD37C206043F0499F
:1051300008180590818C38460691FAF7CBFF0029B4
:1051400002D0304607B0F0BD28460699FAF7C2FFF4
:105150000029F6D1059880693E1A30460699FAF77B
:10516000B9FF0746039670190190069E3146FAF77B
:10517000B1FF0546C01B04900598006A02903146B5
:10518000FAF7A8FF049981420FD20026BD42D8D970
:105190002046394600F03CFB2046FFF77DFD002805
:1051A000FAD17F1CAF42F3D3CBE700900398029D66
:1051B0002946FAF78FFF0646284670430399081AD6
:1051C000019800D0761C2946009D7543FAF782FFAE
:1051D0000590029941430198401A03900699FAF705
:1051E00079FF0490AF420BD22046394600F010FB05
:1051F0002046FFF751FD0028FAD17F1CAF42F3D3C0
:1052000005988642069D009F0CD220463146FFF746
:105210007BFC2046FFF740FD0028FAD1761C05985C
:105220008642F2D30398A84203D20026304607B044
:10523000F0BD059847430025E919204600F0E8FA3B
:105240002046FFF729FD0028FAD16D1C002604989E
:105250008542F1D375E7C046F0B585B0002803D08C
:105260000124204605B0F0BD7822A14FB85C00288B
:1052700003D00024204605B0F0BD0492002905D0DB
:10528000384614300CC90CC01CC91CC00020F8667C
:1052900015242046FEF7D2FF204603F0B3FF3868FE
:1052A0001021C16104F092FC04463868C169C90646
:1052B00007D504F08BFC001BB98A8842F5D9386801
:1052C00000E0B98ABA7D1207120B5218F97DCB079C
:1052D000DB08D2188B07DB0F5B05D218CB06DB0F80
:1052E000DB05D2184B07DB0FDB06D2188B06DB0F72
:1052F0005B07D2180907C90F890711430160002411
:105300000A21204600F07EFB3220FFF76FF80821CB
:10531000204600F077FB04F059FC05463868C16967
:10532000890606D404F052FC401BB98A8842F5D99C
:105330003868017D0A46C23A5342534174257B5571
:105340000904027D12025118007D0B180220032669
:1053500068A2314605F096FC785D0128039619D1C4
:10536000F87D029000260621304600F04BFB072115
:10537000304600F047FB012102988143785D012807
:1053800047D138688901017506757521795C012955
:1053900038D048E00020032100F034FB04F016FC74
:1053A00006463868C169890606D404F00FFC801BE4
:1053B000B98A8842F5D93868007D46080122F87D0F
:1053C000014631431640C90701D0304036D002951E
:1053D000002506212846019200F014FB07210095C4
:1053E000284600F00FFB019846400298385C0128DF
:1053F00013D13868B1010175009901757521795C87
:10540000012910D114307621795C4A424A41510079
:1054100008E038680675490003E0386800990175AE
:10542000710014300170374800687D21C900FAF717
:1054300051FE28214143002000F0B6FA7720385C65
:10544000012803D102200021FEF788FF04F0BEFBF3
:1054500006463868C069C00705D004F0B7FB801B5A
:10546000B98A8842F5D904F0B1FB06463868C169AB
:10547000890706D504F0AAFB801BB98A8842F5D9B2
:105480003868E249816117203856002829D57868A4
:10549000002816D40146039A91431C4A8B5885076D
:1054A000ED0EFF26AE40B3438026AE401E438E5025
:1054B0001F210140012088401549086015490860F6
:1054C0000FE08107C90EFF228A400F230340083BEB
:1054D000039883430C481D58954380228A402A43F1
:1054E0001A500120049978543861204605B0F0BD67
:1054F000009301026A656465635F69642025780D25
:105500000A00000014B401021CED00E000E400E019
:1055100080E200E000E100E080B57C214143A64844
:1055200042187823D25C002A05D0405802494160D5
:105530000F20FEF75BFF80BD008020B980B57C2185
:1055400041439D4842187823D25C002A05D0405838
:10555000024941601E20FEF749FF80BD008020AB5C
:10556000F0B593B07C270A9047439348C619980733
:1055700004D0F07D4024044000D017E10125880EBE
:105580002ED0002B2CD08120C004C01A884227D3F3
:1055900009920122EFF31084144002D1EFF310803E
:1055A00072B6304610300590306900250628089103
:1055B000069310D8079414468440E106490F04D19D
:1055C00061210C4203D0154604E0022502E00221CD
:1055D000059B1960079C002C00D162B6002D02D0FB
:1055E000284613B0F0BD344617347348C059102113
:1055F0000491C1613746143704F0E8FA0546306873
:10560000C069C00605D504F0E1FA401B398888421C
:10561000F5D92078400665D40297B78C069C2046C1
:105620003946FAF757FD079039464143601A03900F
:1056300035462435A74200D894E0039800281CD0B2
:1056400006210A9C204600F0DDF928880799484386
:10565000089940183168886000272046039C394625
:1056600000F0D0F9079B099A28885843C01931687F
:10567000097D11547F1CA742F6D330680499C1619B
:1056800004F0A4FA0446029D3068C069C00605D53E
:1056900004F09CFA001B29888842F5D904F096FA98
:1056A00004463068C069C00705D004F08FFA001BBB
:1056B00029888842F5D904F089FA04463068C1691E
:1056C000890706D504F082FA001B29888842F5D99B
:1056D00030680121059A1160B24981610025284690
:1056E00013B0F0BD03200025089FF76509993166C6
:1056F00006997166B566F0660120C00731680A68D0
:1057000002430A6006210A9C204600F07BF93068BB
:1057100087602046294600F075F93A4F0BAA0A9295
:105720001BCF1BC21BCF1BC2B48CF0680A99FEF7BB
:10573000CDFEF0683168344A0092069A944200D354
:105740001446A3081431099AFEF730FFB06E001911
:10575000B066306E00193066F06D0019F0652846AD
:1057600013B0F0BD002404E0641C0798844200D309
:1057700063E706210A9800F045F9288860430899F4
:1057800040183168886000270A98394600F03AF9D5
:1057900028880028099AE7D0604310183168097DED
:1057A000C1557F1C28888742F6D3DDE7034804A152
:1057B000064A07A304F038FA00930102A0CA0000C9
:1057C000666C6173685F726561640000C603000007
:1057D00054686520444D412072656164206C656E9B
:1057E0006774682073686F756C64206265207468E4
:1057F00065206D756C7469706C65206F6620340D62
:105800000A000000FCC20000C54D0000000093EB40
:10581000F0B583B00D4604467C26464351488719AF
:10582000F869B98CFAF756FCA84200D894E00195C3
:1058300002940121EFF31080084002D1EFF31082AF
:1058400072B63C4610343B690025062B0CD80A463C
:105850009A40D3065B0F06D161231A4277D00D46DA
:10586000002803D003E00225002800D162B6002DF5
:1058700002D0284603B0F0BD00943C462434394899
:1058800080591021C1613E46143604F09FF9054647
:105890003868C069C00605D504F098F9401B318806
:1058A0008842F5D90621029D284600F0ABF82088F1
:1058B00001994143B8690918386881601721795600
:1058C0003C461734002909D5C16920220A43C26128
:1058D0000121F966890502680A430260042128460D
:1058E00000F090F8207840B22C4600250028C0D463
:1058F0002B4800687D21C900FAF7ECFB20492D31C7
:105900004143204600F050F804F060F9044638683E
:10591000C069C00705D004F059F9001B31888842DE
:10592000F5D904F053F904463868C169890706D5EA
:1059300004F04CF9001B31888842F5D93868012100
:10594000009A116017498161284603B0F0BD032118
:10595000216000288AD08AE7034804A1084A09A3E5
:1059600004F062F900930102A0CA0000666C617342
:10597000685F736563746F725F6572617365000061
:105980002B020000736563746F722069647820696C
:1059900073206F7665722072616E67650D0A000074
:1059A00014B40102000093EBF0B583B001917C22A6
:1059B0000290424353498C182546143504F006F9E9
:1059C00006460221029800F01DF804F0FFF8074691
:1059D0002068C169890606D404F0F8F8C01B29883C
:1059E0008842F5D92068007DC00708D06420FEF702
:1059F000FDFC04F0EBF8801B01998842E1D903B06B
:105A0000F0BDC046F0B585B0049104467C206043EB
:105A10003C490F183D46143504F0D8F8064638685E
:105A2000C069C00705D004F0D1F8801B29888842DE
:105A3000F5D904F0CBF806463868C069800705D56B
:105A400004F0C4F8801B29888842F5D91421049BEE
:105A50005943DC2060432C4A1018039002914018EF
:105A6000018A8268C47C7426BE5D012E0DD101912D
:105A7000012B02990CD0012B0DD07526BE5D012E95
:105A80000ED0019E072B0ED10EE00E4602990BE0C0
:105A90000222012BF1D138247526BE5D012EF0D1F2
:105AA0000326072B00D0019E184B33402406920793
:105AB000D20A1219D218039B5958C907490C521817
:105AC0004168CB071B0CD218837C5B075B0BD21899
:105AD000C0684007000A10183A685060002E0ED0C7
:105AE00001290CD104F072F804463868C0698007B7
:105AF00005D404F06BF8001B29888842F5D905B05D
:105B0000F0BDC0460093010244C40000FF3F000006
:105B1000F0B59DB00D460126890E2FD0002B2DD05B
:105B200011928121C9041093C91AA94226D30121D7
:105B3000EFF310840C4002D1EFF3108272B67C2296
:105B40000F904243E74814928718384610303B695B
:105B50000026062B0DD80A469A40D3065B0F07D1C4
:105B600061231A4200D16FE30E46002C03D003E0FC
:105B70000226002C00D162B6002E02D030461DB0A5
:105B8000F0BD0290BD650021139179651098401E0B
:105B900012904019B964B9690D916E1A1199B962E0
:105BA000FD6238637E63F98C0E913046FAF792FA03
:105BB0000446B863129830180E9E3146FAF78AFAF6
:105BC000109B011B4A1CF86339647A64139A0029FC
:105BD000194608D0704359190D9BC91A0A1A744303
:105BE000581B80190119384648300E903846443009
:105BF0000D90384640300B90384626300590384698
:105C000058301390384654301290F9643A6514981D
:105C1000B44908581021C1613846143014903846F0
:105C2000503004903D464C3503F0D0FF04463868B0
:105C3000C069C00606D503F0C9FF001B1499098886
:105C40008842F4D9F87D40060C9500D574E2012312
:105C50000E9803600D98016800290F9800D1CDE2DD
:105C60003A4674320A92DA0407921A050992192206
:105C7000520606920722D206089216E09A48006859
:105C80007D21C900FAF726FA109941430F9C20465E
:105C9000FFF78AFE20460C9D0E9A11684B1C13607C
:105CA0000D9909688B4200D9A8E20B9A1268012A63
:105CB00055D0002A00D0A8E02E6812990C681399DC
:105CC0000D6806211091FFF79DFE386885601198D8
:105CD000051903F07BFF04463868C069C00706D089
:105CE00003F074FF001B149909888842F4D903F06B
:105CF0006DFF04463868C169890707D503F066FF60
:105D0000001B149909888842F4D938680A990A78DE
:105D1000012A089900D00699012A099A00D0079A09
:105D20003346724C234013430B4371490B4343608A
:105D3000002EA3D003F04AFF04463868C0698007EC
:105D400006D403F043FF001B149909888842F4D954
:105D50003868297801756D1C761EFAD18EE7012B03
:105D600000D0C7E02E6812990C6813990D680621BF
:105D70001091FFF747FE386885601198051903F008
:105D800025FF04463868C069C00706D003F01EFF2F
:105D9000001B149909888842F4D903F017FF0446C0
:105DA0003868C169890707D503F010FF001B1499F3
:105DB00009888842F4D938680A990A78012A08992A
:105DC00000D00699012A099A00D0079A3346474C19
:105DD000234013430B4346490B434360002E69D0D5
:105DE00003F0F4FE04463868C069800706D403F067
:105DF000EDFE001B149909888842F4D93868297887
:105E000001756D1C761EFAD154E0012B00D0C9E05B
:105E10002E6812990C6813990D6806211091FFF7EE
:105E2000F1FD386885601198051903F0CFFE04462E
:105E30003868C069C00706D003F0C8FE001B14997B
:105E400009888842F4D903F0C1FE04463868C16964
:105E5000890707D503F0BAFE001B14990988884208
:105E6000F4D938680A990A78012A089900D0069965
:105E7000012A099A00D0079A33461C4C2340134349
:105E80000B431B490B434360002E13D003F09EFECF
:105E900004463868C069800706D403F097FE001BEB
:105EA000149909888842F4D93868297801756D1CDD
:105EB000761EFAD10C4800687D21C900FAF70AF96C
:105EC000109941430F9C2046FFF76EFD20460C9D24
:105ED0002A68139B196889181960129B1968891818
:105EE0001960D9E60093010214B40102FF3F0000DB
:105EF000008080008B4200D0CEE604990E68129993
:105F00000C6813990D6806211091FFF77BFD386826
:105F100085601198051903F059FE04463868C06978
:105F2000C00706D003F052FE001B1499098888426E
:105F3000F4D903F04BFE04463868C169890707D5D8
:105F400003F044FE001B149909888842F4D938688C
:105F50000A990A78012A089900D00699012A099A13
:105F600000D0079A3346D44C234013430B43D34904
:105F70000B434360002E00D180E603F027FE044669
:105F80003868C069800706D403F020FE001B14990E
:105F900009888842F4D93868297801756D1C761E05
:105FA000FAD16BE6129A1268119CA618139A15681A
:105FB0008B425FD104990C6806210391FFF722FD03
:105FC0003868856003F002FE05463868C069C0077E
:105FD00006D003F0FBFD401B149909888842F4D9D0
:105FE00003F0F4FD10900C9D3868C169890708D54D
:105FF00003F0ECFD1099401A149909888842F3D9EE
:1060000038680A990A78012A089900D006991091EF
:10601000012A099A00D0079A2346A7490B40134347
:1060200010990B43A5490B434360002C14D003F097
:10603000CDFD10903868C069800707D403F0C6FD15
:106040001099401A149909888842F3D93868317830
:106050000175761C641EFAD19A4800687D21C9003A
:10606000FAF738F8039941430F9C2046FFF79CFC50
:10607000204611E605990C8806210391FFF7C2FC22
:106080003868856003F0A2FD05463868C069C0071E
:1060900006D003F09BFD401B149909888842F4D96F
:1060A00003F094FD10900C9D3868C169890708D5EC
:1060B00003F08CFD1099401A149909888842F3D98D
:1060C00038680A990A78012A089900D0069910912F
:1060D000012A099A00D0079A234677490B401343B7
:1060E00010990B4375490B434360002C14D003F007
:1060F0006DFD10903868C069800707D403F066FD15
:106100001099401A149909888842F3D9386831786F
:106110000175761C641EFAD16A4800687D21C900A9
:10612000F9F7D8FF039941430F9C2046FFF73CFC49
:10613000204605990A88CCE65E4815A90A4678C823
:1061400078C278C878C20125E8073A681368034323
:106150001360B868FEF7BAF902200026139C216884
:10616000BA6AF9653A6610997966BE66F8660C985F
:106170000068129A1168091811600E9B19684A1C70
:106180001A60226810182060002900D0F6E41095EB
:106190003846603013903C465C34384608301290E4
:1061A00006210F98FFF72EFC3868216881600C9853
:1061B0000068119003F00AFD04463868C069C00702
:1061C00006D003F003FD001B149909888842F4D916
:1061D00003F0FCFC0446109D3A68D069800707D59F
:1061E00003F0F4FC001B149909888842F4D93A683A
:1061F0007420385C01282DD0E9042CE003F0E6FC83
:1062000004463868C069C00706D003F0DFFC001BF5
:10621000149909888842F4D903F0D8FC04463868F8
:10622000C169890707D503F0D1FC001B14990988BF
:106230008842F4D938680121029A116022498161AB
:10624000002630461DB0F0BD04210160002C00D1B5
:1062500091E491E42905119C174B2340591801281A
:106260000C9D02D01920400601E00720C006081846
:10627000124940185060002C0ED003F0A7FC0446D1
:106280003A68D069800707D403F0A0FC001B14997A
:1062900009888842F4D93A682B68139801681298E3
:1062A0000068074C00941432FEF780F930461DB0A8
:1062B000F0BDC046BCC20000FF3F0000008080006F
:1062C000114F000014B40102000093EB3120C00014
:1062D000014909680858704790920102F0B50329F6
:1062E00020D8C0467944097949008F4401080F1528
:1062F000012181403D4B1B685963D96212E00121A5
:1063000081403A4B1B681963D9620BE0012181403F
:10631000364B1B68596304E001218140334B1B68F5
:106320001963996283003149CB18DA608A68002AC0
:1063300029D14A68002A16D4032314469C43174BDC
:10634000E5589607F60EFF27B740BD438027B740B4
:106350002F43E7501F23134001229A40104B1A602D
:10636000104B1A600FE09307DB0EFF259D400F24B2
:106370001440083C03229443074AA658AE438025A4
:106380009D403543A550012282400868026288681A
:1063900010438860F0BDC0461CED00E000E400E062
:1063A00080E200E000E100E010B501242046FDF7A6
:1063B00045FF204602F026FF002010BD012181404C
:1063C0000A48006842688A43426070470749096882
:1063D0000968C140012008407047C0460121814042
:1063E0000248006842680A43426070478093010295
:1063F00010B5054804680548006860430449F9F78A
:106400007FFE201A10BDC0467400004090A8010213
:1064100040420F00124A072809D880000F2383400A
:1064200081401940106898430843106070470F2856
:106430000AD8800020380F238340814019405068DB
:106440009843084350607047800040380F238340D2
:106450008140194090689843084390607047C04657
:1064600034000040F0B54307DC0E0726A640C30801
:106470009D000E4BEF187D68B5433E1D002908D0E6
:1064800035600122824001290CD118681043186040
:10649000F0BD01218140186888431860A24015436F
:1064A0003560F0BD186890431860F0BD0C010040E5
:1064B00010B582B014460A46014604980093019034
:1064C0000820234600F092F802B010BDB0B584B0A9
:1064D00014460A4601460898022500950193029049
:1064E0000720234600F052F904B0B0BD70B5002873
:1064F0005BD031490A783149002A03D14A68012327
:1065000013434B60428803881B049A180B46183BC0
:106510001A60828883891B049B180C460C3C2360FC
:106520000B46083B84681C60446903232340057CB8
:10653000AD00EB188569AD072D0D5B19457C2D036A
:106540005B19C569AE07B60A9B19867CB6059B190F
:106550000E1F3360036A122B04D107240C60541EF3
:10656000A2410AE0032C05D1012D03D807220A60BD
:10657000012202E006220A600122114C002525704A
:106580000F2464012034C57C6D0225401B069B0B43
:10659000D218C3791B07DB0ED21880790007C00D13
:1065A000101840191439086070BD064806A18622EB
:1065B00009A303F039FBC046F8A6010218100050E9
:1065C000FAA6010252CD00006C73705F656E6769B8
:1065D0006E655F72756E0000506172616D65746505
:1065E00072206973206E756C6C000000F0B58BB082
:1065F000109E34043ED00D46D64C21400127019711
:106600007F06B9423CD111462140B9423FD11C40DE
:10661000BC4243D1119902AC0027E781E780668034
:1066200027802782A774E1749908A181A908A18015
:106630000A90099708970797900880B2049020461F
:10664000FFF754FFAA480078002801D00BB0F0BD36
:10665000AB480168C90708D10168C90705D10168BD
:10666000C90702D10168C907F3D07F4801990170B9
:106670000BB0F0BDB8480D49AF22C14B03F0D4FABE
:106680000095B5480949B022754B03F0CDFA009248
:10669000B1480649B122724B03F0C6FA0093AE48E6
:1066A0000249B2226E4B03F0BFFAC04628CD00006B
:1066B000F0B58DB00392139E340446D00A46A54C23
:1066C0002140012502956F06B94244D1039921402A
:1066D000B94247D11C40BC424CD11499129D04AC24
:1066E000E174294921820027E781E78066802780BD
:1066F0009908A1819108A1800B95012D01D16121FB
:10670000CF43A7740C9002200A9009900398800848
:1067100080B206902046FFF7E9FE75480078002811
:1067200001D00DB0F0BD76480168C90708D10168F5
:10673000C90705D10168C90702D10168C907F3D0AB
:106740004948029901700DB0F0BD83480D49FB2204
:106750008B4B03F069FA00927F480A49FC22404BB8
:1067600003F062FA039800907B480649FD223C4BF7
:1067700003F05AFA009378480249FE22384B03F09E
:1067800053FAC04635CD00008E8E0000F0B58BB0B8
:10679000119E340447D00D466E4C214001270197CD
:1067A0007F06B94245D111462140B94248D11C402B
:1067B000BC424CD11299109F02ACE174294921824C
:1067C0000021E181E180668021809908A181A908EA
:1067D000A1800997012F01D0712100E06121C943F7
:1067E000A1740A90032008900790900880B204904A
:1067F0002046FFF77BFE3E480078002801D00BB012
:10680000F0BD3F480168C90708D10168C90705D133
:106810000168C90702D10168C907F3D0124801997C
:1068200001700BB0F0BD4C480C49D522544B03F01D
:10683000FBF9009548480949D622094B03F0F4F9C1
:10684000009245480549D722054B03F0EDF9009326
:1068500041480249D822024B03F0E6F944CD00003A
:1068600072CD000086860000FAA6010210B582B043
:1068700014460A4601460020009301900420234656
:10688000FFF7B4FE02B010BD10B584B014460A463E
:106890000146002000900193029004202346FFF758
:1068A00007FF04B010BD000070B50D460646042475
:1068B0002046FDF7C3FC204602F0A4FC0B4805600F
:1068C0000B480670002E0ED00A48016880220A4349
:1068D0007F218A43026001200003074908600749BD
:1068E000086007480460002070BDC046FCA6010295
:1068F000F8A601020CE400E080E200E000E100E024
:106900001C100050B0B582B0144602461148204019
:1069100001256D06A8420DD1180413D01748016057
:10692000002000930190062011462346FFF75EFEEB
:1069300002B0B0BD0094FF228C320748074908A37B
:1069400003F072F9FF208C30421C034803490C4BC2
:1069500003F06AF90300FCFF52CD00001ACD0000DD
:1069600044737420616464726573732025782069B0
:106970007320696E76616C69640000000810005035
:1069800090CD000080B582B00B46014600200092F9
:10699000019003200A46FFF729FE02B080BD0000E7
:1069A000002801D0042100E00221C34A5172411E97
:1069B0008841800103490A6840239A4310180860FF
:1069C0007047C04650A00050F0B583B002912E49E8
:1069D000CD7A0E7B771987424FD9089901911825F6
:1069E00045434126F604BF00BE19745B34490C4090
:1069F00057033C199B07D90C6418324B1B681B7A50
:106A0000745375196C880326B60326409B079B0CAC
:106A10009B193F2404401819029CA3061B0DC018A3
:106A20006880012A184E13D8707B14224243307BB1
:106A30005023434324011B199A18F37AC0181C23CE
:106A40004343D01880081E4A104007430F432F804D
:106A50000198686001F0AEFEA860E8681A49084035
:106A60003030E860286908402721715C40182861AF
:106A700000F000FE686103B0F0BDFF2288320348D9
:106A800003A108A303F0D0F804A70102E1CD0000A0
:106A90006D61635F63735F636F6E7374727563744C
:106AA00000000000435320696E64657820697320FC
:106AB0006F7665722072616E67650D0A00000000D6
:106AC000FF070000E89301020000F0FFF0B581B07D
:106AD000009314460D46074606263046FDF7AEFBEA
:106AE000304602F08FFB26211D48475400210170DB
:106AF00041708171017181704171C170C171022257
:106B00004272C16201634163816304734273C5725F
:106B1000009A561C134A168001724120C0040121BC
:106B20004903F9F740FB5020604329010818611917
:106B30008A00801818224A438018B2B24A4380184B
:106B4000094940180949884204D200F0B7F80020EA
:106B500001B0F0BD064807A19A2209A303F064F82A
:106B600004A7010200A70102280008020120080270
:106B7000E1CD00006D61635F696E69740000000023
:106B8000454D206F766572666C6F770D0A000000C8
:106B9000BC48C179002901D001207047007A411E0C
:106BA00088417047F0B583B002912A494B7B8342FC
:106BB00048D9CB7A0C7BE31818245C439B00E3187C
:106BC0004124E4041A191424019005466543002663
:106BD000565100925519EE882E4F0B467A1C3240C2
:106BE0002D4E3688497A711A2C4E0E40B618EE801A
:106BF0003740997BEF80AA88294F17404A424A4183
:106C000091007918274A8918A980274F0F402D1D18
:106C1000029801280AD125490E400921C90271189C
:106C200069800121C9037918298000E02F8001982B
:106C3000444300980019074A918C4182118C0182CB
:106C400003B0F0BD3520C200034804A109A302F03F
:106C5000EBFFC04604A70102E1CD00006D61635F58
:106C60006C696E6B5F646573635F636F6E73747280
:106C7000756374004C696E6B206465736320696E84
:106C8000646578206973206F7665722072616E6723
:106C9000650D0A00FFFBFFFF00A70102FF030000D4
:106CA00003D0FFFFE80F0000EF1F0000FF8300008C
:106CB000D54A50639163704704A70102F0B581B0D3
:106CC0004348CC21016003214160CF490A7BD304B2
:106CD000404C1B19CC7AA218541E1C431823534352
:106CE00092009A184B7B14255D435219920122435E
:106CF000012463061343436100228262C26202637D
:106D000042638263C26342650267334B1A605A6012
:106D10009A60324B1A601A619A61DC61304C1C62D5
:106D2000304C251D1D6325460C3D5D632546283DE1
:106D30009D632D4EDE631C645C642C4D2F461C3716
:106D40009F642746143FDF64103C1C65284C5C653B
:106D5000284C9C650C369E67274CA5634035E5633F
:106D6000DA651A665A669A66DA661A67234DDD672F
:106D700002258561224DC561C325AD03CD620A633D
:106D8000D2435A601F4A1368FF25AB4326254D5D49
:106D9000AD072D0EEB1813601B4A102313601B4A1E
:106DA0001360272260238B5419498160C1600161FF
:106DB00021607D210901016641661649C1641649B9
:106DC00041641649016400F045FC01B0F0BDC046C5
:106DD00004A000500000F8FF94A0005034A100501F
:106DE000FF185A0030040040041000401C200040EE
:106DF0005430004060400040B8A10050140014001E
:106E0000FF3F3FFF04E400E080E200E000E100E03B
:106E1000DC05DC053F0270020133D007D007D00744
:106E200070B5182002F0EEF9192002F0EBF90624F3
:106E3000204602F0E7F92046FDF700FAD54C002580
:106E400025706570A5712571A5706571E570607B11
:106E500014214143207B50224243E37A1E019219C0
:106E60005118C0181C22424389184120C004F9F768
:106E70009AF9E5712572FFF721FF70BD2921C54AF6
:106E80005054704704A70102F0B58BB007920891E7
:106E90000146C04FB8780991FFF784FE78793A7BB4
:106EA00079790691824200D89FE0FB7A9A181823DC
:106EB000534392004124E10404915218D2187B7B81
:106EC00014214B43D21850246043155801230A93D0
:106ED000DB022E469E4316504E4B2B4005937D7B86
:106EE00003914D433E7B7443F97A0B011B195B19E7
:106EF00071181C24029461435918A74B1B88069CE7
:106F00005C430919C904490D059BC9181150101893
:106F10000799416038787979089A00920322099B91
:106F2000FFF752FDF87A397B09183878814263D926
:106F300083000993049AD45C0894F7212140D1542A
:106F4000D1184D788E7836027619CB781B04F31859
:106F500007900A9886051E43330CCB70FB7A387B6A
:106F6000BC784D709E4D3540039E6643C018029B11
:106F70004343981940029B4B03405C19200A8870D8
:106F8000200CC870F023089D2B401B1D3D7B0895ED
:106F9000FE7A099D5355C8700620079A5043801900
:106FA000089A801848701F22D20222400243100A19
:106FB00088707879401C7871387B7979814201D367
:106FC000002179713978491C3970F97A08183978B3
:106FD000884201D80020387028200A993954387A1C
:106FE000401C3872387A0BB0F0BDA7204200D1485F
:106FF0000649074B02F018FEA72042007A32CD481E
:107000007249734B02F010FE04A7010201CE00008A
:10701000AACD000000F0FFFF0320000605490A6822
:1070200082430A600A6802430A6003480121016042
:107030007047C0461C0000401CA0005080B50120D5
:10704000FDF7B2FB80BD0000F0B587B006930646A1
:10705000504C607A504B1B88181A0C9DA84200DCDB
:1070600089E00F460592012E06D156480021C162E3
:107070000169554A89180160A0783146FFF792FDF1
:10708000E078E178069A2B4600F0AEF82078E178B7
:107090000097002206923346FFF796FCE07A217BA8
:1070A0000818217888426ED94120C20404918800D2
:1070B000815C0391F7250D40029285544549455C5A
:1070C0004549465C360276194449475C3F04F61947
:1070D0000127BF0537433E0C4654E67A217BA3784F
:1070E0003C4A85543E4D3D4014275F4389191C237B
:1070F0004B43D91949023B4B0B405D19290A364BCA
:10710000C1542E0C35494654F02703990F40059978
:10711000002900D13F1D217BE37A029A87542F4A30
:1071200086540622049E7243D2185118294A81546B
:107130001F22D20215400D43290A274A8154E078C4
:10714000401CE070E07AE178814201D30699E17059
:107150002178491C2170217B08182178884201D8A8
:1071600006982070E079401CE071A07A401CA07263
:10717000E07907B0F0BD3920C2001632074808A1F7
:1071800009A302F051FD3920C20004480F49104BF9
:1071900002F04AFD04A7010200A70102E1CD0000B0
:1071A0006D61635F747800004D4143205458206C3A
:1071B000656E206973206F7665722072616E6765F7
:1071C0000D0A00000804004090D0030017CE000014
:1071D000C8CD0000010008020200080203000802F6
:1071E000FF07C0FF00F83F00F0B589B00893019297
:1071F00004914F4DEF7A874200D891E0297B5026C9
:1072000032464A434124E3040693D218CC19A10024
:1072100051181822059254430A19697B14230793C5
:107220005943531802900001195804460390504ADC
:107230000A40A97AC902511808988205D2088A180A
:107240001A514C4911402A7B00965643384CE57A36
:107250002C0106982418A719354E5419A5007D193C
:10726000059844432819747B079D6C430519049FB6
:10727000D2194148048854432A19089CD204520D5B
:1072800051181D460398195000F0FEF90146707A16
:10729000001902043E460CD080B2C000002900D183
:1072A000801E029FA5214900F8F714FF1F2101400D
:1072B00001E00021029F38012818427983791B02DE
:1072C0009A18C3791B04D2182C4B1340437109043C
:1072D0005918090CC171002C20D0154835460646B6
:1072E000007B009B4343F17A0A01069F3A43D21880
:1072F00041188B00D218059B4B43D118727B079B1A
:107300005343C91840191C4A1288424388180199EE
:10731000884203D001992246F8F72CFF09B0F0BD4E
:10732000FF225C32034804A109A302F07DFCC046A1
:1073300004A70102E1CD00006D61635F74785F64B2
:107340006573635F636F6E737472756374000000BE
:107350005458204445534320696E6465782069730E
:10736000206F7665722072616E67650D0A000000FD
:10737000FF0700E000F8FFFF00A70102EFFFE000B9
:107380000168044A11604168516081689160C06879
:10739000D060704780A0005082B0FCF735FD05201A
:1073A00000252946FFF736F806202946FFF732F870
:1073B0000A202946FFF72EF809202946FFF72AF868
:1073C0000124204603F086FD284603F083FDFCF7E8
:1073D0004DFD01F097FE01F08FFE404801684048E6
:1073E00000688903019408D4032109070840210794
:1073F000884202D0FCF7D6FC06E0FCF7AFFAFCF7B7
:10740000E9FC0020FDF7C2FCFCF77AFD00252846C8
:1074100004F082FDFEF7C8FF324E311D284603F00E
:1074200083FF31483149016000F082F86949887A68
:107430002F4A107088882F4A10807D20C000C9888C
:10744000F8F748FE2C4F38702C4964222C4B284604
:1074500004F03EF801F034FC2A4A019C2046214603
:1074600002F09AFAA00302F0C7FA09E000242046CD
:1074700001F0D6FB642220462049214B04F028F875
:107480007078002802D0757002F098F8FCF7D0F8F8
:107490000B20FEF79BFF3178002804D0002905D18E
:1074A0000198307002E0012900D135707878002809
:1074B000E6D003F013F8EFF31080C007D6D1EFF356
:1074C000108072B60024204601F0AAFB64222046F8
:1074D0000A490B4B03F0FCFF62B6D1E718000040ED
:1074E0003000014014900102F09501028D37000038
:1074F000B9960102E496010230970102F495010267
:1075000005B7000071990000014800687047C04647
:107510000C00004081B080B581B0039303AB0093B1
:1075200003F058F801B080BC02BC01B0084700006D
:10753000F0B581B0002630463146FDF78DFE0125BD
:10754000AC022349234F30463A462346FEF708F85B
:1075500039882148814238D064217E5262217E528E
:1075600060217E5244217E5250217E52FD87BD878C
:1075700078217987022139874321F986BE83FD81ED
:107580001649B9817E810A2139811549B98038802F
:10759000FE831420B8827D208000F880EFF31080F5
:1075A00072B630463146FDF757FE00280CD12A034B
:1075B00000263046064D2946FDF7A8FD054A30460F
:1075C00029462346FEF7A4FA62B601B0F0BDC046D4
:1075D00000E002049AA20102AA550000E1FF0000A7
:1075E000341200000020704710B50024002809D094
:1075F000002905D003464A0003481946F8F7BAFDAA
:10760000204610BDE04310BDF89201020146002063
:107610000A2901DAC0437047014A11807047C04609
:107620007C9301020020704780B50188064A1180D2
:107630008178064A1170C178054A11700079FCF70B
:107640007FFB002080BDC046D4930102D693010287
:10765000B4A70102044805490160152109044160ED
:10766000034981607047C0469C30004041000800DB
:10767000340007000748006840697047FD2040005B
:1076800004490968085C7047024800686221405C50
:107690007047C046E893010210B5064804680648E2
:1076A00000686421F8F72CFD0221C9434143081901
:1076B00010BDC046B8A70102BCA701020A491A22A0
:1076C0000A600A4948704878FF210902084A13688D
:1076D0008B43800380B2C0181060064820210160EF
:1076E000054801600020704770200040D8930102D7
:1076F00004E400E080E200E000E100E0F0B5A9B0C1
:1077000016460F460546C648002B024600D01A46CC
:107710003921CC003D21C9005118119182421892A3
:1077200006D001204202BE491898F8F723FD189AA6
:107730006120111913910E21119C0A91A170002F43
:107740000D9501D00A2100E00921592317938300E8
:10775000E170784278411399087030781090107079
:10776000F17AE17471785170B7789770F178D170CF
:107770003579157174795471B1799171F179D1714B
:10778000317A1172717A5172B17A91727E1EF0B2B1
:1077900000210328169106D870B28000A1A21058CB
:1077A0006A00805A1690179882001898C018149092
:1077B000F81E022804D3012E084604D89D4800E094
:1077C0009D48031918781290189DA81817902846FC
:1077D000303015902C4656346D2080002950974A41
:1077E000974B149E33627262B362F2623176F18219
:1077F000139B597009229A70281841608160C160FA
:107800000161109880008F490858F9F773F8012F2B
:1078100010900F9104D0022F05D17F217E2004E02B
:107820007C217B2001E05B215A20159DA9842070DA
:1078300003200C90A080012666701F200B90A88268
:107840001820A8740A46083A179BDA76169B129AF3
:10785000D2184A439100189A9163B702791E8B425D
:107860000E9109D97848608034206884774828824E
:1078700077481399088339E07F2B10DD802B18D0CF
:1078800031028B421BD071028B4227D16E4961803D
:1078900068846F4813990883CF20C00025E0202B0F
:1078A00017D0402B1AD1684860800420688469484A
:1078B0001BE06548608006206884674815E06248E0
:1078C000608010206884624813990883C520C00036
:1078D0000BE0624860800220688404E00420688431
:1078E000812040006080FF2002302882104600F096
:1078F00005FF1298102806D0402808D108201499B6
:10790000C876072000E004201799887002E01798D5
:107910000C9981701898169A8078C11E02290CD390
:10792000022811D001280CD12672BA4200D90026B3
:107930006672BA4213D8F44812E00D200002119981
:1079400008800120800201E00C9800022081BA42E8
:1079500001D8EE4800E0FA20179988600EE0FA207E
:1079600017998860139800780028119901D0E84889
:107970004880E848139A1083E7480880A88CF8F7F5
:107980001BFF0026E54B3246F8F79EFD02460B46EC
:10799000E3493046F8F700FEE24B3246F8F794FD33
:1079A000F8F75CFF0746E080DF493046109A0F9BEE
:1079B000F8F7F2FDDD4B3246F8F786FDF8F74EFF9B
:1079C00078434042800B608116990E98814208D915
:1079D0000C20149FB872D648179988831220189AE1
:1079E0000EE0480A189A149F01D00D2003E0080AFF
:1079F00000D1DBE20A98B872CE481799888312202A
:107A0000F872D078052844D878440079400087443B
:107A10000227402C3339C848B881C8482FE0C046F7
:107A2000909001028CC200008CC200009CC2000039
:107A30009CC20000E4BF0000EBBF000030750000F6
:107A4000102700003CC0000005020000FF060000F7
:107A5000040800000A0400003604000003020000CD
:107A6000B748F881B748388013E0B748F881B7487D
:107A70003882B74838600CE0B448B881B5481799E7
:107A8000C88306E0B4487882B448B8800B980006F2
:107A90009064AE483881A748F880B14802882A84AB
:107AA000B0480078E874B0480078119F7875387D48
:107AB000139000285ED0AD490A681023DA413A607D
:107AC0000A794B79CF8867801B029A186A840A7AF0
:107AD0004B7A8F7AC87A0D7B65701B029A183B042B
:107AE000D21800061018179FF860487B8A7BCB7B62
:107AF0003B77120210186081087C7877487C149AD2
:107B00009072887CD072C87C159B1874087D58745C
:107B1000487D11909874C87D0A7E120212181A844A
:107B2000887DD87418464B7EC375887ECD7E2D0225
:107B30002818B880087F4D7F2D022818F880887F8C
:107B4000B877C87FF8772020085C149D287321201F
:107B5000085C68732A20085C2A314D782D022818A9
:107B60008D782D044019C978090640181899886441
:107B7000119801E0EB7DA87C7D498B700A80800024
:107B80001F38C882C883139800281FD02222774844
:107B9000825C034622335B781B029A180A842422F3
:107BA000825C034624335B781B029A18CA8426221F
:107BB000825C034626335B781B029A188A8328224C
:107BC000825C283040780002801888846948032548
:107BD00069A2294603F056F8189F387814907B78EC
:107BE000B8780F90FA78B8791390F8791190387ABC
:107BF0001090787AB97A0890099100930F980190C3
:107C00000292169803901298049013980590119878
:107C1000069010980790FAA2F8482946149B03F0A2
:107C200031F83D46643580212846F8F7BCFAB8782B
:107C3000C11E02290ED3012800D18FE1022800D0F5
:107C4000ABE11691149078787F225043F7494018A1
:107C5000F74907E01691149078785B225043F14978
:107C60004018F14941182846F8F784FA0D9D1898F4
:107C7000C6870E34324602E0641C0F2A0ADA2178E5
:107C80000029F9D0491C8907C90F91400E43C687C6
:107C9000521CF1E71699022907D31499491E0129AC
:107CA00000D97DE14279D24901E04279CF49891872
:107CB0000C78002D00D177E1C1790E91032900D90C
:107CC0004AE14279062A00D979E14921890041181F
:107CD0001191E43010900E98401E129019A80019CE
:107CE0000F9000231392149403E01898290600D1F2
:107CF0005AE1052A5AD8C0467A441279520097446C
:107D0000455C728598ABC04688130000E204000011
:107D10000C080000060A0000040F000000001041DB
:107D200030C1BD41000070400000F0400000D04173
:107D3000120C0000140B000012120000140E0000C0
:107D40000E160000130D0000121600000E120000A7
:107D5000140B0E0A12080000101600000E0B000093
:107D6000D4930102D6930102B4A70102C0A7010275
:107D70004094010201080000436173652070617244
:107D8000616D65746572733A200D0A001693DFB257
:107D9000002F04D019A801223946F8F7FDF9002C6C
:107DA00000D191E019A8C019BB498AE0E8B20228C5
:107DB00067D00027022867D06BE00E98022872D1A6
:107DC000E8B2022800D103461693DFB2002F04D098
:107DD00019A801223946F8F7DFF9002C74D019A848
:107DE000C019ACA16DE0E8B2022800D104231693BB
:107DF000DFB2002F04D019A801223946F8F7CCF9D8
:107E0000002C61D019A8C0199FA15AE0E8B202283D
:107E100000D106231693DFB2002F04D019A8012247
:107E20003946F8F7B9F9002C4ED019A8C01992A11B
:107E300047E0E8B2022800D10C231693DFB2002FEE
:107E400004D019A801223946F8F7A6F9002C3BD036
:107E500019A8C019874934E0E8B2811E4A424A4154
:107E60009700022804D119A801223946F8F794F99D
:107E7000002C16D019A8C0197CA12246F8F77AF96F
:107E80000FE00627022804D119A801223946F8F785
:107E900083F9002C05D019A8C01980492246F8F7AB
:107EA00069F9169710E01693DFB2002F04D019A8D5
:107EB00001223946F8F770F9002C05D019A8C0192D
:107EC00073492246F8F756F93C193F2C05D80F980C
:107ED000C0194021091BF8F766F912980228189872
:107EE00001D2002002E0C078411E88411599087037
:107EF000611E2E46E8B202280CD1179A517019A9BA
:107F0000119AB8C9B8C2B8C9B8C2B8C9B8C2B8C954
:107F1000B8C20DE0179A117019A9109AB8C9B8C261
:107F2000B8C9B8C2B8C9B8C2B8C9B8C2C10709D1BE
:107F300080073546149C139A169B00D4D5E6022080
:107F40008543D2E6FE20354605401898149C139AC6
:107F5000169B290628D0CCE637A231E01691149062
:107F600078780B994143334808181F386F21C9436B
:107F70000D9D7A180378D427D3554378D827D35545
:107F80008378DC27D355002900D170E6C378E02739
:107F9000D3551031001D189FEBE70120404A10E037
:107FA0000024002D00D087E629B0F0BD80290ED333
:107FB0000F20B872104817998883102020E525A259
:107FC0000120014602F05EFE189829B0F0BD102095
:107FD000402904D3B8720849179B998310E5B872F9
:107FE00004481799888314200AE5C046EBBF0000B7
:107FF000E4BF0000150F0000140B00000108000092
:1080000025642025642025642025642025642025FE
:1080100064202564202564202564202564202564AF
:108020000D0A00009DD700001DF7FFFFB5CE000030
:1080300089FBFFFFA5D600007472785F6D6F6465E1
:1080400020706172616D65746572206572726F7205
:108050000D0A00004E73666420706172616D657474
:108060006572206572726F720D0A0000FFFFFFFFDC
:1080700001FF00001CC30000FFFFFFFFFF0101FF25
:10808000FF01FF01FFFF01FFFFFFFF01FFFF01FFF6
:1080900020C50000FFFF01FF3CC30000ACC2000090
:1080A00053CE0000002800D101481D4908607047E8
:1080B0009090010210B5002801D0044601E0184854
:1080C0000468204600F006FC204600F021F80B482A
:1080D00041780B4A1A23136041704078FF2109024E
:1080E000084A13688B438007000CC01810600648CC
:1080F000202101600548016010BDC046D8930102EF
:108100007020004004E400E080E200E000E100E0D4
:10811000F0B586B0002805D10148006802E0C046ED
:10812000E89301023121C900049141188A791F2383
:108130001A40CD79ED06AD0DAA180D7AED066D0C3D
:1081400052194D7AED062D0B52198D7AED06ED0977
:108150005219CD7AED06AD0852194D7CED07521932
:10816000BD4C22600A7B1A404E7BF606B60DB21853
:108170008E7BF606760C9219CE7BF606360B92199C
:108180000E79F606F60992194E79F606B608921996
:1081900062604A6AB14D2A40A2608A6A2A40E2605F
:1081A0002D22D20087183A7E1A4003937E7EF6066F
:1081B000B60DB218BE7EF606760C9219FE7EF60655
:1081C000360B92193E7FF606F60992197E7FF60667
:1081D000B60892190E7CF60792192261BA7F1A40EE
:1081E0000597FE7FF606B60DB218049BC35CDB064E
:1081F0005B0CD2184B78DB061B0BD2188B78DB0696
:10820000DB09D218CB78DB069B08D2186261CA69F9
:108210002A40A2610A6A2A40E2618A7C01252A403A
:10822000CB7CDB079B0F9A180B7DDB075B0FD2180B
:108230004B7D9B07DB0ED2188B7DDB079B0ED21884
:10824000CB7D1B079B0D9A180B7E1B079B0CD2182E
:108250004B7E5B06DB0A13438A7E520612091A43E1
:10826000CB7E5B075B0813432362CA6A62620A6BB8
:10827000A2624A6BE2628A6B22633922D200835C7B
:108280001E462E4066635E425E41B304AE04744FE8
:108290003C68B443E3183B6083185A782A409C78C2
:1082A0002407E40EA2188C8F6401A2186D4C1440B0
:1082B000C98FC905490A0919DA78D207120A89183B
:1082C0001A791207120989185A79D207D20889181F
:1082D000FB4EB1639968F163997904952940DA7985
:1082E000D207920F51181A7B5207D20E89185A7B67
:1082F000D206920D51189A7B5207D20C8918DA7B5C
:10830000D206920B89181A7CD206520A89185A7C16
:10831000520792090A43997CC906490851183164E9
:10832000D97C039A11401A7DD206920D51185A7DBC
:10833000D206520C89189A7DD206120B8918DA7D62
:10834000D206D20989187164197E0F2421405A7E01
:10835000120151189A7E12038918DA7E1207120A46
:1083600051181A7F1207120989185A7F12078918A3
:10837000B164997F01942140DA7F1207120E5118DF
:108380003D22D200835C5B075B0D5918841862782C
:108390001207520C8918A278D206120B8918E278BB
:1083A000D206D2098918F164217907220A4061793D
:1083B000C9008918A2795206920B5118E2799207E6
:1083C000120B8918227AD2078A18BF490A60627A8A
:1083D000A37A1B029A18E37A1B04D2184A60E28936
:1083E000BA4B13400394228AD2049209D2188A60AD
:1083F00003463033598CB64A114002939A8CD20509
:10840000D20A51185622825C12068918B14D296091
:10841000014656314A788C782402A2188C8864056B
:108420006409A218CC78240712196A60CA880C7AE9
:10843000A407A40BA2184C7A6407E40A1219AA60D4
:108440004989E960492189004118FF226632821872
:1084500000921035002207E000300040FFFFFF00CF
:1084600004040040FF3F000084186427E65D0327F2
:108470003E406523E35C9B071B0F9B196626A65DA8
:10848000B607B60EF3186726A65DB601F318DBB281
:108490006826A65DB607B60DF3186926A65DB60771
:1084A000360DF3186A26A65DB607B60CF3186B26D0
:1084B000A65DB607360CF3186C26A65DB607B60B9C
:1084C000F3186D26A65DB607360BF3186E26A65D6B
:1084D000B607B60AF3186F26A65DB607360AF31874
:1084E0007026A65DB607B609F3187126A65DB60715
:1084F0003609F3187226A65DB607B608F318732678
:10850000A45DA407E31808C51032802AACD1019AF3
:10851000D243704EB4180B783B404D78AD072D0F09
:10852000EB188D78AD07AD0EEB18CD78AD01EB18DB
:10853000DBB20D79AD07AD0DEB184D79AD072D0D03
:10854000EB188D79AD07AD0CEB18CD79AD072D0C7F
:10855000EB180D7AAD07AD0BEB184D7AAD072D0B6F
:10856000EB188D7AAD07AD0AEB18CD7AAD072D0A61
:10857000EB180D7BAD07AD09EB184D7BAD072D0951
:10858000EB188D7BAD07AD08EB18CD7BAD07EB1875
:10859000A3641031121DBDD1009B19785A7852077F
:1085A000520D51189A78D207120D8918B164059BA3
:1085B0001968F164D97D5A681202511831659968B9
:1085C000454A0A40998A490589187165D9683D4C20
:1085D0002140B16519692140F165029E3178049D01
:1085E000294082785207120F5118C2799207920ED1
:1085F0008918427A9207920D5118827A9207120DC9
:108600008918C27AD207920C89189A7DD207520C27
:10861000891872789207D20B8918B2781207D20A99
:108620008918F2781207D2098A182C490A60327C1C
:10863000737C1B071B0D9A18B37C9B069B0BD218EF
:10864000F37C1B079B0AD218337DDB065B09D2182B
:10865000737DDB071B09D2184A60B27D2A40C38FA5
:108660005B009A188A60826CCA60C26C22400A6100
:10867000F27D7F231340328C5204520AD2184A6191
:1086800002698A614269CA6182690A62C2694A6290
:10869000026A8A62426ACA62826A0A63C26A4A6378
:1086A000039A927CD201121D0A64027A3A40CA658A
:1086B000808F074A10400866002006B0F0BDC04613
:1086C00000300040FFFFFF009C300040FF1F000013
:1086D000FF03000000400040FFFF1F00002000409B
:1086E00004480068806B8008034909684900401805
:1086F00009307047E89301021004004010B52D21A5
:10870000C9004118027A032A04D10079002807D051
:10871000082006E08378DA1E022A05D2032412E03C
:10872000142088601C203DE0012B02D1C8228A6001
:1087300012E00479042C01D3462404E0032C01D177
:10874000322400E014248C605B1E022B04D3022A26
:1087500010D24279154B01E04279154B9B181B78DA
:10876000402B04D0102B06D11423442405E02A23E7
:108770003E2402E04279342348244B800C80022AB4
:1087800006D0062A08D0052A08D118224C2301E079
:10879000142250230B8000E01C224A80C078042859
:1087A00003D1142048806420088010BDEBBF000076
:1087B000E4BF0000424800687047C04610B53F4A19
:1087C000107091703E49002813D050680861042051
:1087D00048619078FF2212023A4B1C689443800350
:1087E00080B20019186001204007054A1060364A1F
:1087F000106000200860354901220A6010BDC046A3
:1088000080E200E03148002101602D4801680268E3
:108810008A420BD0016802688A4207D00168026868
:108820008A4203D0016802688A42EFD17047C0468D
:10883000F0B581B021480178214D002911D081780F
:10884000FF2212021F4B1C689443890389B2091945
:108850001960012149071C4A116040682861042001
:1088600068610127EFF310803840009002D1EFF3E8
:10887000108072B6154807602E682868B04208D18B
:108880002868B04205D12868B04202D12868B042B9
:10889000F3D0FDF7ADFD0446F7F773FF0C49F7F78A
:1088A000E6FCF7F7C6FF3018B843286000980028A8
:1088B00000D162B6204601B0F0BDC046D893010297
:1088C000180400401CE400E000E100E070000040FB
:1088D00080096E45F0B591B0002801D1C04800680C
:1088E0008778F91E022913D3012F21D0022F3CD102
:1088F0001021CA4344782146193991423DD8009746
:108900000125B94A28462946234602F0BBF953E11E
:108910000821CA43447821462139914218D800974A
:108920000125B14A28462946234602F0ABF943E126
:108930000821CA43447821460939914234D8009726
:108940000125A94A28462946234602F09BF933E12E
:10895000032F3CD0042F43D1C3780125042B00D032
:108960002DE106462A02042343E00125A6A228465B
:1089700029463B4602F086F91EE1C3780125052B06
:108980000AD806462A02284698401B21084230D1C0
:108990000021052B08462ED002200090914A28463F
:1089A000294602F06FF907E10646C3780021022B41
:1089B0001ED3032B1CD0042B08460A461BD00125CE
:1089C0000095884A2846294602F05CF9F4E0C3780D
:1089D0000125032B00D0FAE006462A02032308E013
:1089E000012583A2284629463B4602F04BF9E3E0E5
:1089F0000A46012148020F91592189007518FD216D
:108A0000490071180291314662313F05D219641E46
:108A10001F2727405C013C19144304433279520755
:108A2000D20C22432B789B065B0BD218B379DB0761
:108A30001B0B13436D4D2B60F279032310931A40E7
:108A4000737A9B079B0E9A18B37A5B07DB0D9A1813
:108A5000F37ADB079B0DD218337BDB075B0DD21853
:108A6000737B1B075B0CD218AA603269EA607269DB
:108A70002A61B2696A61F269AA61326AEA61726A5C
:108A80002A62B26A6A620F980870F06AA8623F2090
:108A9000C4432C353046E4300F903046E5300E901C
:108AA0003046E6300D903046E7300C903046E830E6
:108AB0000B903046E9300A903046EA300990304653
:108AC000EB3008903046EC3007903046ED300690A1
:108AD0003046EE3005903046EF3004903046F030AE
:108AE00003903746F1373046F230F3360F990A19C2
:108AF0004021525C109B1A400E9B1B195B5C9B072C
:108B00001B0F9A180D9B1B195B5C9B079B0E9A18F9
:108B10000C9B1B195B5C9B019A18D2B20B9B1B1917
:108B20005B5C9B079B0D9A180A9B1B195B5C9B0760
:108B30001B0D9A18099B1B195B5C9B079B0C9A18D1
:108B4000089B1B195B5C9B071B0C9A18079B1B1946
:108B50005B5C9B079B0B9A18069B1B195B5C9B0736
:108B60001B0B9A18059B1B195B5C9B079B0A9A18A9
:108B7000049B1B195B5C9B071B0A9A18039B1B1920
:108B80005B5C9B079B099A183B195B5C9B071B0965
:108B90009A1803195B5C9B079B089A183319595C58
:108BA0008907891802C51034A0D1029800780421E1
:108BB00001430E48C1630025284611B0F0BD0420D2
:108BC0000090084A2846294602F05CF8F4E70320A2
:108BD0000090044A2846294602F054F8ECE7C046C3
:108BE000E893010228CE00006ECE00000010004085
:108BF000556E646566696E6564206D65616E2050B2
:108C000052462025640D0A00496E76616C69642025
:108C10006D65616E205052462025640D0A000000EB
:108C2000B0B584B00446FBF73EF91F4801680091D7
:108C30004168019181680291C0680390FFF7E2FDED
:108C400000F014FF1948016804220A430260184D1D
:108C50006868A021002C01D1884300E008436860C7
:108C6000FF200230FBF76AFAFBF782FE0020FFF7D5
:108C700021FAFEF7D5F86846FEF782FB0D48016839
:108C8000C907FCD0012080022968814329600A4875
:108C9000FBF754FAFFF7CCFD4B49086000F004FFE6
:108CA000FBF706F904B0B0BD80A0005010ED00E065
:108CB0002C0000402C020040010200007047704769
:108CC00080B50E490E480246083A1268920000D458
:108CD000603142680A4342600A490A6808239A439D
:108CE0000A60091F012252040A60032189040268F4
:108CF0008A430260FBF7F4F880BDC0462000008084
:108D00002800004004020040B0B5032000072D49B0
:108D10000A6882430125680710180860002420466D
:108D2000FFF7CDFF2046FFF7C9FFEFF31080284083
:108D300002D1EFF3108172B68021C943224A5368F1
:108D40000B40536093680B409360D3680B40D36033
:108D500013690B40136153690B405361002800D124
:108D600062B6B0BD70B50C4603210907154A1368F9
:108D70000B4313600122EFF31081114002D1EFF396
:108D8000108272B68025EA430F4B5E6816405E6023
:108D90009E682E439E60DD681540DD601D691540AC
:108DA0001D615D6915405D61002900D162B6002832
:108DB00002D00120FFF783FF002C02D00120FFF733
:108DC0007DFF70BD00040040589501020D4A002946
:108DD00007D001290BD10121814010688843106020
:108DE00007E00121814010680843106001E0012183
:108DF0008140101F02680A430121C9071143016025
:108E00007047C04644000040032804D8400006498B
:108E1000085A00B27047002000B27047032802D8F9
:108E20004000014A11527047EEA701029E490870A6
:108E30007047C04670B58AB00C460546FF20FC302E
:108E4000A8490E68315C59208000335CB2783078D4
:108E500008AE069609AE05960C4E049621267606B7
:108E600003960B4E0296012601960E2600965B1C79
:108E7000DBB2F9F7C5FA0998F7F7C2FC2870089831
:108E8000F7F7BEFC20700AB070BDC046000020415C
:108E900000000443F0B58BB00446457C824800785E
:108EA0008249002822D000200880814A1080814B0E
:108EB00001269E761E830A907F4800787F4E367882
:108EC0006DB205957E4D04957E4D03950AAD0295D4
:108ED0007D4D01950096F8F7D1FF0A9D112020568F
:108EE0007A497B4A00F0B2FD064626E000260E8055
:108EF0006F4A16806F4B01209876188309966E484A
:108F000000786E4F3F786DB205956D4D04956D4DAF
:108F1000039509AD02956C4D01950097F8F7AEFFEA
:108F2000099D112021567F20C005009001900296D6
:108F3000664A674B3046FAF7F5F8432001062846A3
:108F4000F7F795F9F7F75CFC08906248007800287D
:108F500024D05120800060494A7D42438D185F48EB
:108F60000068A8642F46403750480078B8745048CD
:108F70000078F87455480078387555480078787549
:108F800057480078F87550480069F7F739FCB8750C
:108F900052484069E8644C4800686864FF20FE302D
:108FA00050490968085C3922D2008918022812D376
:108FB00003D04E48007801280DD14B480660434845
:108FC00000883A4A108042480088394A10800920B7
:108FD0000790089605E04448089A02603548C08B1F
:108FE00007900B780022002B01D0114600E0D143FE
:108FF0000125002B01D0042300E0EB43A67AAD1B32
:10900000EE175B1971416568AE0F277AAD00ED1957
:109010005641677A3F1FF817ED1970414000EE0F77
:1090200080196D00EB1848418001990E4118980194
:1090300027239B02C31A91411D4805881B480088BD
:10904000854201D00798421B10202056C001194DBF
:109050002D8C032D07D1E468E5176D0A6419E4151A
:109060000519EC170FE0E468E5176D0A6519EC17B0
:10907000ED15C6174519744197B2002F00D034463C
:10908000002F00D00546581BA141130409D012B28D
:10909000D2015242D31780185941089BDA17C01ADF
:1090A00091410BB0F0BDC0467E930102A4A601021F
:1090B000A2A6010240940102819001028090010267
:1090C000909C0102909A0102A8A60102F2A6010258
:1090D000F0A601025CA00102949D01026420004000
:1090E000A0A60102E89301029CA60102F4A60102D7
:1090F000C10D4002803070470120C0071B49086045
:109100007047C04610B519480068C10710D18107E3
:1091100011D4410712D4010713D4C10614D4810617
:1091200015D4410616D48021084016D031A215E08E
:1091300001240FA213E0022411A210E0032414A2C0
:109140000DE0042416A20AE0052419A207E0062473
:109150001CA204E0072421A201E0254A0409022000
:10916000032101F08FFD204610BDC0465C00004089
:10917000526573657420627920504F520D0A0000C9
:10918000526573657420627920424F520D0A0000C7
:1091900052657365742062792050494E0D0A0000B3
:1091A0005265736574206279205744540D0A00009B
:1091B0005265736574206279204C4F434B55500DB6
:1091C0000A000000526573657420627920535720AD
:1091D0005265626F6F740D0A00000000526573657E
:1091E00074206279205359535245510D0A000000F2
:1091F000FECA0000526573657420627920445644AB
:10920000440D0A0001218140044A1F2802D0106841
:109210008843106010680843106070471C000040CD
:10922000F0B583B0029104469949F6F753FF05461D
:10923000984901942046F6F74DFF974946189749FB
:10924000714300956F189649441864212046F6F73B
:1092500041FF3818A108471A92492046F6F750FFF7
:10926000381891494518914F05D464213046F6F7D6
:1092700031FF0C4614E0A6B264213046F6F72AFF0F
:10928000B7204000A20701D1002907D1884B7343C2
:109290000422D341874A934200D3401E0C4645190D
:1092A0000098474302980680192001013046F6F7DE
:1092B00011FF2A461F3A284600DB1046019BFF1883
:1092C000B30705D1002C03D01F2D05DA0120C5E01E
:1092D0001F2D0BDA0120C1E005461D3D034600DBD2
:1092E0002B461C2808DC02201546B7E000290CD0CC
:1092F0001C21451A0CD50CE019461F39184600DB15
:1093000008461F2B1DDA0320A8E01D21451A00D4B2
:109310002846002D08D401461F39024600DB0A46C4
:109320001F2804DA032099E00220154696E015462E
:109330001E3D104600DB28461E2A0CDA04200D468E
:109340008CE005461E3D024600DB2A461E280BDA4D
:1093500004200D4682E001461F39024600DB0A4622
:109360001F280ADA052079E011461F39104600DB74
:1093700008461F2A0BDA052070E015461E3D1046F0
:1093800000DB28461E2A0CDA06200D4666E005465C
:109390001E3D024600DB2A461E280BDA06200D463B
:1093A0005CE001461F39024600DB0A461F280ADA44
:1093B000072053E011461F39104600DB08461F2ADC
:1093C0000BDA07204AE015461F3D134600DB2B460B
:1093D0001F2A0CDA08200D4640E005461F3D0246D4
:1093E00000DB2A461F280BDA08200D4636E0194616
:1093F0001E39184600DB08461E2B0ADA09202DE02C
:1094000011461E39104600DB08461E2A0BDA0920D9
:1094100024E01F28054601DB05461F3D1F280CDA06
:109420000A200D461AE01F28054601DB05461F3DB0
:109430001F2806DA0A200D4610E01E2D05DB0C2041
:1094400004E01E2D06DB0C2005E00B201E2D05DBA5
:109450001E3D03E00B201E2D00DB1E3D029EB07062
:10946000681CF070E12001013846F6F733FE3071D8
:10947000C0B211494143CC193C212046F6F72AFEDF
:1094800070713B21C94341430819B07103B0F0BD6D
:10949000805101008033E101B207000093FEFFFF1D
:1094A000B107000070FEFFFFA7FA0A0080AEFEFFC2
:1094B000295C8FC20BD7A300F0F1FFFF70B5044603
:1094C000FFF722FCA08A244EB082B18A002908D07E
:1094D000F0820220B07100207082FFF76BF9F0611A
:1094E00070BDE08A7082A169728A1C48F6F742FE5C
:1094F0002046FFF7CFFC05460C461948007BFFF7D6
:1095000083FC81B2C90B401800B2C1174010281A61
:1095100030678C417467FFF74DF9B061F06D401C06
:10952000F065FEF7B9F8F064FAF710FC0446306510
:109530000C48406AF7F7DEF90B4A0C4BF6F7C4FF0C
:10954000F7F78CF901462046F6F7DAFDFAF7C6FD83
:109550000120B07170BDC046B8960102F8A70102A3
:10956000829001023CC000008DEDB5A0F7C6B03E70
:10957000F0B581B0EFF3108072B600200146FBF722
:109580006BFE0446002803D062B6204601B0F0BD51
:1095900001273A030025074E28463146FBF7B6FD62
:1095A000BB02054A28463146FCF7B2FA62B62046AD
:1095B00001B0F0BD00E002049AA20102F0B589B04A
:1095C00002F032FCDA4C607802F032FAD9498A882B
:1095D00007A882800A884988090489180791FEF73C
:1095E00023F86078052804D00222D349092804D141
:1095F00004E00122D049092800D08918497920784F
:10960000621C02F0D9FA607AFFF710FCCB48CC4913
:10961000FDF74EFBCB48007800230028069309D0C5
:10962000C9491A31C94A034610CA0C80891C5B1EFD
:10963000FAD10346C64DA872C24FB88D68717A78C8
:109640002A70BA78EA70000AA871501CB8702846CF
:109650000B30BD4C21464C315E0003913246F6F78B
:1096600089FD70190B3021461A313246F6F782FD1A
:10967000202068720698787138896870000AA8708E
:10968000C32006908401FFF795F803193B633878EF
:1096900081000D3101222846059202F012FCB862C9
:1096A0003C6BFFF71DF80019FFF722FD05460E463B
:1096B0009F48007BFFF7A8FB81B2C90B401800B29E
:1096C000C117401028183D46B8667141F966FFF78A
:1096D00071F8B861FDF75CFA0028FBD1FFF76AF872
:1096E000E861286B9B49401868637D2006010024CF
:1096F00020462146324602F0BAFBA862FFF75AF82C
:10970000069909022A784A4393495118A863E963E4
:109710000918481C00D008462864FFF74BF8686415
:10972000296C8E4F0EE00020A8710146324602F0EF
:109730009EFBA862FFF73EF82862FFF73BF8A8619E
:10974000296C686C884202D3C919884277D9FFF71F
:1097500031F86864FFF72EF8E861FDF719FA002880
:10976000FBD1FFF727F82862A8790228DBD001286F
:10977000E6D10020A8717A4A517A21295FD1517926
:1097800093791B025918AB8D994258D16978137897
:109790008B4254D12646517893781B025918E9819F
:1097A0002B79002B2FD02B78002B0BD0664C4C3410
:1097B000002025888D4204D0A41C401C8342F8D18F
:1097C0001846604DC0B228822B6FA96CAC6E15464E
:1097D000223500955B4D0191029411461A311E32DB
:1097E000F9F7BEFE288A2979884208D34100564AF3
:1097F0005118EA894C23CA522978491C29705249C8
:1098000005220A5414E04C204F4B19520598287039
:10981000052018702B6FA86CA96E14462234009492
:109820000190029111461A311E320020F9F798FE7C
:1098300034464B489621F6F7B6FC00206882A86EA5
:10984000E96EF7F7D3FAEC70287800282FD03F485C
:109850004C21254626463C4B06E0069C891C001DF3
:10986000E2B26D1C954219D206945C5D002CF4D0D6
:10987000641E5C55B2000592E4B23A4FBC505C5A8B
:109880007300394FFC52069C641C2E4BDC7003683D
:10989000364A059FD3512C4B761CDFE704922948AA
:1098A000047104700694E0B2022806D228E02C79F4
:1098B00004940694E0B2022822D30498471E0021A3
:1098C000059703E0491C059FB94219D0274A106843
:1098D000254D244C0FE0136050606B882E886E80FD
:1098E0002B8048CC083C266063607F1E121DAD1C97
:1098F000241D002FE6D053689842ECDC1846F4E7AC
:1099000006980006049C10D0620017490398F6F7E9
:1099100031FCA2000D481549F6F72CFC0A4A114803
:1099200002C81170521C641EFAD109B0F0BDC046C5
:1099300082900102F0BF00002C9A010295AE000057
:10994000BD940000B89601023497010240A70102BD
:10995000F2BD0102A06D010080E701000026B803FE
:10996000F8A70102F8BC0102C0BD01025CBD010202
:1099700007488178491C8170C9B2782903D1012137
:109980004170002181700348012141707047C04639
:10999000309701021490010270B514460D46064638
:1099A0001120FAF74BFC2248042101600C480460A6
:1099B0001E4805608660002E0DD0FF200006094974
:1099C0000A6882430120C007101808600648082171
:1099D0000160064801601A200221FFF7F7F970BD07
:1099E00094A8010200E400E080E200E000E100E071
:1099F0000C4908607047C04610B504460948006825
:109A000060430949F6F77CFB00190849486008489B
:109A10000022026002460C3A4B681360096801603C
:109A200010BDC04690A8010240420F0008900102FC
:109A30002C10014000480047C100000080B50249D9
:109A40000968C96D884780BD0090010280B582B069
:109A500013460A4600900348011D0348F9F70EFB20
:109A600002B080BDD0A80102C49901023B48002188
:109A7000016081684068401C534A13685B0104D44C
:109A80000029024609D00A4607E04D490B685B1CD5
:109A90000B60012149061160024649494860801A5D
:109AA000CA688018C860704770B5454E716827480D
:109AB000821C91422AD2491E284A516028490B68CB
:109AC0000340032084071B190B6000219160106084
:109AD000FCF78EFC054674682146F6F7FBFAF16840
:109AE000491922464243891AF160A14204D3091B55
:109AF000401CA142FBD2F160316809183160002896
:109B000003D03069002800D0804770BD104811494B
:109B1000E622114B00F088F810B50C498A1C9042DF
:109B20000DD2401E0D4A50600D4803680B400321C2
:109B30008C071B19036000209060116010BD044861
:109B40000449E622044B00F06FF8C046FFFFFF0017
:109B5000D5CA0000EFCA0000BBCA000010E000E058
:109B600020ED00E0B0B50120EFF31081014002D1FB
:109B7000EFF3108272B6124A1368124C22686468BE
:109B80008506114800682840850E5D192923DB00F1
:109B90006B43002C1D4606D1002809D11E206843C6
:109BA00000290AD0B0BD121BD218551C0028F5D0D0
:109BB0001D461E2068430029F4D162B6B0BDC046E0
:109BC00000B4010214E000E004ED00E080B50020E4
:109BD000FAF740FD404280BDB0B586B010486946F6
:109BE0000A4638C838C238C838C200242046FAF7B6
:109BF00037FD03992046FAF7CDFD0198012803D0DF
:109C00000824002804D102E00424002800D10446DE
:109C10000220FAF71BFBE0400249086006B0B0BD25
:109C2000F8BF000014B4010290B01C4605AB07C396
:109C3000EFF31080C00702D1EFF3108072B6EFF39C
:109C400010800B9068460E907046089010AB0F93F2
:109C5000CF4F3E1D01200490C502304629462246C2
:109C600000F0B8FC00213154EFF303800990EFF3CA
:109C700008800C90EFF309800D90EFF314800A90A8
:109C800000F02CFC3868012833D80028C14F00D0E0
:109C9000C14F2A20C1497A69920703D50A783A60F0
:109CA000401E491C0028F6D1B948041D2046FFF784
:109CB000C5FE002807D079698907FAD5217839606F
:109CC000401E641CF5E70220B5497A69920703D566
:109CD0000A783A60401E491C0028F6D12A20AF4974
:109CE0007A69920703D50A783A60401E491C002819
:109CF000F6D1FFF737FF0346AA4A30462946FDF75B
:109D000009FC04463018291B089F3B1F049A934303
:109D1000A5A2FDF7FFFB9E490968012966D8001935
:109D200000299C4C00D09C4C00280AD09849091D61
:109D30006269920703D50A782260401E491C0028F8
:109D4000F6D10A209F496269920703D50A782260FA
:109D5000401E491C0028F6D10598FFF76FFE002829
:109D600009D061698907FAD5059A11782160401EEA
:109D7000521C0592F3E7022089496269920703D5D4
:109D80000A782260401E491C0028F6D10A208EA1C4
:109D90006269920703D50A782260401E491C002898
:109DA000F6D10698FFF74AFE002809D061698907B5
:109DB000FAD5069A11782160401E521C0692F3E7EC
:109DC000022077496269920703D50A782260401E13
:109DD000491C0028F6D10A207EA16269920703D5AA
:109DE0000A782260401E491C0028F6D17CA2304629
:109DF0002946079BFDF78EFB6549096801290E9BE3
:109E00001BD80029634900D0634900280AD0604A62
:109E1000121D4C69A40703D514780C60401E521C17
:109E20000028F6D102205E4A4C69A40703D51478B5
:109E30000C60401E521C0028F6D16AA2304629460A
:109E4000FDF768FB04463018291B694A3B46FDF7BD
:109E500061FB4F490968012911D8001900294D49B2
:109E600000D04D4900280AD0494A121D4B699B0772
:109E700003D513780B60401E521C0028F6D15D4AB2
:109E800030462946099F3B46FDF744FB0446F8004F
:109E9000C00FB900C90F7A00D20F00920191029051
:109EA0003019291BFB0F544AFDF734FB04193019F4
:109EB000291B3F233B40514AFDF72CFB34490968DD
:109EC000012911D820180029324900D03249002830
:109ED0000AD02F4A121D4B699B0703D513780B60DC
:109EE000401E521C0028F6D1454A304629460B9B9D
:109EF000FDF710FB04463018291B424A0A9BFDF768
:109F000009FB23490968012911D8001900292149B1
:109F100000D0214900280AD01D4A121D4B699B0719
:109F200003D513780B60401E521C0028F6D1364A28
:109F3000304629460C9BFDF7EDFA04463018291BE4
:109F4000324A0D9BFDF7E6FA114909680129114AC9
:109F50000DD80019002908D00F4A06E05169890779
:109F600003D531781160401E761C0028F6D12849AF
:109F70000E98091AA94200D32946890800F00CFE60
:109F800024480068002800D0804700F045F8C0460B
:109F9000E4B401020090014000A001402FCB00007A
:109FA00092CE000018CB00000D0A2323232041533A
:109FB00053455254204020307825303858202323F0
:109FC000230D0A00F2CB000046554E4354494F4E34
:109FD0003A2000004C494E45202020203A20000025
:109FE000256400000D0A53503D253038580D0A00F5
:109FF000B7CB0000CDCB0000D9CB0000C1CB000017
:10A0000076CB000085CB000094CB00009FCB0000F6
:10A0100000F80202E0B40102F7480068012811D8F4
:10A02000002801D00B4800E0FC480C210A4A01E05E
:10A03000002907D043699B07FAD513780360491EAE
:10A04000521CF5E71E20FFF7DDF800BF00BF00BF80
:10A0500000BFFAE700A0014022CB00008AB006460C
:10A06000E448B06600F03AFAFFF77CFD0346E248A8
:10A07000041D01200590C502E04A20462946FDF74F
:10A0800049FA074608942018DB4C0995E91BF36C44
:10A090003F2206921340DAA2FDF73CFA216801291B
:10A0A00010D8C0190029DD4900D0DD49002809D0A9
:10A0B000221D4B699B0703D513780B60401E521C71
:10A0C0000028F6D1F36BD7A2089C2046099D2946AB
:10A0D000FDF720FA0746291A2018336C069A134018
:10A0E00007D1D8A2FDF716FAC34C2168012907D978
:10A0F00017E0CEA2FDF70EFABF4C2168012910D857
:10A10000C0190029C54900D0C549002809D0221D21
:10A110004B699B0703D513780B60401E521C002827
:10A12000F6D10027CBA5B8003058009008980999BF
:10A130002A463B46FDF7EEF9216801290FD8002990
:10A14000B64900D0B649002809D0221D4B699B07AB
:10A1500003D513780B60401E521C0028F6D17F1CDB
:10A160000D2FE0D1736BBFA2089C2046099D2946A4
:10A17000FDF7D0F9074620189F4CE91BB36BBC4A8A
:10A18000FDF7C8F92168012910D8C0190029A34991
:10A1900000D0A349002809D0221D4B699B0703D595
:10A1A00013780B60401E521C0028F6D1336CB14A64
:10A1B000089C2046099D2946FDF7ACF90746326CFC
:10A1C000D000C00F9100C90F5300DB0F0093019125
:10A1D0000290E019E91BD30FA74AFDF79BF932461D
:10A1E000C619A019A91B1546136C069A1340A34A59
:10A1F000FDF790F980490968012911D880190029D3
:10A20000864900D0864900280AD07B4A121D4B6936
:10A210009B0703D513780B60401E521C0028F6D113
:10A220002E466B6C964A089C2046099D2946FDF7F0
:10A2300071F907462018E91B0796B36C914AFDF7A0
:10A2400069F96D4A1168012910D8C01900297349AC
:10A2500000D07349002809D0121D4B699B0703D514
:10A2600013780B60401E521C0028F6D10798426EEE
:10A27000042360215C2004931A400B4600D003465F
:10A280000693002A00D00846079E33587E4A089C51
:10A290002046099D2946FDF73DF9074606983358A3
:10A2A000E019E91B794AFDF735F9C619A019A91B70
:10A2B000079A536E76A2FDF72DF94F4909680229D6
:10A2C00011D280190029554900D0554900280AD0DB
:10A2D000494A121D4B699B0703D513780B60401E3A
:10A2E000521C0028F6D10798C36C06466DA2089C44
:10A2F0002046099D2946FDF70DF907462018E91B60
:10A30000336D6B4AFDF706F9C619A019A91B079F03
:10A310007B6D68A2FDF7FEF88619A019A91BBB6D1D
:10A3200067A2FDF7F7F8344909680129059C11D89F
:10A3300080190029394900D0394900280AD02E4A0D
:10A34000121D4B699B0703D513780B60401E521CEE
:10A350000028F6D10798476B5D4A974237D2032011
:10A3600087430026059CB00039580246049B1A43D7
:10A37000BA5808230343FB580C2505437D59009127
:10A380000192029303953B1808980999514AFDF7E9
:10A39000C1F81949096801290FD800291F4900D0BF
:10A3A0001F49002809D0089A4B699B0703D51378E9
:10A3B0000B60401E521C0028F6D11B2E444A06D8C2
:10A3C0000798406B361DB10040189042CBD30798D8
:10A3D000406B111A099A914201D8890800E0610284
:10A3E00000F0DAFB3C480068002800D08047FFF707
:10A3F00013FEC04622224B4DE4B4010218CB0000EC
:10A400000D0A0D0A23232320455843455054494F34
:10A410004E202564202323230D0A000000900140D4
:10A4200000A0014050433D25303858002C2045788D
:10A4300063657074696F6E4E756D6265723D2564FB
:10A440000D0A00002C205468726561644D6F6465CC
:10A450000D0A000052252D32643D253038580D0A72
:10A460000000000053503D253038580D0A00000010
:10A47000B7CB0000CDCB0000D9CB0000C1CB000092
:10A4800076CB000085CB000094CB00009FCB000072
:10A490004558435F52455455524E3D253038580D6E
:10A4A0000A000000494353523D253038580D0A0038
:10A4B000AACB00005343523D253038580D0A000006
:10A4C0004343523D253038580D0A0D0A0000000064
:10A4D00000F802025ACB0000E0B40102F0B583B0EC
:10A4E000344D2C68012C06D8601E8441204601F0B2
:10A4F0007BFA0028FAD10120EFF31081014001918D
:10A5000002D1EFF3108072B62B48285A2B49695AB2
:10A51000814245D02A68002A01D02A4E00E0284E08
:10A520001F23DB020293284C022A27D205E01046A3
:10A53000214AA85282B2914232D087B2B9420A4629
:10A5400000D8621C131A21482B5218040DD0E819A8
:10A55000001D9FB201E0002F07D073699B07FAD559
:10A56000037833607F1E401CF5E7A242DFD90298D2
:10A570001018DDE7304683B299420CD0024680B213
:10A5800081420E4600D8661CA642F3D902983018C4
:10A5900083B29942F2D108496852B01A0B49685205
:10A5A0000B48002129540198002800D162B603B05D
:10A5B000F0BDC046E4B401020A080000080800002B
:10A5C0000090014000A00140FF0700000C080000BF
:10A5D0000F080000F0B58DB00793174600240C94C7
:10A5E00009AA13C215E006986849F5F740FEF6F788
:10A5F00007F9C117401848406549F5F76BFD00950C
:10A6000009A806223346F9F705FABDE0002C00D56B
:10A61000BEE138787F1C25280DD0002800D1B7E195
:10A620000B9A511C0A9B9942F0D8099B9854641CC0
:10A630000C940B91EAE708940025397823390D2909
:10A6400014D801207944097949008F44090F0F0F6C
:10A650000F0F0F0F0B0F060F0F0D05437F1CECE7BD
:10A660000820FAE70420F8E70220F6E738780146E8
:10A6700030390024092902D9264639460BE0002644
:10A680000A2171430E18303E791C78780246303A20
:10A690000A2A0F46F4D32E2817D14A1C48780146BF
:10A6A0003039092905D911464F1C2538532811D9AD
:10A6B0006AE000240A2161430C18303C511C507898
:10A6C0000246303A0A2A0A46F4D34F1C253853284A
:10A6D00000D959E04000C046784480884000874453
:10A6E000A000530053005300530053005300530085
:10A6F00053005300530053005300530053005300C2
:10A7000053005300530053005300530053005300B1
:10A7100053005300530053005300530053005300A1
:10A720005300600053005300530053005300530084
:10A730005300530053005300530053005300530081
:10A74000530053005300980053005300530053002C
:10A75000530053005300530053005300AD00B600A4
:10A760005300600053005900530053005300590038
:10A77000530053005300DE0053005300BD0053004C
:10A78000D3005300530098000C9C3FE70024744909
:10A7900040420F00791C38780F4625385328F3D8EB
:10A7A00098E70799C91D0720814308680791496800
:10A7B000F6F7B4F800210690F5F782FF00280BD1D8
:10A7C0000B99481C0A9A904206D8099A2D23535493
:10A7D0000899491C0C910B9007980830079006982F
:10A7E000F6F70EF80095C2178118514009A82246C5
:10A7F0003346F9F70FF90B98411C0A9A914200D998
:10A80000F1E6099A2E2313540B910C98401C0C90DE
:10A81000E9E6079802C807900096019509A810225A
:10A8200039E00B98411C0A9A9142ADD8099A252328
:10A8300013540B910C98401C0C90A5E70B9A511CDB
:10A84000079C201D0A9B994239D907909CE70798DD
:10A8500002C80790009509A82246D3E6079901C9C6
:10A86000079109990A9A089E02E0401C002E8BD499
:10A870000378002B88D00B9D6C1C9442F5D84B5567
:10A88000761C0C960B94F0E7079802C80790009688
:10A89000019509A80A222346F9F75AF974E7079B9C
:10A8A00010CB102C079308D300202146401C0A0926
:10A8B000FF291146FAD806280AD8082009E023689B
:10A8C000099CA354089A521C0C920B9107905BE7C9
:10A8D000401C069009230C980B9D099905910A9E2E
:10A8E00004940DE0202104463046059E715506462D
:10A8F0002046049C401C15460146089100290AD4B4
:10A900005B1E0699994206D26A1CB242EAD908999E
:10A9100008910029F4D50C900B950898002800D5D3
:10A9200032E70126082501E06D1E3601022DFBD21B
:10A9300020463146F5F7CEFB0F28F6D80C98059047
:10A94000099803900A9806900B9D20463146F5F72A
:10A95000C1FB691C069A914204D908990891002903
:10A960000CD511E00C4A125C039B5A55089A521CF4
:10A970000D46059211460891002905D47043241A0A
:10A980003009102E0646E0D205980C900B95FBE698
:10A9900020460DB0F0BDC0467CC20000F0B583B0CB
:10A9A0000C460023D943012C56DB074602910126B1
:10A9B000EFF31085354002D1EFF3108072B658499D
:10A9C000584A505C002800D0A3E056545F48115A02
:10A9D0005F48105A0196F202161A814240D8324658
:10A9E0005218A24240DB00930295A642354600DB96
:10A9F00025464C490818001D39462A46F5F7BAFB8A
:10AA0000A642484E04DA7919621B301DF5F7B2FBF5
:10AA10004F48305A001981B24E4A914201D94E49ED
:10AA20004018029D009B4A49705230464B4E805D53
:10AA3000002865D1EFF310850198054002D1EFF3AE
:10AA4000108072B6374A4148115A4148105A88421C
:10AA500032D1434813524FE00C46204603B0F0BDBC
:10AA600042425218A242BEDA3C4A2E4EB25C002A42
:10AA70000CD03B4AB25A51188AB2364CA242284CEA
:10AA8000029F01D9344A8918314A02E0244C304AE5
:10AA9000029F3355B152421A89B2884202D22D48E0
:10AAA0008018421C93B23048012130A200F0EAF82D
:10AAB0003C46002DD1D128E0019F9755884201D80E
:10AAC0002448401C421A90B2800A01D001988202A8
:10AAD0002348144F3A52386801280DD8431E984134
:10AAE000104B5918091D92B21E4B00F017FE009B27
:10AAF000002801D00B488355002D029D00D162B67D
:10AB0000074808490B54002DA7D162B6204603B070
:10AB1000F0BD054805A1094A09A3FFF785F8C0461D
:10AB20000E080000E4B401026ECC00007472616390
:10AB3000655F6F7574707574000000000E02000090
:10AB40005452414345204255535900000A08000021
:10AB500008080000FF07000000F8FFFF0F080000D2
:10AB60000C080000B1AD000002FF00000D0A547295
:10AB7000616365206275666665722069732066751B
:10AB80006C6C2C206469736361726473202575207A
:10AB900062797465730D0A00F0B587B0054600262A
:10ABA00006960596049603960296800701D007B094
:10ABB000F0BD019102A8142126A2FCF7ABFC2949A3
:10ABC0000968012911D80029274900D02749002800
:10ABD0000BD002AA01E0002807D04B699B07FAD5E9
:10ABE00013780B60401E521CF5E701990029DED056
:10ABF000204C3746B8002B58D80724D0581EA04206
:10AC000004D31B4818181C4A90421CD802A81421CF
:10AC10001AA2FCF77FFC13490968012911D8002901
:10AC2000114900D0114900280BD002AA01E00028E8
:10AC300007D04B699B07FAD513780B60401E521C56
:10AC4000F5E7761C01997F1C8F42B0D2322ED1D30A
:10AC5000ADE7C0460D0A4261636B74726163653A89
:10AC6000200D0A00E4B401020090014000A0014060
:10AC7000FFFFFFFCFFFF0200FEFF010025303858F8
:10AC80000D0A000081B0F0B5C4B00E4607464993E6
:10AC9000812000012F49085C002845D00292012044
:10ACA000050204A82946F5F77EFAFCB20021C84344
:10ACB0000C2C3AD8721E032A37D82748005DB042C0
:10ACC000084632D3F80535D50021B8050DD404A8BF
:10ACD00001904018691AA20022A39B582E4AFCF743
:10ACE00019FC0198FEF7AAFE014678050ED404AFC0
:10ACF0007818691AB20029A3D218121F1368264ABD
:10AD0000FCF708FC3846FEF799FE0146029A04AEAD
:10AD100070180C46691A49AB0393FFF75BFC0119E5
:10AD20003046FFF73BFE00E0002044B0F0BC02BC20
:10AD300001B00847FEF716FF034604A8019007A2DA
:10AD40002946FCF7E7FB0198FEF778FE0146B805B7
:10AD5000BDD5CAE7E4B4010275DA000025313075CB
:10AD6000207C200012CC000068CC000062CC0000E7
:10AD700041CC00000CCC00002DCC00005BCC0000CE
:10AD800054CC00004FCC000005CC000018CC0000D3
:10AD900028CC0000FDCB000089CC000047CC00008F
:10ADA00033CC00003ACC00001ECC000000000000B4
:10ADB000F0B581B00B460120EFF31084044002D1BE
:10ADC000EFF3108172B6990F07D0022001212DA256
:10ADD000FFF758FF002C3DD141E02249224D0027CA
:10ADE0006F54224AAB5A224AAE5AF3189EB2F60A60
:10ADF00001D0204E9B19AB52EFF31086064002D1D2
:10AE0000EFF3108372B6AA5A1C4BEB5A934202D14D
:10AE100016482F521AE06854934201D8164B5B1C17
:10AE20009B1A99B2890A00D0830210482B522868D5
:10AE300001280BD8411E8841A918091D9AB2104B50
:10AE400000F06CFC002801D006482F54002E03D0DF
:10AE5000002C04D001B0F0BD62B6002CFAD162B66D
:10AE600001B0F0BD0F080000E4B401020C080000BE
:10AE70000A08000000F8FFFFFF07000008080000B4
:10AE8000B1AD000055415254204572726F722025B9
:10AE9000780D0A0010B50446FDF736FFA08A002899
:10AEA00000D010BD0A4CA06D401CA065FDF782FCCF
:10AEB0006062606D002805D0FDF77CFC60660020B4
:10AEC000606510BDA06920660120606510BDC046A8
:10AED000B896010270B5012801D9012070BD482241
:10AEE0004243734B9C58A5691F218D43A5610625DC
:10AEF000A5600F2525629C18A27C002A05D1627CE2
:10AF0000002A02D1227C002A14D06368002B11D4BD
:10AF1000251D0B40012216469E400C4B1E60BFF3C0
:10AF20004F8FBFF36F8F2B68002B03D40B409A40D9
:10AF300007490A60002803D0012804D1092000E055
:10AF40000820F9F773F90020A06170BD80E100E0EE
:10AF500080E200E0F0B585B00D460278E348C368B2
:10AF6000934219D0446D944216D08368934203D023
:10AF7000016D914200D07FE09B1A591E8B410493D2
:10AF800048215943032D46D14418E16900294ED088
:10AF90001C34002020606DE09B1A5A1E93410493DC
:10AFA000032D1AD1039548225A438418A26B01211C
:10AFB000EFF310850D4002D1EFF3108772B6A76949
:10AFC0001026B743A761A669002E01D1183421606D
:10AFD000002D00D162B6039D0CE048215943421870
:10AFE00091691832302902D0116810294CD1802182
:10AFF00011600022482159434018002181630162F9
:10B000008162243000210160002A33D004A829463F
:10B01000904705B0F0BD421891691832302902D02E
:10B020001168202939D180211160002216E0039592
:10B03000E26B0126EFF31085354002D1EFF310816A
:10B0400072B6A1692027B943A161A169002901D184
:10B0500018342660002D00D162B6039D4821594363
:10B0600040180021C163C16241633030002101609A
:10B07000002ACBD105B0F0BD00920E4A2E329C487A
:10B080000D490E4BFEF7D0FD1068009301909848D3
:10B090000949084A0A4BFEF7C7FD10680093019062
:10B0A000044A243292480449054BFEF7BDFDC046D0
:10B0B00080940102B1020000EDCC0000C2CC00007F
:10B0C000A6CC0000F0B585B0049048210A46424362
:10B0D000864B9C58E6690F2535409A18167C002E41
:10B0E00031D04F2040026169014200D185E0A06962
:10B0F00004218843A0610220206201208107691891
:10B10000D161D36BEFF31084044002D1EFF31085CB
:10B1100072B695692026B54395619569002D00D1D9
:10B1200073E010463C30002C00D162B6002404606D
:10B13000D4625463303200201060002B63D004A826
:10B14000984705B0F0BD0C2D5DD8C0467D442D79E3
:10B150006D00AF4467586B580658A163585858584B
:10B1600006009569202D04D0154618352D68302D20
:10B1700049D1156B566B3432AE4217D26669360729
:10B1800014D5646815686E1C166048431818C06AA8
:10B19000445504980C4644431A19156B566B3432C7
:10B1A000AE4203D21C5966693607EAD41268AA4235
:10B1B00029D14143585882690524A24382615A1813
:10B1C000D36B0121EFF31080084002D1EFF310841C
:10B1D00072B694692025AC4394619469002C02D125
:10B1E00014461834216014463C34002800D162B65D
:10B1F00000212160D16251639CE70C2D00D176E7DC
:10B20000012D00D173E705B0F0BD15461835286053
:10B2100010463C30002C00D187E787E704202062ED
:10B2200005B0F0BD0120206205B0F0BD0825256203
:10B23000164618369569102D02D03568302D4BD141
:10B240000396566A15462835976AB74228D1A069F1
:10B2500002218843A061936B0121EFF31080084025
:10B2600002D1EFF3108472B6039E34681027BC43FA
:10B2700034603468002C00D1316014463834002822
:10B2800000D162B6002121602960116224320020C1
:10B290001060002BB7D052E70220206205B0F0BD4D
:10B2A0002A68B242AFD262699207ACD52A68561CAE
:10B2B0002E6048431818006A805C206004980A4693
:10B2C00042439D18AC6A6E6AB4429CD228359C58A1
:10B2D00062699207EAD496E73168009001910448C8
:10B2E00004A1094A09A3FEF79FFCC046809401020D
:10B2F0008CCC0000756172745F6972715F68616EF9
:10B30000646C6572000000003D03000055617274BA
:10B3100020256420737461746520676F65732077DE
:10B32000726F6E6720256400F0B585B00E46054645
:10B33000022804D3002E02D1012005B0F0BD002D5B
:10B3400003D0012D08D1092400E008242046F8F795
:10B3500075FF2046FDF756FF48216943E74A5058DC
:10B3600083691F240294A3438361062383600F2310
:10B370000193036257180023BB62BB63FB633B620C
:10B380007B62FB623B63317F3974727F7A74B27F78
:10B39000BA7404937B637368B268F46892002243C2
:10B3A0005B1E032B0ED8C0467B441B795B009F4479
:10B3B00001050307082304E0282302E0182300E026
:10B3C00038231A43C260C907090F72699201D2B2C9
:10B3D0008918B2699207920E8918491C81607961B7
:10B3E0003169012901D122210161012D5CD8316827
:10B3F0000E2959D23846123003900324002D01D073
:10B40000204600E004204C432D490E19B178F8F78E
:10B41000A5FF3968CA68802510462843C8602848B7
:10B42000005D73781B021818C862AA43CA60F8F757
:10B43000DDFF03980078002809D1384611300078E4
:10B44000002804D1384610300078002827D07868CA
:10B45000002815D4032102468A431B495358840708
:10B46000E40EFF26A640B343A5401D435550029964
:10B47000014001208840A2490860144908600EE09C
:10B480008107C90EFF228A40019C0440083C03202A
:10B4900084430C48235893438D401D43255001207D
:10B4A000B861049805B0F0BD02480349DA22034BA5
:10B4B000FEF7BAFB8CCC0000FFCC0000DCCC000017
:10B4C00010C000001CED00E000E400E000E100E03E
:10B4D000F0B58FB00E900125002900D14BE0039309
:10B4E00004910592002A00D145E00121EFF310827A
:10B4F00001910A4002D1EFF3108172B648270297FA
:10B5000047437E49CE19B5690023302D23D83146F3
:10B510001831C0467D442D796D00AF442024262685
:10B520002626262626262626262626265E26262683
:10B5300026262626262626262626262618262626B9
:10B5400026262626262626262626262618000223F6
:10B55000002A0CD00CE0402D01D0802D05D1012314
:10B56000002A04D004E020240C60002A00D162B636
:10B570001D46002B02D028460FB0F0BD0025756394
:10B580000399F1630499F162059931635B4CE359C6
:10B5900059691322D202114205D0062199600F2168
:10B5A000196271699960317C00290CD0F5610995A7
:10B5B0000895079506950D950B9502210A9101288E
:10B5C00010D017200FE0717C9A6900292CD09520AB
:10B5D00002439A6128460FB0F0BD30240C60002A67
:10B5E000C5D0C5E71920049F0C907068002805D4C9
:10B5F0001F21084001998140414801601420986151
:10B60000B06806A9F8F762FF0E98029941436018E6
:10B6100080686158F34A0092091D3A46059BF8F785
:10B62000C5FF28460FB0F0BD3436110602D5802183
:10B630008A439A6131680025059A91422DD2059579
:10B640005D694F214A0215421BD1E90502D4029CD3
:10B65000EC4F0AE0596833685C1C3460029C60431C
:10B66000E84F3818C06AC1540E98214641437E18ED
:10B67000736B346BA34238D234367B585D69154204
:10B68000E3D002211962019EB10729433546DD4C02
:10B69000EFF31082324006D008E02946019EEFF316
:10B6A0001082324002D1EFF3108372B6029B434303
:10B6B000E01883692024A34383618369002B05D0AC
:10B6C000002A08D0C26B002A0AD154E70346183377
:10B6D0001E60002AF6D162B6C26B002A00D14AE78A
:10B6E0000EA8904728460FB0F0BD2946059D019E43
:10B6F0003C46EFF310823240D5D0D7E78094010268
:10B7000080E200E080B5012002496422024BFFF78D
:10B71000DFFE80BDF495010205B70000F0B591B0E1
:10B7200010900126002900D19BE003930591002A87
:10B7300000D196E007900121EFF3108002910840BC
:10B7400002D1EFF3108172B6049248230693079951
:10B750004B43AC49C9188D690026302D6ED80C4674
:10B760001834AD00374602A675593E46AF46C0466E
:10B7700045B800004DB8000051B8000051B80000B5
:10B7800051B8000051B8000051B8000051B8000095
:10B7900051B8000051B8000051B8000051B8000085
:10B7A00051B8000051B8000051B8000051B8000075
:10B7B00035B8000051B8000051B8000051B8000081
:10B7C00051B8000051B8000051B8000051B8000055
:10B7D00051B8000051B8000051B8000051B8000045
:10B7E00051B8000051B8000051B8000051B8000035
:10B7F000E3B8000051B8000051B8000051B8000093
:10B8000051B8000051B8000051B8000051B8000014
:10B8100051B8000051B8000051B8000051B8000004
:10B8200051B8000051B8000051B8000051B80000F4
:10B8300035B80000022600280CD00CE0402D01D0C5
:10B84000802D05D10126002804D004E010252560B4
:10B85000002800D162B6002E069D6A4F049C07980E
:10B8600002D0304611B0F0BD00268E62039A8A6382
:10B87000059A0A624C620A7C002A0BD00C960B9641
:10B880000A96099608960E9602220D9201282DD04E
:10B8900018202CE08A7C2831002A3BD00A68A2427A
:10B8A00016D22B464343FA585469A40710D50868AA
:10B8B000441C0C60F918096A085C1060109829464D
:10B8C00041437A1811462831936A526A9342E8D369
:10B8D00045437859816982220A438261304611B01A
:10B8E000F0BD302525600028B4D0B4E71A200F90B1
:10B8F000C86808A9F8F7EAFD109845437A597819FD
:10B90000C0683849009105992346F8F74FFE304644
:10B9100011B0F0BDFB589A69140602D58024A243E9
:10B920009A610A680026049882422ED25D694F22ED
:10B930005202154207980AD002211962029EB107ED
:10B9400029431FE028315D6915423E46F4D1374650
:10B950005C69A40702D406992A4E0AE00C68661CAA
:10B960000E6006994843274E3018006A005D186043
:10B9700010984143735871188C6A4E6AB442E1D3EF
:10B9800029463E46069D1F4F01E0314607985A6AF8
:10B99000002AFCD1EFF31082029B1A4002D1EFF390
:10B9A000108372B64543781983691024A3438361D9
:10B9B0008369002B05D0002A09D0826B002A0BD1A5
:10B9C0004FE703461833029C1C60002AF5D162B68B
:10B9D000826B002A00D144E710A89047304611B08E
:10B9E000F0BDC04655AF000048214143054842180C
:10B9F0009269D20601D40020704740584169012065
:10BA0000084070478094010205480068202803D050
:10BA100005480649086070470248044908607047B5
:10BA20000C00004024D6010330CF01030090010236
:10BA3000F0B587B001460127022505283A4600D017
:10BA40002A4600200929014600D01146C900374A7C
:10BA500054180E210591615EFDF7E0F91026A15FF3
:10BA60003846FDF7DBF91227E15F2846FDF7D6F9E6
:10BA700006951425615F03200490FDF7CFF9059822
:10BA8000235EA05FE15F625F00AD07C528A2069F4D
:10BA90003846049D2946FFF7F5F82046263004264F
:10BAA0003146FBF7A1FD2620235E2820205E2A21B7
:10BAB000615E2C22A25E00900191029224A238467F
:10BAC0002946FFF7DFF827463E3738463146FBF771
:10BAD000A9FD3E20235E06983C5EB95F0622BA5E51
:10BAE00000940191029221A207462E462946FFF7B3
:10BAF000C9F856240D4D285FFBF788FD2B5F2C46B7
:10BB000021A2384631463546FFF7BCF8264658365E
:10BB10003046FBF767FD5820235EF05F00901FA2C0
:10BB200038462946FFF7AEF807B0F0BD2C9A01025F
:10BB3000546F4620616E742064656C6179732025B2
:10BB4000642025642025642025640D0A000000007F
:10BB500050446F412064656C617973202564202511
:10BB6000642025642025640D0A00000050446F41C4
:10BB7000206761696E732025642025642025642078
:10BB800025640D0A0000000050446F4120616E746E
:10BB90002073706163652025640D0A0050446F4175
:10BBA00020616E676C65206F66667365747320250F
:10BBB000642025640D0A0000F0B587B01546774B68
:10BBC0001A680F24A2432F783A431A60744C234614
:10BBD0002C3B744A1A60049003462246283A1268A5
:10BBE0001207FAD5704E092F0291039306D97249B4
:10BBF000316071600C2F09D171480FE0042F07D913
:10BC00006C4931606C497160092F06D36D4805E0BD
:10BC1000664830607060664800E068486A490860BD
:10BC2000EB7AFF2B02D10020B0620AE003210B4027
:10BC30006648C05C40220243B2620220644AFFF7B9
:10BC400021F8039F0021384605952A460B46FBF74D
:10BC500055FD0646022503215EA228460191334682
:10BC6000FFF710F806963046FCF71CFA01210498FD
:10BC7000009108402CD13D4033D15C4900283AD195
:10BC8000002D1ED06048A062E062206360635F48C0
:10BC900060625F480860152085046E1C8E608D60B0
:10BCA000642420460F46F8F7A1FB3E603D60204625
:10BCB000F8F79CFB281D38605648032156A2FEF772
:10BCC000E1FF0598007BFAF76BFE069807B0F0BD20
:10BCD0002E4605460698FCF7FDFD284635463D40B4
:10BCE000CBD02E4605460698FCF712FA2846354674
:10BCF0003E490028C4D03E4808613E4848613E485D
:10BD000088611520C8613D48016840220A430260ED
:10BD100007210803244B5A698243009840031018F6
:10BD200058610522029842432748036898182F4E0D
:10BD3000766B47780F40995C0907490EC919CA0309
:10BD40002F4B33409A18C90151182E4A8918274A97
:10BD500051632649896B3822914382785207920EAB
:10BD6000891804220A4321498A630F4E31690279F6
:10BD7000019B1A40C0784007C00E80181F229143D3
:10BD80000818306155204003411C21602060642068
:10BD9000F8F72CFB1549002D93D073E704040040FD
:10BDA0002C60004000040080000600400F040F04D7
:10BDB00091C600000304030400040004C2C700008D
:10BDC00060C50000F3C80000EC93010224CA000023
:10BDD0000DCD000050485920706172616D73207361
:10BDE00065747320253038780D0A0000906000409B
:10BDF00012A83E009DD79B5AD579BD493402004018
:10BE00003F0080FF404000002008820002D50F0064
:10BE100002025500020800007577625F72785F6960
:10BE20006E69740D0A000000B0B51820FDF7EAF93C
:10BE30001920FDF7E7F9002420462146F7F730FFE7
:10BE400020462146FAF730FD012503217F232846AD
:10BE50000A46FAF73BFE2846FBF710F80220FBF7EC
:10BE60002DFC28462946FCF7A9FC2046B0BDF0B5BC
:10BE700081B0164600910446002001273946FCF7A0
:10BE800071FFEFF310853D4002D1EFF3108072B6E1
:10BE90002720400170430A21F4F71CF90246002CC8
:10BEA00002D00020009901E002200021FAF7ECFF07
:10BEB0000446FBF7B1F8002D00D162B6204601B070
:10BEC000F0BDF0B581B01D460E460446022A09D1E8
:10BED000012738463946FCF745FF009600223846D0
:10BEE00029460FE0174601200021FCF73BFF012FF8
:10BEF00004D1009600202946024603E00096022065
:10BF000000210A462346FBF79FF80446FBF784F816
:10BF1000204601B0F0BD000070B5002801D001201E
:10BF200070BD0325A9020F4802680F4B535000242F
:10BF30009460012253030D4E3360BFF34F8FBFF364
:10BF40006F8F0B4E336003685A5084720481102047
:10BF5000F8F76CF9022007A22946FEF793FE204667
:10BF600070BDC0461095010251E5CC1A80E100E099
:10BF700080E200E057445420636C6F73650D0A0043
:10BF80002021020C01D010211046020A01D01046D7
:10BF90000839020901D01046091F820801D0104655
:10BFA000891E420801D0881E7047081A704702E0B7
:10BFB00008C8121F08C1002AFAD170477047002034
:10BFC00001E001C1121F002AFBD17047000084C1AB
:10BFD000000008C10000C03F000038410000AC4133
:10BFE0000000D44108400800000810080408102090
:10BFF0002800040000000000000000000000000015
:10C0000001000000FFFFFFFF000000000000000033
:10C0100059062014032145012882003241003219BB
:10C0200000411300390300B506002D03002D020066
:10C030002201002201003E01002000008009EE4D97
:10C040005048504F80096E4F58E5854F80096E4F1C
:10C05000B867C14F5048D04FB867C14FE828DF4F8D
:10C060008009EE4F18EAFC4F8009EE4F58E5055065
:10C07000A4550D50F0C51450A4550D5000002110CA
:10C08000422063308440A550C660E7700881299142
:10C090004AA16BB18CC1ADD1CEE1EFF131121002EA
:10C0A00073325222B5529442F772D6623993188392
:10C0B0007BB35AA3BDD39CC3FFF3DEE362244334B6
:10C0C00020040114E664C774A44485546AA54BB5E2
:10C0D00028850995EEE5CFF5ACC58DD5533672268A
:10C0E00011163006D776F6669556B4465BB77AA732
:10C0F00019973887DFF7FEE79DD7BCC7C448E558D6
:10C100008668A7784008611802282338CCC9EDD981
:10C110008EE9AFF9488969990AA92BB9F55AD44A29
:10C12000B77A966A711A500A333A122AFDDBDCCBD1
:10C13000BFFB9EEB799B588B3BBB1AABA66C877CF5
:10C14000E44CC55C222C033C600C411CAEED8FFD21
:10C15000ECCDCDDD2AAD0BBD688D499D977EB66EC9
:10C16000D55EF44E133E322E511E700E9FFFBEEF71
:10C17000DDDFFCCF1BBF3AAF599F788F8891A98133
:10C18000CAB1EBA10CD12DC14EF16FE18010A1001D
:10C19000C230E3200450254046706760B98398930D
:10C1A000FBA3DAB33DC31CD37FE35EF3B10290126D
:10C1B000F322D2323542145277625672EAB5CBA5D9
:10C1C000A89589856EF54FE52CD50DC5E234C324BD
:10C1D000A01481046674476424540544DBA7FAB7AD
:10C1E0009987B8975FE77EF71DC73CD7D326F2360D
:10C1F0009106B01657667676154634564CD96DC9F9
:10C200000EF92FE9C899E9898AB9ABA9445865485C
:10C2100006782768C018E1088238A3287DCB5CDB4C
:10C220003FEB1EFBF98BD89BBBAB9ABB754A545AAC
:10C23000376A167AF10AD01AB32A923A2EFD0FED18
:10C240006CDD4DCDAABD8BADE89DC98D267C076CFC
:10C25000645C454CA23C832CE01CC10C1FEF3EFFEC
:10C260005DCF7CDF9BAFBABFD98FF89F176E367E4C
:10C27000554E745E932EB23ED10EF01E30313233E5
:10C280003435363738394142434445461000400082
:10C2900080000001000200040008001010001800D7
:10C2A000200030004000600080000001FFFFFFFF21
:10C2B00001FF01FFFF0101FFFF010000000000007E
:10C2C000000000000000000000000000000000006E
:10C2D0000200000000000000140000000200000046
:10C2E0000700000002000000020000000000000043
:10C2F0000200000000000000140000000200000026
:10C300000100000002000000020000000200000026
:10C31000000000001400000000000000FFFFFFFF0D
:10C32000FFFFFF01FFFF01FFFF01FF01FF01FFFF13
:10C33000FF0101FFFFFF01FF0101FFFF000100FFFF
:10C34000010000FF000064009E00C800E800020138
:10C3500019012C013D014C015A01660172017D0158
:10C36000870190019901A101A901B001B701BE01A6
:10C37000C401CA01D001D601DB01E101E601EB01F4
:10C38000EF01F401F801FD010102050209020D02AD
:10C390001102140218021B021F02220225022802A7
:10C3A0002B022E023102340237023A023D023F02D2
:10C3B0004202450247024A024C024F025102530216
:10C3C000560258025A025C025F0261026302650271
:10C3D000670269026B026D026F02710273027502DD
:10C3E000760278027A027C027E027F028102830258
:10C3F00084028602880289028B028C028E028F02DE
:10C400009102920294029502970298029A029B026C
:10C410009D029E029F02A102A202A302A502A60201
:10C42000A702A902AA02AB02AD02AE02AF02B0029D
:10C43000B102B302B402B502B602B702B902BA023F
:10C44000BB02BC020000000000000000020000006F
:10C4500004000000001003EB0000000001000000D9
:10C460000100000004000000000100320000000094
:10C4700000000000000000000100000001000005B5
:10C4800000000000000000000000000001000000AB
:10C490000100003500000000010000000000000065
:10C4A0000400000000000020000000000100000067
:10C4B0000000000004000000000000D800000000A0
:10C4C0000100000000000000010000000000000664
:10C4D000000000000100000000000000010000005A
:10C4E0000200000100000000000000000000000049
:10C4F000010000000300009F000000000100000098
:10C500000000000001000000000000B90000000071
:10C51000010000000000000001000000000000AB6E
:10C52000000100FF010000FF000100FF010000FF0B
:10C53000FF00000100FF00010001000000FF00FFFC
:10C5400000FF00000100FFFF00FF010000000001EC
:10C55000010000FFFFFF01FF0101000000000101D9
:10C5600000030201000005020100000103010000B8
:10C5700003030100010003010001020301000200A6
:10C58000030100020203010003020301000304038C
:10C590000100040203010000000302000003030283
:10C5A0000000060302000100030200010303020071
:10C5B000010603020002010302000204030200025A
:10C5C0000703020003030302000001070300000643
:10C5D0000703000100040300010007030001040732
:10C5E000030001070703000200070300020407031A
:10C5F0000002070703000302070300030607030006
:10C6000004020703000406070300050104030005F4
:10C6100002070300050607030006000703000604DF
:10C6200007030006070703000703070300070707C0
:10C6300003000802070300080607030009020703B6
:10C640000009060703000A020703000A07070300A0
:10C650000B050703000C030703000C070703000D7D
:10C66000070703000E070703000E060704000E0766
:10C670000704030E070704030E070704030E07074A
:10C6800004030E070704030E070704030E0707043D
:10C69000030007000202010000020200040102027E
:10C6A000000701020202020002020101010202016E
:10C6B0000601020203050002020402000202020651
:10C6C0000102020300010202030501020205030048
:10C6D000020204050102020204020202020702022F
:10C6E0000205030102020506010202060001020220
:10C6F000060301020202050302020206030202010E
:10C7000006040202010607020202030402020203F7
:10C7100007020202060702020302070202030507DC
:10C7200002020307070202040704020205010402D1
:10C7300002050107020205030702020506070202BD
:10C7400006020702020605070202070107020207A6
:10C750000407020208010402020802070202080597
:10C76000070202090304020209040702020A000781
:10C7700002020A020702020A050702020A0707026A
:10C78000020B030702020B060702020C010702025A
:10C790000C040702020D010702020E000702020E3E
:10C7A000040702020F010702020F050702020E042E
:10C7B0000703030F030703030F070703030F07070D
:10C7C0000303000000020200000002020000000259
:10C7D000020000000202000000020200000002024B
:10C7E0000001000202000400020200070002020130
:10C7F000010002020104000202010700020202031A
:10C800000002020104010202010601020203050006
:10C8100002020204010202030101020203030102F7
:10C8200002040101020204040102020206020202E1
:10C8300003020202020106030202020203020201D3
:10C8400002070202010407020203030302020204B8
:10C8500004020202050702020301070202030504A3
:10C860000202040107020204030702020506030292
:10C870000205000702020502070202050407020280
:10C880000600070202060207020206050702020668
:10C890000707020207040702020707040202080250
:10C8A000070202080507020209010702020904073C
:10C8B00002020A000702020A030702020A0607022E
:10C8C000020B020702020B050702020C010702021B
:10C8D0000C050702020D020702020C010703030CFC
:10C8E000060703030D020703030E020703030E07E7
:10C8F0000703030000000202000000020200000023
:10C900000202000000020200030002020100000215
:10C9100002010200020200050102020202000202FC
:10C9200003010002020201010202020401020201EB
:10C9300002020202010402020203040102020202D4
:10C9400002020202050202020002070202000407BC
:10C9500002020006070202010207020201040702A6
:10C960000201060702020203070202020507020291
:10C970000302070202030407020204020702020480
:10C98000040702020406070202050107020205036A
:10C990000702020505070202060207020206040753
:10C9A0000202060607020207040702020801070244
:10C9B0000209000702020901070202090307020235
:10C9C0000A000702020A020702020B000702020B1A
:10C9D000020702020C000702020B060702020C0407
:10C9E0000702020C060702020D030702030C0007F0
:10C9F00003030C020703030C050703030C070703DB
:10CA0000030D050703030D070703030D07070303C2
:10CA10000D070703030D070703030D070703030DA6
:10CA2000070703030E0D0B07696E636C7564652FB2
:10CA3000647269766572732F6D6B5F6164632E63D8
:10CA400000696E636C7564652F64726976657273D4
:10CA50002F6D6B5F6165732E630033324B206C6FFB
:10CA60006164206361702076616C2025640D0A008A
:10CA70005854414C206C6F61642063617020766172
:10CA80006C2025640D0A00556E65787065637465C9
:10CA90006420646D61206368616E6E656C0D0A00D0
:10CAA000696E636C7564652F647269766572732F45
:10CAB0006D6B5F666C6173682E630052656C6F61AD
:10CAC000642076616C756520696D706F737369623F
:10CAD0006C650D0A00696E636C7564652F6472691C
:10CAE000766572732F6D6B5F6D6973632E63007370
:10CAF00079735F7469636B5F7374617274005265FC
:10CB000073657420627920756E6B6E6F776E20731B
:10CB10006F757263650D0A0025313064207C200D2D
:10CB20000A00437261736865642121210D0A002D9A
:10CB30002D2D2D2D2D2D2D2D2D2D2D2D2D2D2D2D25
:10CB40002D2D2D2D2D2D2D2D2D2D2D2D2D2D2D2D15
:10CB50002D2D2D2D2D2D2D0D0A00253038583A2044
:10CB60002530385820253038582025303858202591
:10CB70003038580D0A005052494D41534B3D253035
:10CB800038580D0A00434F4E54524F4C3D25303813
:10CB9000580D0A004D53503D253038580D0A0050AD
:10CBA00053503D253038580D0A0041495243523DFB
:10CBB000253038580D0A004C523D253038580D0AA2
:10CBC00000495053523D253038580D0A00785053D3
:10CBD000523D253038580D0A004E3D25642C205A10
:10CBE0003D25642C20433D25642C20563D25640DB5
:10CBF0000A0046494C45202020203A20005B534340
:10CC00005030335D005B464952415D005B555742F1
:10CC10005D005B4D41435D005B4343435D005B56FC
:10CC20004552424F53455D005B53455D005B5543A4
:10CC3000495D005B5741524E5D005B494E464F5D7A
:10CC4000005B4150505D005B4552524F525D005BAE
:10CC50004F535D005B424F4F545D005B544553544E
:10CC60005D005B4452565D005B5048595D00696E43
:10CC7000636C7564652F647269766572732F6D6B72
:10CC80005F74726163652E6300257300696E636C67
:10CC90007564652F647269766572732F6D6B5F754D
:10CCA0006172742E6300556E657870656374656497
:10CCB0002075617274202564207374617465202569
:10CCC0006400556E657870656374656420646D6199
:10CCD000206368616E6E656C20256400506172612E
:10CCE0006D74657220696E76616C6964007561723D
:10CCF000745F646D615F63616C6C6261636B00752E
:10CD00006172745F626175645F736574004F706512
:10CD10006E20414E5425640D0A006C73705F73637E
:10CD2000616C655F663332006C73705F675F6F7054
:10CD30005F663332006C73705F675F6F705F696E40
:10CD4000743136006C73705F675F6F705F696E740B
:10CD500038002E2E2F2E2E2F2E2E2F2E2E2F2E2E13
:10CD60002F647269766572732F6D6B5F6C73702EB2
:10CD700063004F706572616E6420616464726573F4
:10CD80007320257820697320696E76616C69640070
:10CD90004E656564206174206C65617374206F6EEC
:10CDA00065206F706572616E64005258204445536F
:10CDB0004320696E646578206973206F7665722000
:10CDC00072616E67650D0A00455420696E6465786E
:10CDD000206973206F7665722072616E67650D0A37
:10CDE000002E2E2F2E2E2F2E2E2F2E2E2F2E2E2F8C
:10CDF000647269766572732F6D6B5F6D61632E630C
:10CE0000006D61635F72785F646573635F636F6E0B
:10CE1000737472756374006D61635F65745F636FD3
:10CE20006E73747275637400556E646566696E65C1
:10CE30006420626974207261746520256420666FC5
:10CE400072206D65616E20505246206F6620256409
:10CE50000D0A004D45414E205052462070617261CE
:10CE60006D65746572206572726F720D0A00436F92
:10CE700064652069647820256420616E64206D6596
:10CE8000616E2050524620256420636F6E666C6987
:10CE900063740D0A002E2E2F2E2E2F2E2E2F2E2EA7
:10CEA0002F2E2E2F647269766572732F6D6B5F70F3
:10CEB00068792E630001000001000000FF00FFFF01
:10CEC0000000FFFF01000100010000FF01FF010160
:10CED0000001000000000101FF000000010000FF50
:10CEE0000000FFFF00FF01000100FFFF00FF010144
:10CEF0000100010100000001FF00010000FF00012E
:10CF000001FF000101010000FF010000010001001C
:10CF1000FF000101FF01FFFF010000000000000110
:10CF20000000000000FF0100000000FF00FF000003
:10CF300000FFFF01010100000100FF0100000100EE
:10CF40000001000000000000FF000000FF0000FFE3
:10CF5000FF000000FF0001FF0100FF0001FF00FFD4
:10CF600001000000000001FF0000010100FF0001BE
:10CF70000000FFFF0100000101FF010001FF0001AF
:10CF800000000000FF00FF00FF00FF0101FF0100A3
:10CF9000010000010001000000FF0100010101008B
:10CFA0000000FFFFFFFF010101000000000101017F
:10CFB00000FFFFFF01FF00000000010000FFFF0075
:10CFC00000000000FF000100010001FF000100005F
:10CFD0000100000100FF0000FF010101000001004D
:10CFE0000000FF01000100FF00000000010101013D
:10CFF00001FF010001FFFF0001FF000101FFFF0031
:10D00000FF0000000100FF010000010001FFFFFF21
:10D01000FF000000FF000000000000FF0100000111
:10D02000FF0001010000000101FF00000101FF00FD
:10D03000FF00FF01000101000000000000FF0001EF
:10D0400000FF0100FFFFFF01FF01010000FF0100E1
:10D050000101000100010001000000FF0000FF00CD
:10D0600000FF01000001FF0101000000FF01FF00BF
:10D07000FF010100FF000101010100FF0000FF00AE
:10D080000101000001000100000101FF000001009A
:10D09000000001FF000000FF00FFFF010000000092
:10D0A000FF00000000FFFF0001000000000001FF82
:10D0B000FF01000000FFFF00000000FFFF01010072
:10D0C000FF0101010100FF000101000100FF00005C
:10D0D000FF0100010100000101FF0001010001FF4B
:10D0E0000100FF0000010000FF00FFFF000000FF43
:10D0F00001FF00000100000000FF000101FF00002F
:10D1000000000001FF00FF000000000000FF000021
:10D11000FF01FF0101FF01000000FF00010001000D
:10D12000010101FF0000FFFF0000010001000000FD
:10D1300001000000010100FF000100FF000001FFED
:10D1400000FF0100FF0000010001000000000100DD
:10D1500001FF0000000001010000010001010101C8
:10D1600001FF0100FF0001FF00FFFF01000101FFBF
:10D17000FF000000FFFFFF000100000001000100B0
:10D18000FF01FF00000000000001FF01FF00FFFFA2
:10D1900000000101000000FF00000100000101FF8C
:10D1A0000000FFFF0101FF0000FF00000000000081
:10D1B00001FF00000100FF000000FF01010000006E
:10D1C00000FFFFFF0101000000010001FF00FF015F
:10D1D0000000FF01000000FFFF00FF0000FFFF0054
:10D1E000FFFF010101FF0100FF0101000001FF013C
:10D1F00001000100000000000100FF00010101FF2B
:10D20000000001000001000000FF0000000001001C
:10D2100000FFFF010001010001000100FF0000FF0D
:10D2200000FF01FF000100010100000000000101FA
:10D23000000000000100000001000001FFFF0001EC
:10D24000FF010100FF000000FFFF000001FF0001DF
:10D2500000000101000000010101000001000100C7
:10D26000FF00FF01FF00FF000100000100000100BE
:10D270000101FFFFFFFF0100000101FFFF010001AD
:10D28000FF00FFFF01000000000000FF00FF0000A2
:10D290000000FF0100FFFF0000010000000000018E
:10D2A000FF0101000000FF00FF0100010001FFFF7E
:10D2B000000000FF00FF0000000001FF0000000070
:10D2C000000100000000000001FFFF01FF0101005C
:10D2D000FF00010001000001FF000001010100FF4B
:10D2E000010100FF00000100FF010000000101003A
:10D2F000010101FF00FFFF00010001FF00FFFF002F
:10D3000000FF000001000000FF010100000000011B
:10D31000000101FF01FF00000100010001FFFF000B
:10D3200000FFFF00FF00000001000001FFFF0001FF
:10D33000010100000000010101FFFFFFFF000000EC
:10D340000101010001FF00000001000100000100D7
:10D3500001FF0101FF00FF00FF00FF0000000001CE
:10D3600000FF010001FF0101000001FFFF000001BB
:10D3700000FF0001010000FF01000000000001FFAC
:10D3800000FF0100FF0001FF0100FF000000FFFFA0
:10D390000000FF000000FF0000000000000100008E
:10D3A00001000001FF000100000101FF00FF010179
:10D3B0000000FF0101000000010100FF0100000169
:10D3C000FF000000000000FF000000FFFFFFFF0162
:10D3D0000001000001FF0001000000FF00FFFF014D
:10D3E0000100FF0100FFFF010001FF010101010138
:10D3F00000000000FF00010001FF0000000100002C
:10D40000010101FF0000FF00010000010000010018
:10D41000FF010001000100FF0000000000FFFF000D
:10D42000000100000000FF01FF00FFFF01000000FD
:10D4300000000100FFFF00000000FF0000000001ED
:10D44000FFFF00FF000000FF01000000010000FFDF
:10D45000010100000100010000010100FF0000FFC8
:10D46000000101010100FF000101FF00FF01FF00B9
:10D4700000000101FF01000001FF0000FF0000FFAC
:10D4800000000001000100010001010001FF000097
:10D490000101FF01FFFFFF0001FF000100FF00008D
:10D4A0000000000001010001FF0100010000FFFF7A
:10D4B0000000FF0101010001000100FF0000000168
:10D4C000FF0101FF01FF0000FF000000000000FF5E
:10D4D00000FF010000000000FF010100FF0000004C
:10D4E00000010000FF01FF000000FFFF00FF00003F
:10D4F000010000FF0001FF0100010100FF01010028
:10D500000001010001FF0000FF000100010100FF18
:10D510000001010101FF000101FFFF00000000FF09
:10D52000FF0000000100000000FF0000FF0101FFFC
:10D53000FF0000FF01010000010000FF00000001EA
:10D54000010000FFFF00FF01FF01000000000000DC
:10D55000FF01FF000100010000000100FFFFFF00CC
:10D560000000FFFF01010001FFFF00FF0100FF00BD
:10D5700001FF0101010101000100000101000000A3
:10D5800000FF010001000000000100010000FF0099
:10D5900001FF00FF010000FF000100FF000101008A
:10D5A000000001000000000000000101000100FF78
:10D5B00001FF00FF0000FF00010001000101000168
:10D5C000FFFF00000100000000FF0000000100005C
:10D5D000010000FF01010100FF0001000000000048
:10D5E00001000101FF0100000101FF0001FF010135
:10D5F00001FFFF00FFFF0000FF00FFFF0000000130
:10D60000FF000001FF00FF0100010000000101FF19
:10D61000FFFF000000000101FF000000FF0001000B
:10D6200000FF01000000010001FF00FF00000001F9
:10D6300001FF010000000000010000FFFF0001FFEA
:10D6400000000000FF00FF00000000000001FFFFDD
:10D6500000FF010001FFFF0101000001FFFFFFFFCC
:10D660000101000100000100000100FF00FF01FFB7
:10D6700000FF0001000100000101010000000101A4
:10D6800000000100FF010000FFFF000000FF00019B
:10D6900001FF0100FFFF0100000100000001000088
:10D6A0000000010100FF000000000100FF00010177
:10D6B000010001FF00000001FF0101010000FF0166
:10D6C00000FF000000010001FF0001000100000058
:10D6D000FF010100FF01FFFFFF0000010000010149
:10D6E000000000FF01000101000000FF01FF010137
:10D6F0000000010100010000FF00000000FF000128
:10D7000000FF0000000001FF0000FF0000FF01011A
:10D7100001010001FF010000000100FF0001010004
:10D72000FFFF0001FF0000010101FF01000000FFF9
:10D73000010001010100FF000100000000FF0000E6
:10D7400001010000010000FFFFFF01FF000101FFD8
:10D7500000000001000100FF0100010000000001C5
:10D760000000000001FF00010001000001000000B6
:10D7700001000101FFFFFF00FF010000FF010001A8
:10D780000000FF00FF00010100000000FFFF01009A
:10D7900000FF01000101FF010100010000FF000185
:10D7A000010101FFFF01FFFF01FF01010101FF0175
:10D7B000FFFFFF0101FFFF010101010101FF010165
:10D7C000FF01000001FFFF0100FFFF010001010157
:10D7D0000101FFFF010101FFFF00FFFF0001FF0149
:10D7E000FFFFFFFF00FF01FF01FF010001FFFF013D
:10D7F00001FF01FF0101010001010001FF01FFFF25
:10D80000FF0101010101FF01FF0101FFFF01FFFF16
:10D810000101FFFFFF01FF0001010100FF01010104
:10D8200001FF01000100FFFF0001FF0101FF0101F5
:10D8300001010101FFFF01FF01010000010101FFE2
:10D84000FF0001FFFFFFFFFF01FF0001FF01FF01DC
:10D85000FFFFFF010101FFFF010101FFFFFF01FFCA
:10D8600001FF00FF01FFFF000101FF01FF0100FFB9
:10D8700001010101010101010101FFFF01FFFF01A0
:10D8800001FF0101000101FF01FF01FFFF01FFFF97
:10D89000010101FFFFFF00FF010101FF0001000086
:10D8A000FFFFFF0101FF01FFFF00FF010100010178
:10D8B000010101FFFF010101FF0101FFFFFF01FF66
:10D8C00001FFFF000101FFFFFF01FF010001FFFF5A
:10D8D000FFFFFF0100010101FFFF01FF01FFFF0149
:10D8E000FF0101FF0101010100FF00FF0101000034
:10D8F00001FF010101FF0101FF0100FF0100FFFF26
:10D9000001FFFFFF010101000101FF00FFFF01FF17
:10D910000101FFFF00010100000101FF0101FFFF04
:10D92000FFFFFF010101010101FF0001FFFF01FFF6
:10D930000101FFFF01FF010101FFFF0101010101E1
:10D940000101FF0101010001FF01FF00FF00FF01D4
:10D9500001FFFFFF0100FFFFFF010100FF01FF01C9
:10D96000FF0101FFFF010100FFFF000101FF0000B7
:10D97000FFFF0101FF0101FF01FFFF0101010101A3
:10D98000FFFFFF010101FF01FF0001FF01FF010097
:10D990000101010101FF010101FF010101FF01007E
:10D9A000FFFFFFFFFFFF0101FF0101FF0100FFFF7C
:10D9B000FFFF01FF01FF00010001FF010101FFFF67
:10D9C00001FF010100010101FFFF0101FF00010151
:10D9D0000000FFFF0101FFFF010101FF01FFFFFF49
:10D9E000FFFFFF00010101FF0101010101FFFF0134
:10D9F000FF0101FFFFFF01FF01FFFFFF01FF01002A
:10DA0000FF01FFFF00010001FF0101FF0101000113
:10DA1000FF01FFFF000101010101FF0101010101FF
:10DA2000010101010101FFFFFF01FF0101FFFF01F2
:10DA3000010000FF01FF0100FF01FF00FF0101FFE6
:10DA4000FF010101FF01010100FFFF000101FF01D2
:10DA5000FF01FF00FFFFFF0101FF00FFFFFFFF01CC
:10DA6000010101FF01FF000100FF01FF0101FF01B2
:10DA700001FFFF01FF040000040404040404040483
:10DA800000000000A8DA000008900102180500005C
:10DA9000800B000080DC0000209501026829000056
:10DAA000BEBF00000000000052033280420133017B
:10DAB00001C20702100352015526B8030145900028
:10DAC00050084202C203001515C0C1C2C3C4C5C676
:10DAD000C7C8C9CACBCCCDCECF000101013C018063
:10DAE0000302090203020201013302036509020372
:10DAF00001420257140019412717901D070605041B
:10DB000003020100F29798DDC89D5CB81CC0DEA737
:10DB1000DB615BCA010200035240480510040601A4
:10DB20000001522D2C280004007C007B010502031B
:10DB300008FF5B0F010065F901417B0707010160E8
:10DB4000002000881333E0536420ACFF501B0D0706
:10DB50000E080E080E080E080C030D050B050D0728
:10DB60000D070D070D0701012E010402004003FF00
:10DB7000FF7F00FFFF7F0816FFFFFF00FFFFFF3A58
:10DB8000010001000A00010106401E4005120512B5
:10DB9000000515040201020301024004020103030F
:10DBA000020C0E0900087A0232413428002A82034E
:10DBB00003455006C570014013E620700140144C27
:10DBC00007001000D6FF00B000500B420282034550
:10DBD000FFFF0F20320442083201045510000134C7
:10DBE000B400030550200050079D280004000102E6
:10DBF0000100FFFFFFFF3790900102F3C8005115AD
:10DC00001EC135BF80F3E2BDC0B464BF871699BDA5
:10DC1000AD178DBF941799BD33A876BFC4780DBDDD
:10DC20002BC162BA0CB0AFBEA9F6E9BAFC567BBEF6
:10DC300007254CBBEC8823BE5DC0CBBB0CCE20BD02
:10DC40007BA095BCD40F3A3E2D5EACBD5913073F67
:10DC500064010042420944030006320145100140BC
:10DC60000FC20E520145900140184204023D054585
:10DC7000A00140194206023D07454001400D8201C6
:020000040000FA
:10DFC000A5A54B4D0000001000000002AAAA5A7F30
:10DFD000C0DF0000000000000200000000000000A0
:10DFE0000000000000000000000000000000000031
:10DFF0000000000000000000000000000000000021
:10E0000058E00000000000000A56656E646F720957
:10E010003A204D4B53454D490A43686970093A20EF
:10E020004D4B383030300A44617465093A205365ED
:10E030007020203420323032340A56657273696F92
:10E040006E093A2056302E362E32000000000000B5
:08E050000000000000000000C8
:04000005000000C136
:00000001FF
